:020000040000FA
:040000006FD00400B9
:101000006F00107D00000000000000009020002014
:10101000AA220020A9BDF9F56C23002000000000E1
:10102000000000006C230020902000200000000041
:101030000000000090200020000000009020002010
:101040000000000090200020902000209020002030
:101050009020002090200020402F00207A240020A3
:101060000000000090200020902000200424002098
:1010700090200020D22300209020002090200020EB
:101080009020002090200020902000209020002020
:101090009020002001A04111B7170040985F3AC688
:1010A000945F3247E39CE6FE3245410182800111A4
:1010B00013078008F337078093F787083EC20100C3
:1010C0000100B7170040930570052380B70413068D
:1010D00080FA2380C7040100010083C6B70493F699
:1010E000F60DA385D704238007049246F3A6068055
:1010F0000100010093760502D5CEF336078093F602
:10110000860836C4010001002380B7042380C70489
:1011100001000100B70614007D89558D88C70100C4
:1011200001000100010023800704A246F3A6068007
:101130000100010073370780137787083AC6010062
:1011400001002380B7042380C704010001000100CF
:1011500001003727004093061005A303D7802380A2
:101160000704B247F3A70780010001009307800836
:10117000F3B7078093F787083ECE01000100B71749
:101180000040130770052380E704130780FA2380CB
:10119000E7040100010003C7B70413670708A3852C
:1011A000E70423800704F247F3A70780010001004A
:1011B0000561828093760504BDC6F336078093F6F9
:1011C000860836C8010001002380B7042380C704C5
:1011D00001000100B7061400938606047D89558D31
:1011E00088C7010001000100010023800704C246F6
:1011F000F3A6068001000100733707801377870884
:101200003ACA010001002380B7042380C70401000B
:1012100001003727004093062005A303D7802380D1
:101220000704D24781B773370780137787083ACC12
:10123000010001002380B7042380C70401000100DE
:1012400098471367070C98C723800704E24719BF24
:101250000111814601468145114506CE97000000E7
:10126000E780C05693078008F3B7078093F7870895
:101270003EC601000100B717004013077005238028
:10128000E704130780FA2380E7040100010003C785
:101290006704136717002383E70423800704B2471A
:1012A000F3A7078001000100F2400561828041112F
:1012B000814601468145114597000000E7800051B5
:1012C00013078008F337078093F787083EC40100AF
:1012D0000100B7170040130670052380C70493066A
:1012E00080FA2380D70401000100FD552396B70240
:1012F00023800704A245F3A5058001000100733790
:101300000780137787083AC6010001002380C704CD
:101310002380D7040100010003C767041367170087
:101320002383E70423800704B247F3A70780010063
:10133000010001A0B1473305F50201007D1575FDDF
:101340008280411122C426C206C6AA8401446317C2
:101350009400B24022449244410182800504130566
:10136000803E420497000000E78000FD4180C5B741
:101370009305000273A04580824573901534924016
:101380002242B2424243D2436244F2440255925551
:101390002256B2564257D2576258F25806499649D9
:1013A000264AB64A464BD64B664CF64C065D965DD1
:1013B000265EB65E465FD65F09617300203041113C
:1013C000B7170040985F3AC6945F3247E39CE6FE49
:1013D000324541018280B71700401307000323887C
:1013E000E702854717170000232EF74473002030CB
:1013F000411122C406C637040020976000E0E78050
:1014000060441C408297D5BF373700408347470070
:101410009146BD8B639ED702B73600401306F00F8E
:10142000973500009385051F9737000083D7872ED7
:1014300003C7A6001377F70F1DE3B7E70400BC4FFF
:101440000946894517150000034585F7829731A0A5
:1014500099466394D700834757007300203003C731
:1014600086001377F70FE365F6FC13851700AE9738
:10147000173800002310A82A2380E70075B7B78724
:10148000004003C76700098B6309071003C7770093
:101490009306000313770703630DD708173800007E
:1014A00003481875173600001306C6730547B306C0
:1014B00006012380E60083C5770017370000130775
:1014C000E772429793F5F50F2300B70003C5870035
:1014D0009735000093854571C2951375F50F2380EC
:1014E000A5000347070089451377F703630CB70C82
:1014F00063E7E50A6306071A8545630CB712973759
:10150000000083C7F76E3307F60003470700137721
:10151000F70F19CB850793F7F70F0D476363F71A9A
:1015200017370000A306F76CB787004009472383ED
:10153000E700B787004083C77700E207E18763DEF3
:1015400007049737000083C7B76A173700001307EF
:1015500067693E9785462300D700173700001307B9
:10156000E7683E97930600032300D7001737000073
:10157000130787673E97A14685072300D70093F797
:10158000F70F0D476364F71417370000A302F766DF
:10159000B787004009472383E70073002030930694
:1015A00010026300D70E930620026305D706930648
:1015B0000002E316D7F403C727021377C70F136798
:1015C0002700D5A803C767001377070465CB03C7B7
:1015D000A70217380000130828421735000013052A
:1015E0006539134707082385E70203C7A702137766
:1015F000370F136787002385E7028147130700042D
:10160000B305F5008C41B306F80091078CC2E3994D
:10161000E7FEF5B503C7A702134707042385E702D2
:1016200003C7A7021377C70F136727002385E702B5
:10163000F9B503C767001377070449C303C76702F7
:10164000173800001308082F17350000130545262A
:10165000134707082383E70203C767021377370F8F
:10166000136787002383E702814713070004B3054C
:10167000F5008C41B306F80091078CC2E399E7FEB0
:10168000BDBD03C76702134707042383E70203C7EF
:1016900067021377C70F136727002383E70285B517
:1016A00003C767001377070411CB03C7270213771B
:1016B000370F136787002381E70291B52380060067
:1016C0003DBD97370000A3850752B9BD973700008D
:1016D000A380075275BD2303048015472303E480CC
:1016E00001002302A480828083076480E3CE07FE8A
:1016F00023030480828083076480E3CE07FE0345D2
:101700004480828083076480E3CE07FE2302A480A6
:101710008280411126C44AC24EC006C61377F50B1B
:10172000AD47AA892E899544630CF70019459700A7
:101730000000E78080FA97000000E78020FB8D44DE
:101740004E8597000000E78040F9FD59FD1463982D
:101750003401B240A24412498249410182801355AA
:1017600009011375F50F97000000E780E0F92209E1
:10177000F1BF011126CC06CEB70408009700000087
:10178000E780C0F6154597000000E78000F5970058
:101790000000E78080F697000000E78000F62AC688
:1017A00097000000E78080F432459377150089EBBD
:1017B000136515001375F50FF240E2440561828050
:1017C000FD14E9F00145CDBF397126DC4ADA4ED867
:1017D00052D656D45AD25ED006DE62CE66CCB7E779
:1017E00000E07D5783AA070022C603AA470023A072
:1017F000E71823A2E718B7170040130770052380E6
:10180000E704130780FA2380E70483C74704930B98
:1018100075FFB684E20793FBFB0F8546AA892E8BE2
:10182000328937240040E187015763FA7601630863
:10183000D5008946130700026313D5000157D98FDD
:1018400093F7F70FB71C00402382FC0411472303D2
:10185000E4801305F00F97000000E78000E8094CD2
:1018600097000000E78080E863657C15B7050700F6
:10187000DA9537870700795563FEE504B38795004D
:10188000636AF704370B0800A94733EB65016395DA
:10189000F90881E8814497000000E78020E526856B
:1018A00015A8DA85094597000000E780C0E605091C
:1018B0000345F9FFFD14050B97000000E780C0E425
:1018C00081C49377FB0FE5F797000000E780A0EA5B
:1018D00069F17D55B7170040130770052380E704B1
:1018E000130780FA2380E70403C74704418B238250
:1018F000E704F250B7E700E023A0571123A24711F5
:10190000E25432445259C259325AA25A125B825B93
:10191000724CE24C21618280A547639BF906856980
:101920001309F00FB3069900B3742B01B694134951
:10193000F9FFB3749900856B33796901416B938723
:10194000F9FFB3F7270199E363FC340193D9490008
:10195000C147E3E637FF3DBF0569C1697D19D9B7C6
:101960001305800D63886901130500026384790102
:1019700013051008CA8597000000E780C0D99700BA
:101980000000E78040DF31D54E99B38434416DBF0C
:10199000DA852D4597000000E780E0D7CA94E30B75
:1019A00099EE050997000000E78020D5A30FA9FE56
:1019B000FDB79387F9FF93F7F70F636DFC0C83C7AF
:1019C0001C04130730086315F70637070800636126
:1019D000EB06B3079B00B706100063FBD704334B3D
:1019E000EB0089476399F9068980D549E38404EAC5
:1019F000DA85094597000000E780E0D11109032747
:101A0000C9FF91472320E48003076480E34E07FE6B
:101A100023033481FD17EDFBFD14110B81C4937773
:101A2000FB0FE9FF97000000E780E0D461F155B5B6
:101A3000B717004003C75704B7070800137707021A
:101A400019E3B78707007955E376FBE833079B0076
:101A5000E3F9E7F841B58547E380F9F0DA852D45EC
:101A600097000000E78020CB9389F4FFE38404E231
:101A700097000000E78060C893F7390091EB832658
:101A800004800327090093074900E396E6E03E89B6
:101A9000CE84D9BFB5476399F9001305900B970021
:101AA0000000E78080C3FDB3B1471305B00AE388A7
:101AB000F9FE99476397F904B7050800B365BB00C1
:101AC0002D4597000000E78000C581448D4BA1495A
:101AD00097000000E78060C263967401832704804A
:101AE0002320F9008504E39534FF8327048013172E
:101AF0002B01635507002312F90069BB2322F9006B
:101B000051BB9D47639FF90281451305B0049700BF
:101B10000000E78040C0BD442320090023220900C3
:101B2000FD5997000000E78040BD93F77400CA9705
:101B300003C70700FD14398D2380A700E39334FF0A
:101B400091BBA1476397F90697000000E780A0C208
:101B50008144630D0B008D479304C0036308FB00B1
:101B60009304000563048B01930440041375C507B7
:101B7000E30295D2194597000000E78000B6970070
:101B80000000E780A0B6054597000000E780E0B4BC
:101B9000268597000000E78020B7094597000000E0
:101BA000E78080B697000000E780E0BCE31405CE34
:101BB0000DB39147639FF90013056006970000007D
:101BC000E780A0B197000000E78040B213059009BC
:101BD000F9B5E38109CCF1547DB9BD6601471736EB
:101BE00000001306261E938606A685458347060039
:101BF00093F7F70F91C382800507E3F9E6FE973765
:101C000000002381B71CDDB77D166206618693173D
:101C10008601E18763D4070001458280931726007F
:101C20003307F500AE9718439C4363E7E7007D1642
:101C3000E37FF7FC7D55828005458280FD15E20536
:101C4000E18513978501618793F7F50F63480700D6
:101C5000FD15139725002A97584365D7138517005C
:101C60006205618582803308B5021C4283A80600A4
:101C7000B335B502C29733B50701AE98469585488E
:101C80006367B5006394A50063E3070181480C43D3
:101C9000C6950CC388C21CC28280814713978701F6
:101CA00061876343B7008280139727002A97232018
:101CB00007008507E5B78147014793968701E186CD
:101CC00063C5B60013351700828093962700AA9645
:101CD00094428507558FD5B793D755408A07AA9761
:101CE0009C4305453315B5007D8D828017F3FFDFDA
:101CF000E702A33D2A8497000000E78060F405C551
:101D0000931725003E940327C4FF814711EB7D15EF
:101D100016053E954205418517F3FFDF6700233D19
:101D200005838507E5B70145C5BF8147139787013F
:101D300061876343C700828013972700B386E5005D
:101D400094422A97850714C3D5B77D16620661862B
:101D5000014793178601E18763D507001335170004
:101D6000828093172600B306F500AE9794429C43F9
:101D70007D16B58F5D8FF1BF8A05AA950147636314
:101D8000B500828083A6C5FFF11593D71600D98FC1
:101D90009CC11397F601E5B72A8301480147014525
:101DA0006343D7008280B387050183A80700B30788
:101DB00006019C43C697AA976384F80033B51701C0
:101DC0000507B3080301620723A0F8006187110823
:101DD000C1BF2A8301478147014563C3D700828081
:101DE0003388E50083280800330EE600032E0E003A
:101DF0003388A8403308C8416384080133B508011B
:101E00008507B308E300E20723A00801E187110773
:101E1000E9B717F3FFDFE702432B0111B286B28463
:101E20002E86AA850A8597000000E780C0FA2A84DA
:101E3000A6850A8597000000E78020E833348000FB
:101E4000060413351500018D056117F3FFDF6700E8
:101E5000032A17F3FFDFE702C3244111AA89AE8AE0
:101E6000328BB68402C202C402C60144131C840130
:101E7000135C8C4163499C02939B1400FD1B054934
:101E8000138CF4FFF15C33048901620461846340C4
:101E9000740792478E04CE9423AEF4FE410117F3EB
:101EA000FFDF6700832313192400B30B2B01014AC2
:101EB00093172A00D69783A50B0088437800340037
:101EC000500097000000E78040DA050A93178A0166
:101ED000E187F11BE35EFCFC92474E990504232049
:101EE000F900A2473EC2B24702C63EC441B7131A28
:101EF0008901135A8A41131D240093178A01E1872F
:101F000063CF970092470A044E941CC0A24705096C
:101F10001379F90F3EC2B24702C63EC4ADB7B3074C
:101F20009A0313152A005695084178003400500092
:101F3000050AEA97DA978C4397000000E780E0D221
:101F40006DBF0000197106C212C416C61AC81ECA97
:101F500022CC26CE2AD02ED232D436D63AD83EDA69
:101F600042DC46DECAC0CEC2D2C4D6C6DAC8DECA99
:101F7000E2CCE6CEEAD0EED2F2D4F6D6FAD8FEDA49
:101F8000971500009385858B8841E70005009240F6
:101F90002242B2424243D2436244F2440255925535
:101FA0002256B2564257D2576258F25806499649BD
:101FB000264AB64A464BD64B664CF64C065D965DB5
:101FC000265EB65E465FD65F096173002030000072
:101FD0009721002093810103175100201301818272
:101FE00017F5FFFF1305450297050020938585012E
:101FF000171600201306C6FD63FAC50083220500EC
:1020000023A0550011059105E3EAC5FE170502005E
:102010001305C541971500209385C5FB17160020B1
:102020001306466563FAC5008322050023A0550008
:1020300011059105E3EAC5FE171500201305856318
:1020400097450020938505246377B500232005007C
:102050001105E36DB5FEFD42739002BC8D42739095
:102060004280B722000093828288739002309702E8
:102070000020938222F993E23200739052309752FB
:1020800000009382C29E739012346FB07477730015
:102090002030397101436EC619A0397141536AC8A5
:1020A00066CA62CC5ECE19A0397101535AD056D29D
:1020B00052D44ED64AD826DA22DC06DE33016140FD
:1020C000828241114AC026C222C406C68282B24D13
:1020D0004101024D924C224CB24B4101024B924ABB
:1020E000224AB2494101024992442244B24041018C
:1020F00082803D432A876373C3029377F700BDEF65
:10210000ADE5937606FF3D8ABA960CC34CC30CC767
:102110004CC74107E36BD7FE11E28280B306C34090
:102120008A069702000096966780A6002307B700EC
:10213000A306B7002306B700A305B7002305B70021
:10214000A304B7002304B700A303B7002303B70019
:10215000A302B7002302B700A301B7002301B70011
:10216000A300B7002300B700828093F5F50F939684
:102170008500D58D93960501D58D61B7939627007F
:102180009702000096968682E78086FA9680C117AD
:102190001D8F3E96E374C3F8A5B73367B500FD53B2
:1021A0000D8B79E7B7877F7F9387F7F710419441CD
:1021B000B372F6003363F600BE92B3E26200639737
:1021C000720C6318D6065041D441B372F6003363E3
:1021D000F600BE92B3E262006398720A631BD604F3
:1021E00010459445B372F6003363F600BE92B3E235
:1021F00062006391720A631ED6025045D445B372E1
:10220000F6003363F600BE92B3E26200639A72088E
:102210006311D60210499449B372F6003363F60095
:10222000BE92B3E26200639372085105D105E30FD9
:10223000D6F61317060193970601631CF700135790
:10224000060193D706013305F7409375F50F91E921
:1022500082804183C1833305F7409375F50F91E187
:1022600082801377F70F93F7F70F3305F7408280DB
:102270000346050083C60500050585056313D600E2
:1022800065FA3305D640828011059105E312D6FE2A
:10229000014582802105A105E31CD6FC0145828011
:1022A0003105B105E316D6FC014582804105C10523
:1022B000E310D6FC01458280B717004003C77705BD
:1022C0001377E70FA38BE704130700F8A38DE70448
:1022D0003D47238CE70413075003A38CE70403C78F
:1022E000A7051377D70F238DE7048280B717004027
:1022F00003C7E7020D8941111377C70F498F930672
:102300008008F3B6068093F6860836C60100010001
:10231000930670052380D704930680FA2380D704A0
:10232000010001002387E70223800704B247F3A7D7
:102330000780010001004101828041112A83014E82
:10234000930E407E130F0019930F400663E56E1243
:102350009308001913034006B3781503854E0D4FFB
:10236000A14F337365020D891335150063EFBE125B
:102370001308F6FF7946729842081358080133078C
:10238000C70213D61700BE0732976146B3F6C602DE
:1023900013068070B386C6023697A166F58F420792
:1023A0005D8FB716004083C7F60293F70708A303B3
:1023B000F1000346710083C7F60293F70708E39420
:1023C000C7FE83477100B716004093F7F70F638885
:1023D000071293078008F3B7078093F787083EC476
:1023E00001000100B7170040930670052380D70451
:1023F000930680FA2380D7040100010023AA070373
:1024000083C6170393E60608A388D7022380070430
:10241000A247F3A70780010001001166B71700402B
:102420007D16D45BC85F93854703A98EF18EF5FABC
:1024300093068008F3B6068093F6860836C6010038
:102440000100930670052380D704930680FA238049
:10245000D7040100010098C103C7170313670704DD
:10246000A388E70223800704B247F3A7078001008F
:102470000100410182807D133368E3039308E01675
:10248000630E08003368F3039308D016630808004E
:102490009378330093B818009388D81633081E0138
:1024A000131E0801135E0E0155B56393E50305483D
:1024B000638608000148630303002A887108729844
:1024C000FD15131E0801C205135E0E01C18179BD01
:1024D00013F8150063F4BF007908D5B71338180056
:1024E000E5BF83C7F60293F70708A303F10003468D
:1024F000710083C7F60293F70708E394C7FE83478A
:10250000710093F7F70FF1DFE9B531714AD966CB66
:1025100006DF22DD26DB4ED752D556D35AD15ECF09
:1025200062CD6AC96EC7AA8C02D897100000E780F6
:1025300020B12A8993078008F3B7078093F78708AB
:102540003EDA01000100B717004013077005238031
:10255000E704130780FA2380E7040100010003C7A2
:10256000F7021377770FA387E70203C7F702136712
:102570008700A387E70223800704D257F3A70780C9
:1025800001000100054597000000E78060D61307B1
:1025900080C13347E902116A93070AE893065002A3
:1025A000BD69930BA004814A014B13048008930476
:1025B00070057D1AB347F9023307D7023EC0FD8785
:1025C0003ECC938709A69309803E3347F7023AC26F
:1025D0007D873AC4334739038549B399990193D923
:1025E0003940B306D702B30B7703B3C6F602B3CBB9
:1025F000FB0236C6FD8636C893D6FB4136CEB746BB
:102600000F00938606243349D9028566938606FA1D
:10261000B3969601B389E902130760553309D902CD
:1026200093060010B389E9023349D902B3C9F9020C
:102630009316390036CA37190040FD8636D0930DFF
:10264000090493D7F9413ED2F336048093F6860805
:1026500036DC01000100930770052380FD0093061E
:1026600080FA2380DD00010001008346390593F6DE
:10267000860FA309D9048346390593E61600A309FA
:10268000D90423800D00E256F3A606800100010064
:10269000130C80FA116DF336048093F6860836DE4B
:1026A00001000100930770052380FD0023808D0148
:1026B0000100010083463905216693E60602A3095D
:1026C000D90483560905B3E6A6012318D904835615
:1026D0000905D18E2318D90423800D00F256F3A6E4
:1026E0000680010001008346390593F606026381E6
:1026F000061A03463905218A6DDE08189710000076
:10270000E78000987336048013768608B2C2010011
:10271000010023809D0023808D0101000100B71777
:10272000004003C637051376F60DA389C70403C618
:10273000370513660602A389C70483560905216677
:10274000B3E6A6012318D90483560905D18E2318B0
:10275000D90423800D009646F3A6068001000100EF
:102760008346390593F60602638B061483463905C2
:10277000A18AEDFE97000020E780E091AA8636D47A
:1027800097000020E7802091A256E30AD5FE8356E9
:1027900009054255B3E6A6012318D9049710000095
:1027A000E780C08F83463905A18AEDDE035609050F
:1027B0008346290582473376CA00B306DA0293D5E9
:1027C000F641B296B388F640E24733B8C6002E9879
:1027D0003308F840A247B3B616013308D84063C7A0
:1027E0000701631DF800924763FA1701C247634F60
:1027F000F80E63950701B24763EAF80E894663E96C
:10280000660FF2469315180013D3F8015E861395F0
:102810001800B365B30042D646D497C00100E780E4
:1028200020DE3258050B137BFB0F63470001631A50
:102830000838A2586387083813081500B336A80073
:10284000B69513D6F5013298B336C800AE96135834
:102850001800FE06B3E60601733604801376860878
:10286000B2C60100010023809D0023808D0101007C
:1028700001000356C902B296C206C1822316D902CC
:1028800023800D00B646F3A606800100010021B5A5
:10289000F336048093F68608B6C001000100238059
:1028A0009D0023808D01010001008346390593E6D8
:1028B0000602A309D90423800D0086460DB5F33620
:1028C000048093F68608B6C40100010023809D00B1
:1028D00023808D01010001008346390593E606023D
:1028E000A309D90423800D00A646BDB5E30B0BF068
:1028F000F336048093F68608B6C8010001009306FB
:1029000080FA23809D002380DD00010001008346C2
:10291000390593F5FC0F93F6860FA309D904834676
:102920003905CD8EA309D90423800D00C646F3A630
:10293000068001000100130580FA0346390593065D
:1029400039051D8A631C9629733604801376860820
:10295000B2CC01000100130680FA23809D00238081
:10296000CD000100010003C606001376F60D23809A
:10297000C60003C60600136606022380C6008356FF
:1029800009051166D18E2318D904835609052166DD
:10299000D18E2318D90423800D00E646F3A60680C5
:1029A00001000100130680FA8346390593F60602FA
:1029B0006380062683463905130C3905A18AFDDAA2
:1029C000081897000000E780A06BF336048093F6A8
:1029D0008608B6D001000100930680FA23809D008E
:1029E0002380DD000100010083460C00116693F690
:1029F000F60D2300DC0083460C0093E6060223005C
:102A0000DC0083560905D18E2318D90483560905A5
:102A10002166D18E2318D90423800D008656F3A693
:102A2000068001000100130680FA8346390593F6FB
:102A30000602638A062083463905A18AEDFE97F0D7
:102A4000FF1FE78040652A8C97F0FF1FE780A06496
:102A5000E30C85FF8356090511664255D18E231874
:102A6000D90497000000E7806063834639051306A8
:102A70003905A18AFDDAF336048093F68608B6D4C8
:102A800001000100930680FA23809D002380DD0071
:102A9000010001008346060093F6F60D2300D600E0
:102AA00023800D00A656F3A6068001000100835680
:102AB000090503462905D247B376DA003306CA0270
:102AC0001305800C9355F6413696330DF640825728
:102AD000333CD6002E9C3336A601330CFC40330C1D
:102AE000CC403308850392564E86B335A503330593
:102AF000A503C29597C00100E78080B063468001BE
:102B0000631E0C16630C0D16130615003335A60054
:102B10002E959356F5013696B335D600AA95939621
:102B2000F50105828585D18E6346B000639D051A47
:102B3000638B061A0356C90215823305D600333655
:102B4000C500B2956348B000639105241306F00FE9
:102B5000637DA622894663F3561593078008F3B771
:102B6000078093F78708BED60100010037170040A1
:102B7000930770052300F704930780FA2300F704F6
:102B8000010001008356C70289678117D58FC207EC
:102B9000C1832316F70223000704B657F3A7078063
:102BA00001000100FA506A54DA544A59BA592A5AB3
:102BB0009A5A0A5BFA4B6A4CDA4C4A4DBA4D296173
:102BC00082801308F5FF3335A800FD152E951356A6
:102BD000F5013298B336C800AA9695B9F336048049
:102BE00093F68608B6CA0100010023809D00238069
:102BF000AD000100010083463905CD8EA309D9043B
:102C000023800D00D646F3A606800100010035B3EF
:102C1000F336048093F68608B6CE010001002380C7
:102C20009D002380CD00010001008346390593E615
:102C30000602A309D90423800D00F646F3A60680F8
:102C40000100010095B3F336048093F68608B6D2EE
:102C50000100010023809D002380CD0001000100C0
:102C60008346390593E60602A309D90423800D00A3
:102C70009656F3A606800100010045BB9306F5FFBA
:102C800033B5A600FD152E959355F501AE96B3B557
:102C9000B600AA951396F501858269B5F3360480CE
:102CA00093F68608B6D801000100930680FA2380C7
:102CB0009D002380DD00010001008356C9020566E6
:102CC000011693F6F60FD18EC206C1822316D902E1
:102CD00023800D00C656F3A6068001000100850A78
:102CE00093FAFA0F95B233E6B60045C20356C9020D
:102CF0003305D0403338A000B305B040B38505415B
:102D000015826345B000D1E16371A608894663F07E
:102D1000560593078008F3B7078093F78708BEDA54
:102D200001000100B7170040130770052380E70476
:102D3000130780FA2380E7040100010003D7C702CC
:102D40007D8B2396E70223800704D65781BDF33697
:102D5000048093F68608B6DC01000100930680FA31
:102D600023809D002380DD00010001008356C902FD
:102D70000566011693F6F60FD18EC206C1822316A0
:102D8000D90223800D00E656B9B793078008F3B740
:102D9000078093F78708BEDE010001003717004067
:102DA000930770052300F704930780FA2300F704C4
:102DB000010001000356C70293975600B297C2075D
:102DC000C1832316F70223000704F657C1BB9147BE
:102DD00063EEB70217D701001307076E8A05BA958D
:102DE0009C41BA978287B717004003A7470B13454A
:102DF000F5FF698F23AAE70A03A7070B698F23A8AA
:102E0000E70A03A7070A798D23A0A70A8280B717CC
:102E1000004083A6470B1347F5FFF98E23AAD70A74
:102E200083A6070B558D23A8A70A83A6070A758FCB
:102E300023A0E70A8280B717004003A7470B498FFA
:102E400023AAE70A03A7070B1345F5FF45BFB717EA
:102E5000004083A6470B1347F5FF758F23AAE70AA7
:102E600003A7070A598D4DB7B717004003A7470BB3
:102E7000498FEDB7914763EEB70217D701001307EB
:102E8000E7648A05BA959C41BA978287B7170040D4
:102E900003A7470D1345F5FF698F23AAE70C03A786
:102EA000070D698F23A8E70C03A7070C798D23A0D2
:102EB000A70C8280B717004083A6470D1347F5FF84
:102EC000F98E23AAD70C83A6070D558D23A8A70C2E
:102ED00083A6070C758F23A0E70C8280B7170040EC
:102EE00003A7470D498F23AAE70C03A7070D134536
:102EF000F5FF45BFB717004083A6470D1347F5FF01
:102F0000758F23AAE70C03A7070C598D4DB7B71788
:102F1000004003A7470D498FEDB7797122D43714CC
:102F2000004026D24AD0035924028354040206D614
:102F30004209C2044ECE52CC56CA13590901C1806F
:102F40002DE11379F9F793F4F49F4209C204135960
:102F50000901C18093078008F3B7078093F78708BA
:102F60003EC401000100930770052300F404930799
:102F700080FA2300F404010001002311240323102C
:102F8000940223000404A247F3A707800100010074
:102F9000B250225492540259F249624AD24A4561CF
:102FA0008280B7F5070081463000B10519459700CA
:102FB0000020E7806081A24713972701E34A07FCBE
:102FC0001369090893E4044093098008F3B7098062
:102FD00093F787083EC001000100930A70052300A3
:102FE0005405130A80FA230044050100010023114F
:102FF000240323109402230004048247F3A70780CC
:1030000001000100294597F0FF1FE780A032F3B9C6
:10301000098093F989084EC201000100230054057C
:1030200023004405010001008357040293E70720B1
:103030002310F402230004049247B9B7B7170040E5
:103040008847420541819377050491EB9377F50119
:103050003755E801130505803345F50282809377E3
:10306000050C130700046397E7009377F5013745D4
:103070009C1CCDB72165130505D0828037E700E0A1
:103080001C435443A183E206D58F1CC1FD57232066
:10309000F7182322F718828013178500B7E700E09E
:1030A00023A0E710618123A2A7108280B7F700E078
:1030B0008847CC478280814737370040A14663C4A8
:1030C000C700328582800345B740E38EA6FE338574
:1030D000F5000345050085072304A740CDB79707F2
:1030E0000020938727EF9C43173700201307871989
:1030F0003E95636EE500173700201307A7506368FD
:10310000A700170700202327A7EC3E858280FD57E4
:10311000EDBF8280411122C406C62A8497000000B8
:10312000E78000F22947B307E502B2408D83B3D7A9
:10313000870222449507B3D7E70237370040C2071A
:10314000C1832316F70041018280411137150E001B
:1031500006C697000000E78020FCB7370040130741
:1031600070F82381E7000D47A381E70013070004EF
:10317000A380E70005472387E700B2404101828032
:1031800037370040834727001A0593F7F703C98FA5
:1031900093F7F70F2301F7008280B737004003C78A
:1031A000170019C9D98DA380B70003C7070013679B
:1031B00087002380E700828093C5F5FFF98DA38007
:1031C000B7008280AE872A87B7360040214637385D
:1031D000004089E7170300006700E3F383C8B600E7
:1031E000E30916FF05078348F7FFFD17C20723040D
:1031F0001801C183F9BF411122C406C62A84970071
:103200000000E780E0E32947B307E502B2408D8381
:10321000B3D7870222449507B3D7E7023737004078
:10322000C207C1832316F7404101828071654111B5
:103230001305052006C697000000E78000FCB7379D
:103240000040130770F82381E7400D47A381E74052
:1032500013070004A380E74005472387E740B240F7
:1032600041018280CC41411106C6328503C615005A
:1032700083C5050022064D8E42068D654186138862
:1032800075A2630C0611634BC804138845A2630042
:10329000060D634AC800938535A26301B6082390E2
:1032A000060029464DA0138855A26305060D938597
:1032B00065A2E316B6FE8D451D4663E6E508114698
:1032C000198E63F3C7003E86B7E704002390C6005B
:1032D000FC4797D501009385A5219DA0138895A251
:1032E00063030611634E060D1388A5A2630006133F
:1032F000938505A5E315B6FA99451D4663E5E504F2
:10330000198E63F3C7003E86B7E704002390C6001A
:10331000FC4797050020938525D61DA09D451D4699
:1033200063E3E5022146198E63F3C7003E86B7E7E3
:103330000400FC472390C6009705002093850534C0
:10334000BA9582970146B240328541018280AD45EF
:103350001D46E3EAE5FE3146198E63F3C7003E865B
:10336000B7E704002390C600FC4797D5010093857A
:10337000A51AF9B7B1451D46E3E7E5FC3546198EB8
:1033800063F3C7003E86B7E704002390C600FC47FE
:1033900097D501009385451965B78D451D46E3E432
:1033A000E5FA1146198E63F3C7003E86B7E70400BD
:1033B0002390C600FC4797D501009385251449B793
:1033C0008D451D46E3E1E5F81146198E63F3C7000C
:1033D0003E86B7E704002390C600FC4797D501005E
:1033E00093854516B1BFA5451D46E3EEE5F4294694
:1033F000198E63F3C7003E86B7E704002390C6002A
:10340000FC4797D50100938525101DBFB5451D4686
:10341000E3EBE5F23946198E63F3C7003E86B7E762
:1034200004002390C600FC4797D501009385450B07
:1034300001BFB7E7040003A3071397060020938694
:10344000A6C24146A545170500201305E5B802832D
:103450002D455DE703C505000947631FE50803A87F
:103460004500411106C6034718003285034608008F
:1034700022074168518F930828FE6307170563E907
:10348000E80005186303070323900600294591A867
:10349000130648FE630AC7041518E31707FF15460D
:1034A0003E87637BF600154701A8130600023E879E
:1034B0006374F60013070002B7E704002390E600E8
:1034C000FC471316070111A83E8691C30546B7E7CE
:1034D0000400FC472390C6004206CC4541828297F7
:1034E0000145B24041018280130600083E87E37522
:1034F000F6FC13070008C9B7239006000545828033
:103500008280416779176304E504411122C406C62D
:1035100085472A84639FF500B7E70400228522448B
:10352000B24003A38713970500209385652F4101BF
:10353000028389476399F500B7E7040083A7070B67
:103540008545829771D9B2402244410182808280B0
:10355000797122D452CC2E842A8A97D50100938582
:10356000650017D501001305650206D63AC626D2B6
:103570004AD0B68432894ECE97B00100E78080539E
:10358000A68517D501001305650197B00100E780F6
:103590006052294597B00100E780A0568347840018
:1035A00093F70702E1E7834904008947054532475D
:1035B0006396F908544083C7160083C60600A20725
:1035C000D58FC166138616FE638CC7028D16638F76
:1035D000D7068D669386269029456391D706B7E76F
:1035E0000400A285225403A34714B250F249A686D0
:1035F0004A86925402595285624A85474561028340
:103600002D450DEF93070002354563E99702B7E7B3
:103610000400FC47484413060002CA85829781498A
:1036200097070020938787209C43014581CB9C43CB
:1036300091C74E852686CA8582970145B25022548D
:1036400092540259F249624A456182802D457DF7C4
:103650009307700F3545E3E397FEB7E70400FC4797
:1036600048441306700FCA8582975DBF2145F9B79C
:10367000411122C437E404008327841326C2AA849C
:10368000416506C697050020938585197D158297AB
:103690008327C40A170500001305E5E6858882978D
:1036A00095C0032304132244B2409244970600209D
:1036B000938606AE4146C545170500201305459C77
:1036C00041010283B240224492440145410182807B
:1036D00019C59707002023ABA714014582804545F3
:1036E00082801147636AA70A97D60100938646E64F
:1036F0000A0536951841411106C63697AE87B28540
:103700000287130700026145639DE700B7E70400E5
:10371000FC4713060002170500201305A5F6829743
:103720000145B2404101828005476145E39BE7FEC8
:10373000B7E70400FC47054617050020130585F68A
:10374000F9BF1307700F6145E39DE7FCB7E704007D
:10375000FC471306700F170500201305E5F4C1B7E9
:10376000130700086145E39EE7FAB7E70400FC474A
:103770001306000817050020130585024DB71547ED
:103780006145E390E7FAB7E70400FC4715461705E3
:1037900000201305250961B709458280411126C221
:1037A000B7E4040083A7C41322C44AC006C62E840B
:1037B000970500209385C5062A898297058905C546
:1037C000970700209387C78B83D7A70BA28503A3F6
:1037D000440D2310F4002244B24092444A85024929
:1037E000014641010283B2402244924402494945C4
:1037F0004101828097070020238C07029707002051
:1038000023AA0702B717004003A7070CB706C0FF9B
:10381000FD16758F23A0E70C03A7070DB706400020
:10382000558F23A8E70C03A7070C3D9B23A0E70CAB
:1038300003A7070D1367070123A8E70C8280B717BA
:10384000004003A5470C83A7470C59811345150079
:10385000C18B058999E3136525009707002083C76D
:1038600027FD6380A702970700202383A7FC11C9C7
:1038700097070020938707FC03A307006303030057
:1038800002838280114517F3FFFF670043C841118F
:1038900093962500AA852D4506C697F0FF1FE78061
:1038A000A0F2B240014541018280011122CC06CE36
:1038B0003714004026CA4AC84EC652C48344740511
:1038C000034AB405834984050349940597F0FFFF33
:1038D000E780C09E8347A40593F4F40F137AFA0F90
:1038E00093E71700230DF40493F9F90F1379F90FF7
:1038F000B717004003C7A705058B6DFF03D5C705A4
:10390000A38D4705238C3705A38C2705A38B97042C
:10391000F2406244D2444249B249224A056182805F
:1039200041119397050122C406C626C2C1872E8481
:1039300063DC0700B7E40400FC54829719C1BC544F
:1039400082972165218D15A893F7150013C51500E1
:103950008DE793F725009DC797000000E78060EE94
:10396000B7E70400BC4F1306000A8945170500207D
:103970000345C5EC829713452400B240224492448B
:10398000410182809397250163D80702B7E40400C0
:1039900083A7C41E829797000000E780E0EEBC4C2E
:1039A00037560700130606308965170500200345C2
:1039B000E5E88297096579B7939715010145E3DE3C
:1039C00007FA17D50100130565C597B00100E78018
:1039D0004026B7E70400BC4F130600649165170545
:1039E00000200345A5E582971165A9BF2D71232A03
:1039F0009110FD74E98C232C81102328211123269A
:103A000031112A84AE893289930600100A86A68570
:103A10002D45232E111097F0FF1FE780E0DA1315D4
:103A20004401B7E70400FC4751810A0513962900B9
:103A3000CA850A958297A68585660146254597F031
:103A4000FF1FE78060D80A86A685930600102945E7
:103A500097F0FF1FE78040D78320C1110324811115
:103A600083244111032901118329C110156182802A
:103A7000B7F7070003C70701411106C622C426C2D3
:103A80004AC0A547631DF70097000000E78040F695
:103A9000B24022449244024901454101828013947C
:103AA0002500AA843289A286AA850146254597F079
:103AB000FF1FE78060D1A2864A86A685294597F038
:103AC000FF1FE78060D0E9B71D71A2CC37E4040086
:103AD0005C5C485886CE494697D50100938585AFF2
:103AE000829711E917D50100130505B097B00100C1
:103AF000E780201401A0B7F600E0795798CAFD5777
:103B0000DCCA0567B7E700E023A0E7101306F00260
:103B100090C223A0E71801000100370700201847D2
:103B20001306000481459706002023A7E6D04157DD
:103B3000A38AE7403C4408088297970700209387B0
:103B4000E76C3EC8856713870740231AE1001D67AD
:103B50003ACC37070105130707103ACE938757D1A0
:103B60001307B00F2310E1022312F102054797F764
:103B7000FFFF9387E7532301E1023ED817070000B8
:103B8000130727D197070000938767D2B7F507007F
:103B9000BAC23EDC170700001307C7ED9707000005
:103BA000938787CE81463000E1051945BAC43EDED1
:103BB00097F0FF1FE78040C1180881479946300001
:103BC0003E960346060085070507A30BC700E3984A
:103BD000D7FEC24791C70357410185676373F7005A
:103BE00001A0B7E7040083A7470A08088297AA85BF
:103BF00011C917D50100130565A097B00100E78032
:103C000060EB01A0F640664425618280411126C226
:103C1000B7E4040083A7040806C622C41705000001
:103C2000130545D0829717040020130424C12300F4
:103C3000A40097000000E780800297000000E78062
:103C4000A0BB03450400224403A38405B240924470
:103C500013060032896541010283797106D622D4A8
:103C600013078008F337078093F787083EC20100E7
:103C70000100B7170040930570052380B7041306B1
:103C800080FA2380C7040100010083C6F70293F67F
:103C9000A60FA387D702238007049246F3A60680C7
:103CA0000100010073370780137787083AC40100C9
:103CB00001002380B7042380C7040100010003C76B
:103CC000F70213672700A387E70223800704A247B0
:103CD000F3A7078001000100054597E0FFFFE7809B
:103CE000206197000000E78020BA014781468147A4
:103CF000054685451305407E97E0FFFFE780206479
:103D000037E404003C446800514681458297B70778
:103D1000C0A83EC8B787E803938707D03ECA97E795
:103D2000FF1F9387C7693EC67C5868008297B250D0
:103D3000225445618280411197D50100938545F455
:103D400017D501001305858406C697B00100E780EA
:103D500060D617D501001305650B97B00100E78009
:103D600060D5B2402945410117B30100670063D90E
:103D7000411197D501009385E5F117D50100130591
:103D8000E58006C697B00100E780C0D217D50100D4
:103D90001305850697B00100E780C0D1B2402945E0
:103DA000410117B301006700C3D5411122C406C603
:103DB000834705002A849DC797D50100938545F365
:103DC00017C501001305857C97B00100E78080CE00
:103DD0004C4017D501001305A51197B00100E780ED
:103DE00060CD3DA058410DEF97D50100938545F07A
:103DF00017C501001305857997B00100E78080CBD6
:103E000017D501001305451097B00100E78080CA5F
:103E10002244B2402945410117B30100670063CE37
:103E2000A1679386D7036313D70297D501009385C3
:103E300025EC17C501001305657597B00100E780F3
:103E400060C717D501001305250D7DBFED0797D578
:103E500001009385E5E917C5010013052573631B70
:103E6000F70097B00100E780E0C417D50100130503
:103E7000E50B59BF97B00100E780C0C34C4017D590
:103E800001001305A50C91BF411197D50100938541
:103E9000A5E117C501001305656F06C697B00100BF
:103EA000E78040C1B2402945410117B301006700D6
:103EB00043C5797122D426D24AD02E842A898145DD
:103EC000B2844800714606D697E0FFFFE780A02243
:103ED00097F7FF1F9387874CDC4783D7070023148E
:103EE00021012313F10097500000E780A0E59547DA
:103EF000A305F1009307401F3EC6FD572305A1000F
:103F0000230AF10097500000E78000F82686A2857A
:103F1000480097500000E780C0E5B2502254925408
:103F2000025945618280971700202394077E9717D6
:103F30000020238D076CB7E70400BC47411106C67B
:103F400041468145170500201305851A8297972061
:103F50000000E780606097200000E7806041014535
:103F600097600000E780A08A170700200347471AE0
:103F70009307F00A6315F7029307F0F889451705D0
:103F800000201305E518170700202303F7189707EB
:103F90000020A38F071697600000E780E0B19760CC
:103FA0000000E780A0BE8145370504009707002088
:103FB00023AE0712970700202398071297070020C7
:103FC00023850712970700202396070A97070020EA
:103FD00023940708970700202397071097070020CE
:103FE0002390071297300000E780A00D01459760ED
:103FF0000000E78060B597D50100938565CD17C5B2
:1040000001001305A55897B00100E780A0AA17D5B5
:1040100001001305E5F997B00100E780A0A9B240BF
:104020002945410117B301006700A3AD411122C426
:1040300006C626C293F715002E84638F07108146AB
:1040400017F6FF1F1306C6328545170500200355D6
:10405000650097C00000E780A01715C997D501003B
:104060009385C5C717C501001305455297B00100D8
:10407000E78040A417C501001305056997B001004A
:10408000E78040A3294597B00100E78080A797D536
:1040900001009385A5C417C501001305254F97B0EE
:1040A0000100E78020A117C501001305256797B01F
:1040B0000100E78020A0294597B00100E78060A4B7
:1040C00017F5FF1F1305852D5C4505472390E70075
:1040D00097400100E78020C897D50100938505C06F
:1040E00017C501001305854A97B00100E780809C41
:1040F00017C501001305C56397B00100E780809BD9
:10410000294597B00100E780C09F930710F8170773
:104110000020230FF7FE9707002083D767F31707C8
:104120000020A307F7FE17050020130565FEA183F5
:10413000914517070020230EF7FC97070020A38A5C
:1041400007FC97600000E780209713451400B240F9
:10415000224492444101828093F72500E1C317076E
:104160000020035767F845CB97060020938606F892
:10417000944297D701009387A7E5170600200346CE
:10418000C6F6814517050020130585F697700000D7
:10419000E7802024AA8441C197D501009385C5BA40
:1041A00017C501001305853E97B00100E780809098
:1041B000A68517C501001305255997B00100E780B2
:1041C000608F294597B00100E780A09397070020F2
:1041D000239C07F0930710F817070020230AF7F233
:1041E0009707002083D7C7E617070020A302F7F23E
:1041F000A18317070020230EF7F091458D4717057F
:1042000000201305E5F017070020A304F7F09760DE
:104210000000E780608A1345240015BF93F745002E
:10422000D1C397D50100938525B217C501001305A9
:10423000E53597B00100E780E08717C50100130559
:10424000655297B00100E780E086294597B00100EC
:10425000E780208B930720F817070020230AF7EA4E
:104260009707002083D707E117070020A302F7EA8A
:10427000A18317070020230EF7E8854717070020C2
:10428000A309F7E897500000E78000C01705002059
:10429000130505E8914597600000E780E08113452C
:1042A000440075B593F78500A9C797D5010093859C
:1042B000A5A917C501001305652D97A00100E7808A
:1042C000607F17C501001305254B97A00100E7800B
:1042D000607E294597B00100E780A0829707002003
:1042E000239407E097700000E780801E1345840048
:1042F000B9BD93F70501D1C38545170500200355C6
:1043000065D797600100E780E0CF97D501009385DE
:10431000A5A317C501001305652797A00100E78035
:10432000607917C501001305654697A00100E78075
:104330006078294597A00100E780A07C930730F8BA
:10434000170700202306F7DC9707002083D787D2C2
:1043500017070020A30EF7DA17050020130545DB29
:10436000A1838D45170700202305F7DA9750000039
:10437000E780807413450401D9BB93F70502D1C7C8
:1043800097D501009385459C17C5010013050520AD
:1043900097A00100E780007217C501001305454191
:1043A00097A00100E7800071294597A00100E780F0
:1043B0004075930740F817070020230BF7D49707A1
:1043C000002083D767C917070020A303F7D4A18370
:1043D00017070020230FF7D2854717070020A30AED
:1043E000F7D297070020239907C697500000E7806F
:1043F000A0A9170500201305A5D1914597500000ED
:10440000E780806B1345040299B393F70504FDC35D
:1044100097D501009385459317C50100130505172E
:1044200097A00100E780006917C501001305C53991
:1044300097A00100E7800068294597A00100E78068
:10444000406C9707002083C7A7CC1307700A6386C8
:10445000E7061307800A638CE7081307600A639373
:10446000E704930760F8170700202303F7CA9707AC
:10447000002083D747C717070020A30BF7C8A183E5
:10448000170700202307F7C8854717070020A30652
:10449000F7C8B14517050020130585C797500000E0
:1044A000E780806197500000E780009E1345040478
:1044B00097070020239907C259B9930770F8170787
:1044C00000202307F7C49707002083D7C7C1170729
:1044D0000020A30FF7C2A18317070020230BF7C208
:1044E000854717070020A307F7C2994565B79307CB
:1044F00080F8F1B793F705080145E38A07C497D51B
:1045000001009385658417C501001305250897A050
:104510000100E780205A17C501001305652C97A0FC
:104520000100E7802059294597A00100E780605DE0
:104530009307A0F817070020230CF7BC970700206B
:1045400083D707BC17070020A304F7BCA183170774
:1045500000202300F7BC854717070020A30BF7BAFC
:1045600097070020239E07B897500000E780C0916E
:10457000170500201305C5B9914597500000E78045
:10458000A05313450408E1B6411122C497C50100A8
:10459000938545772A8417C50100130525FF06C6B4
:1045A00097A00100E78000514C4017D5010013058A
:1045B000A59197A00100E780E04F294597A0010051
:1045C000E7802054034704009307F00F631FF702AE
:1045D00097C501009385057317C50100130505FBF9
:1045E00097A00100E780004D4C4017D5010013054E
:1045F000A58E97A00100E780E04B2244B2402945F8
:10460000410117A301006700C34FB240224441019A
:104610008280B1C1411122C417C50100130505F7FD
:104620002E8497C501009385E56806C697A0010012
:10463000E7804048A28517D501001305259597A06E
:104640000100E78020472244B2402945410117A3D9
:1046500001006700034B8280411122C426C22E84D0
:10466000AA8497C501009385A56517C501001305A8
:10467000E5F106C697A00100E780C04317D5010009
:104680001305859197A00100E780C042294597A0B6
:104690000100E780004797C5010093856562970791
:1046A00000202399979A17C50100130525EE85442C
:1046B00097070020239E879897070020239B9798B1
:1046C000971700202397870497A00100E780803E7A
:1046D0009715002083D5E50317D501001305458CF8
:1046E00097A00100E780003D294597A00100E780E1
:1046F000404197170020238B97F097200000E78018
:1047000020C7228597500000E7806010054597502C
:104710000000E780604397F7FF1F938727C8DC47B7
:1047200003D70700C167FD176312F7022244B7E7FA
:104730000400B240924403A3870517F5FF1F034509
:1047400065101306000A854541010283B2402244E8
:10475000924441018280011122CC37E404005C5C68
:1047600006CE354697C501009385856B17D50100A8
:1047700013058531829711E917C501001305C5E6B8
:1047800097A00100E780E04A01A097F7FF1F9387F9
:10479000270C3EC4B7F507008567938707808146DD
:1047A00017F6FF1F1306460AE10519453EC697E0B6
:1047B000FF1FE78060017C44194697F5FF1F938532
:1047C000A508170500201305258B8297340017F6DE
:1047D000FF1F1306660797D501009385A5B517D56A
:1047E00001001305A5B697700000E78080932A8426
:1047F0001DCD97C501009385255417C501001305EC
:10480000E5D897A00100E780E02AA28517C501003E
:104810001305056297A00100E780C029294597A0EC
:104820000100E780002EF24062440561828097E03B
:104830000000E78020F517C5010013056556976055
:104840000000E780C08797600100E78060AE17F541
:10485000FF1F130525B197600100E780009717C57A
:1048600001001305E55497600100E780E0AE2A845B
:1048700097600000E78080EE97100100E780408697
:1048800097800100E780601F97700000E780C046B6
:1048900097600000E780806497300100E780A047C0
:1048A00097C501009385454917C50100130505CE3D
:1048B00019C897A00100E780E01FA28517C5010075
:1048C0001305455981BF97A00100E780A01E17C5B9
:1048D00001001305655A97A00100E780A01D294536
:1048E00097A00100E780E02197300100E780802356
:1048F000A94717F7FF1F231BF79417F7FF1F23087C
:10490000F79497F00000E780204155C985453705A9
:10491000040097200000E780C07A97C501009385C6
:10492000A54117C50100130565C697A00100E780E2
:10493000601817C501001305A55597A00100E78071
:104940006017294597A00100E780A01B97F7FF1F7C
:104950009387879483D7070017170020231BF7DA64
:104960008547171700202303F7CA97200000E78028
:1049700020B997200000E780A09F1715002003555D
:1049800045D997500000E78080E805459750000022
:10499000E780801B97C501009385053A17C5010084
:1049A0001305C5BE97A00100E780C01017C5010020
:1049B0001305455097A00100E780C00F85B597C546
:1049C00001009385653717C50100130525BC97A025
:1049D0000100E780200E17C501001305655D97A053
:1049E0000100E780200D294597A00100E7806011B4
:1049F000014569BF411122C437E404008327041A2A
:104A000006C6829797500000E78020E483270408B9
:104A100017F5FFFF1305C561829797F7FF1F2383E3
:104A2000A7E217F5FF1F1305659797400000E78081
:104A300040782244B2404101170300006700E3D1EF
:104A4000B7E70400FC471171A2DDCAD986DFA6DBF7
:104A5000CED72E8432892E86AA8517F5FF1F13051F
:104A6000256B829717F7FF1F1307876A8347070095
:104A7000930680029387E70793F7F70FE3ECF610AE
:104A8000BA898A0717C70100130787B9BA979C43E9
:104A9000BA9782878D4797C501009385252C17C546
:104AA00001001305A5AE630FF40097A00100E78095
:104AB000600017C50100130525E997A00100E780F4
:104AC00060FFBDA497A00100E780C0FE17C50100EC
:104AD000130505E997A00100E780C0FD294597A0CF
:104AE0000100E7800002930720F8114697F5FF1FA9
:104AF000938505624A8517F7FF1F230BF76097F729
:104B0000FF1FA388076097F0FFFFE780C03A2A8461
:104B10001DC997C501009385652417C501001305BC
:104B2000E5A697A00100E780E0F8A28517C501007F
:104B30001305C5E697A00100E780C0F7294597A0B7
:104B40000100E78000FC97C501009385252117C56A
:104B500001001305A5A397A00100E780A0F517C5E4
:104B600001001305E5E497A00100E780A0F42945C2
:104B700097A00100E780E0F84165930730FA054609
:104B800097F5FF1F9385C5587D1517F7FF1F230164
:104B9000F75897F0FFFFE78000322A841DC997C5B8
:104BA00001009385A51B17C501001305259E97A03D
:104BB0000100E78020F0A28517C50100130505DE7E
:104BC00097A00100E78000EF294597A00100E7804A
:104BD00040F3B7E70400BC4F0566130606C8A145BD
:104BE00017F5FF1F034505C68297FE506E54DE542D
:104BF0004E59BE591161828091476303F40297C5F3
:104C000001009385A51517C501001305259897A0E8
:104C10000100E78020EA17C501001305A5DC71BD7E
:104C2000B7E70400FC4F914517F5FF1F034585C109
:104C3000829797C501009385651217C5010013057A
:104C4000E59497A00100E780E0E617C50100130591
:104C500025DB97A00100E780E0E5294597A001004A
:104C6000E78020EA97400000E7800022914535A4C4
:104C700085476303F40297C501009385250E17C588
:104C800001001305A59097A00100E780A0E217C5D9
:104C90000100130565D815B597F7FF1F239C273D25
:104CA000B7E704000566BC4F130606C8C1450DBF33
:104CB0008D476303F40297C501009385250A17C544
:104CC00001001305A58C97A00100E780A0DE17C5A1
:104CD0000100130525D6D5B3930740F8114697F583
:104CE000FF1F9385E5424A8517F7FF1F2302F7420E
:104CF00097F7FF1FA38F074097F0FFFFE780A01BE8
:104D00002A84E30405EE97C501009385250517C5A0
:104D100001001305A58797A00100E780A0D9A2850F
:104D200017C50100130585C797A00100E78080D84B
:104D3000294597A00100E780C0DC45BD9147E31CF1
:104D4000F4F6B7E70400FC4F9305000217F5FF1FC8
:104D5000034545AF829797C501009385250017C588
:104D600001001305A58297A00100E780A0D417C514
:104D700001001305A5CDF1BD894763E3870297C5FF
:104D800001009385A5FD17C501001305258097A097
:104D90000100E78020D217C50100130565CC31BBA7
:104DA00097F4FF1F83C4E43697F7FF1F83C7573676
:104DB00097C50100938585FAA20417B50100130574
:104DC000E57CDD8C97A00100E780C0CEA28517C5E9
:104DD0000100130525CA97A00100E780A0CDC204F9
:104DE000294597A00100E780C0D1C1849305D4FF75
:104DF00093960401C1824A8693F5F50F17F5FF1FBC
:104E00001305353197200000E780602FE35F90DCC9
:104E1000930750F817F7FF1F230CF72E83C73900AD
:104E2000228697F5FF1F9385A52E85074A8517F7DC
:104E3000FF1FA300F72E97F0FFFFE780C0072A842B
:104E4000E30505DA97C50100938545F117B5010023
:104E50001305C57397A00100E780C0C5A28517C5DB
:104E600001001305A511C9B5894763E3870297C5FA
:104E700001009385A5EE17B501001305257197A0D4
:104E80000100E78020C317C50100130565C035B1D7
:104E900097400000E78040FFA28517F5FF1F13052C
:104EA000252797500000E78020C181B38D47630319
:104EB000F40297C50100938565EA17B50100130553
:104EC000E56C97A00100E780E0BE17C5010013055F
:104ED000E5BDE5B6B76602000146B77502000545B7
:104EE00097E0FF1FE780408E930760F817F7FF1FDA
:104EF0002300F72297F7FF1FA38D072093070006D3
:104F000017F7FF1F2308F720894717F7FF1FA30391
:104F1000F72097F7FF1F2380072097F7FF1FA38C29
:104F2000071EC14717F7FF1F2308F71E930720F935
:104F300017F7FF1FA302F71E314697F7FF1FA38E37
:104F4000A71C97F5FF1F9385A51C4A8597F7FF1FA0
:104F50002385071C97F0FFFFE780E0F52A84E3062E
:104F600005C897C50100938565DF17B501001305D6
:104F7000E56197A00100E780E0B3A28517C50100B5
:104F8000130545B455B3B1476303F40297C5010057
:104F90009385C5DC17B501001305455F97A0010097
:104FA000E78040B117C50100130585B339B6B7E7EF
:104FB0000400FC4F9305000417F5FF1F0345858887
:104FC000829797400000E78020ECB145F9B5914702
:104FD00063E3870297C50100938545D817B50100A3
:104FE0001305C55A97A00100E780C0AC17C50100A2
:104FF0001305C5B0D9B497F4FF1F83C4A41197F764
:10500000FF1F83C71711A204DD8C8E04B77702003F
:105010006D14BE942286A68517C50100130545AF01
:1050200097A00100E78000A9B7E70400FC472286AB
:1050300097F5FF1F9385150E28008297931604019C
:10504000C1823000A685094597D0FF1FE780C07751
:105050002A8409C917C50100130545AD97A00100B1
:10506000E78020BD930770F8194697F5FF1F9385D9
:10507000250A4A8517F7FF1F230CF70897F7FF1F2C
:10508000A38A870897F0FFFFE780E0E22A84E30E17
:1050900005B497C50100938565CC17B501001305CC
:1050A000E54E97A00100E780E0A0A28517C50100AA
:1050B0001305C5A895B99947630BF41297C501006C
:1050C0009385C5C917B501001305454C97A001008C
:1050D000E780409E17C501001305C5A7F9BA91479F
:1050E00063E3870297C50100938545C717B50100A3
:1050F0001305C54997A00100E780C09B17C50100B3
:105100001305C5A65DBA97F4FF1F83C4A40097F7E3
:10511000FF1F83C71700A204DD8C8E04B77702003F
:105120006D14BE942286A68517C50100130545A5FA
:1051300097A00100E7800098B7E70400FC472286AB
:1051400097F5FF1F938515FD28008297931604019C
:10515000C1823000A6850D4597D0FF1FE780C0664D
:105160002A8409C917C50100130545A397A00100AA
:10517000E78020AC930780F8194697F5FF1F9385C9
:1051800025F94A8517F7FF1F2304F7F897F7FF1F44
:10519000A38287F897F0FFFFE780E0D12A84E30637
:1051A00005A497C50100938565BB17B501001305DC
:1051B000E53D97A00100E780E08FA28517C50100BB
:1051C0001305059F95B699476303F40297C501003F
:1051D0009385C5B817B501001305453B97A001009D
:1051E000E780408D17C501001305059EF9B0B7E7AC
:1051F0000400FC4F9305000417E5FF1F0345856479
:10520000829797400000E78020C8994579B18D4783
:105210006303F40297C50100938545B417B50100F7
:105220001305C53697A00100E780C08817C50100A7
:105230001305059B59B017C501001305659B97A081
:105240000100E780009F1305C01297D0FF1FE78081
:10525000400F014597E0FFFFE78080E20D45971082
:105260000000E780009F294597D0FF1FE780600D71
:1052700097D0FF1FE780C0FD8DBA99476303F40202
:1052800097C50100938585AD17B50100130505305D
:1052900097A00100E780008217C50100130505965D
:1052A00029B817F7FF1F0347F7E697F7FF1F83C7D4
:1052B00067E622075D8F9166BA96C2061166C182C3
:1052C0001306F6EF8D476365D60297E7FF1F9387B6
:1052D000E70C9C4B17F6FF1F0346B6E39386C70007
:1052E0002DC203D6070069CA8907E39CD7FE894708
:1052F0001307A0F8114697F5FF1F938565E14A85CE
:1053000097F6FF1F2386E6E017F7FF1FA303F7E0DA
:1053100097F0FFFFE78020BA2A84E308058C97C541
:1053200001009385A5A317B50100130525269790C5
:105330000100E7802078A28517C501001305458D7F
:10534000E5B203D60700630EE60A8907E39BF6FE83
:105350008D4779BF91476304F40297C50100938597
:10536000E59F17B501001305652297900100E780BE
:10537000607417C501001305258B6FF00FF4B7E7B4
:105380000400FC4F9305000817E5FF1F0345854BFC
:105390008297C9B897C501009385459C17B5010050
:1053A0001305C51E97900100E780C07017C5010066
:1053B000130505896FF06FF02390E70017E5FF1FD5
:1053C0001305C5FD97300100E780409B97C501009C
:1053D0009385C59817B501001305451B97900100EB
:1053E000E780406D17C50100130585869790010081
:1053F000E780406C294597900100E78080708147E5
:10540000C5BD2390070017E5FF1F130525F9973049
:105410000100E780A09697C501009385259417B5F4
:1054200001001305A51697900100E780A06817C535
:105430000100130565835DBF411122C406C6834781
:1054400005002A849DC797C501009385E58C17B593
:1054500001001305A51397900100E780A0654C405B
:1054600017C501001305C5B797900100E780806458
:10547000E1A05841B707CF009387777D631DF706FA
:1054800097C501009385458917B5010013050510DF
:1054900097900100E78000621C448356E400835526
:1054A000C40003C6070017C501001305E5B49790B3
:1054B0000100E7802060294597900100E780606443
:1054C0000357E4009707002083D7A7246309F70058
:1054D0008355C400084497E0FFFFE780E0CE035601
:1054E000E4008355C40008442244B240410117F34C
:1054F000FFFF67002355B707CC009387777D6315BF
:10550000F70497C501009385258117B501001305A0
:10551000E50797900100E780E0591C448356E400BA
:105520008355C40003C6070017C501001305C5ACA9
:1055300097900100E78000582244B240294541017C
:10554000179301006700E35BB707CE009387777D71
:105550006304F70297B501009385057C17B5010038
:105560001305C50297900100E780C0544C4017C551
:1055700001001305A59DCDBDB240224441018280AA
:10558000B7E70400FC4741112E8606C622C426C296
:105590004AC02E842A89AA8517F5FF1F130545B72F
:1055A000829797B501009385257D17B501001305F6
:1055B000E5FD97900100E780E04F97F5FF1F83C559
:1055C00025B517B501001305252397900100E78045
:1055D000604E294597900100E780A05297F4FF1F85
:1055E000938404B383C7040041479387070693F766
:1055F000F70F636AF75C17B701001307A70C8A0758
:10560000BA979C43BA9782879D476307F40297B580
:1056100001009385657617B50100130525F797906E
:105620000100E780204917B501001305651D97901B
:105630000100E7802048ADAC97F7FF1F83C757AD47
:10564000DDCB17F7FF1F0347D7AC97F7FF1F83C7C3
:1056500047AC22075D8F97F7FF1F83C7A7ABC20731
:105660005D8F97F7FF1F83C7F7AAE207D98F17F758
:10567000FF1F232DF7A683C7640097B5010093850C
:10568000A56F17B50100130565F017F7FF1F230E6F
:10569000F7A497900100E780E04197F7FF1F9387F9
:1056A000E7A48C4317F6FF1F034626A417B5010095
:1056B0001305C51697900100E780C03F29459790D4
:1056C0000100E780004497F7FF1FA38307A422444B
:1056D000B24092440249930700F817F7FF1F2309CD
:1056E000F7A29D4517F5FF1F130585A2410117433A
:1056F00000006700633C97600000E780E0EC97F7EC
:10570000FF1F2388A7A09357850017F7FF1FA30249
:10571000F7A0935705012A8417F7FF1F230CF79E64
:1057200093578501014517F7FF1FA305F79E976063
:105730000000E78020EA97F7FF1F238EA79C97B50C
:1057400001009385656317B50100130525E4979063
:105750000100E780203617F6FF1F0346C69BA2858F
:1057600017B501001305050DB1B7CD476303F4026A
:1057700097B501009385456017B50100130505E154
:1057800097900100E780003317B501001305050C61
:1057900079BD37E404007C44414697F5FF1F9385AB
:1057A000359717F5FF1F1305A594829717F5FF1F6F
:1057B0001305059497100000E780A0CD9710000016
:1057C000E78000BB97F7FF1F83C7A79517F7FF1F59
:1057D00003471795A20703238405D98F17F7FF1FE7
:1057E0002314F7901306000A89452244B2409244DC
:1057F000024917E5FF1F0345E504410102838D4778
:105800006303F40297B501009385055717B50100AE
:105810001305C5D797900100E780C02917B501008F
:105820001305851229B517F4FF1F0344848E97F7DB
:10583000FF1F83C7F78D97B501009385E5532204B9
:1058400017B50100130585D45D8C97900100E780A2
:105850006026A28517B501001305C50097900100C9
:10586000E7804025294597900100E78080290D4673
:1058700097F5FF1F9385C589228597E0FFFFE78095
:105880008063AA8421C197B501009385E54E17B5C1
:1058900001001305A5CF97900100E780A021A68500
:1058A00017B50100130545FD97900100E7808020A2
:1058B0002244B24092440249294541011793010014
:1058C0006700232497E7FF1F2396877AB7E7040032
:1058D000116603A38705130606E8914539B78D477E
:1058E0006303F40297B501009385054917B50100DC
:1058F0001305C5C997900100E780C01B17B50100CB
:10590000130545132DB317F4FF1F0344848097E755
:10591000FF1F83C7F77F97B501009385E5452204F4
:1059200017B50100130585C65D8C97900100E780CF
:105930006018A28517B50100130545F59790010081
:10594000E7804017294597900100E780801B0D46AE
:1059500097E5FF1F9385C57B228597E0FFFFE780D2
:105960008055AA841DC197B501009385E54017B500
:1059700001001305A5C197900100E780A013A6853B
:1059800017B501001305C5F105B797E7FF1F23956C
:10599000876CB7E70400116603A38705130606E8C2
:1059A0009305000299B5894763E3870297B5010023
:1059B0009385853C17B50100130545BD97900100FF
:1059C000E780400F17B50100130585098DB197E4F5
:1059D000FF1F83C4047497E7FF1F83C7777397B5CE
:1059E000010093856539A20417B50100130505BAB6
:1059F000DD8C97900100E780E00BA68517B50100CC
:105A0000130585EB97900100E780C00A2945979020
:105A10000100E780000F228697E5FF1F9385456F01
:105A2000268597E0FFFFE78000492A84630E051A68
:105A300097B501009385453417B50100130505B5E9
:105A400097900100E7800007A28517B501001305B4
:105A5000E5E799BD854763F9871883451900224416
:105A6000B24092440249B335B00097E7FF1F238D3F
:105A7000B76017B501001305A5E6410117930100B2
:105A800067004303A2852244B24092444A850249FA
:105A90004101170300006700032299476303F402E2
:105AA00097B501009385452D17B50100130505AE87
:105AB00097900100E780000017B501001305051459
:105AC000BDB617E4FF1F0344C46497E7FF1F83C7F5
:105AD000376497B501009385252A220417B5010084
:105AE0001305C5AA5D8C97900100E780A0FCA285F4
:105AF00017B50100130545E097900100E78080FB92
:105B0000294597900100E780C0FF194697E5FF1FE0
:105B100093850560228597E0FFFFE780C039AA845E
:105B20001DC197B501009385252517B50100130503
:105B3000E5A597900100E780E0F7A68517B501007D
:105B4000130585DC95B397E7FF1F239B875AB7E7BB
:105B50000400116603A38705130606E893050008F1
:105B600069B1854797B501009385052117B50100F7
:105B70001305C5A1630BF40097900100E78080F343
:105B800017B50100130585D95DB497900100E78032
:105B900060F217B501001305E5D997900100E78081
:105BA00060F1294597900100E780A0F52244B240BA
:105BB0009244024997E7FF1F239807524101176358
:105BC00000006700E39097B501009385E51A17B5CB
:105BD00001001305A59B97900100E780A0ED17B584
:105BE00001001305E505A1B4B240224492440249E4
:105BF00041018280411106C622C497E0FFFFE78081
:105C0000802B9377F50FA1C32A8497B50100938564
:105C1000251817B501001305659797900100E780D7
:105C200060E99375F40F17B50100130525359790BA
:105C30000100E78020E82244B24029454101179342
:105C40000100670003ECB24022444101828041110F
:105C500022C491462A8417E6FF1F1306A6599D65A4
:105C60002D4506C697D0FF1FE78000B6B7F707009F
:105C700003C70701A5476313F70001A093060010AF
:105C800001469D65254597D0FF1FE780E0B397E764
:105C9000FF1F238187562244B240914617E6FF1F1B
:105CA000130646559D652945410117D3FF1F67001F
:105CB000A3B11171CED7B7E9040083A7C904CAD92B
:105CC00017E9FF1F1309C944A2DD2E8686DFA6DB74
:105CD0002E84AA854A85829797E7FF1F83C747438B
:105CE0001307700A6385E710636DF7001307600AF6
:105CF0006385E704FE506E54DE544E59BE5911615F
:105D000082801307800A6385E7161307900AE393DE
:105D1000E7FE8D476306F41C97B50100938545396E
:105D200017B501001305858697900100E78080D89C
:105D300017B501001305053525A08D47630CF40246
:105D400097B501009385C53617B501001305058485
:105D500097900100E78000D617B501001305C52B09
:105D600097900100E78000D5294597900100E780D2
:105D700040D949B7854717B501001305A52B17E78B
:105D8000FF1F2303F73097900100E78080EAB77583
:105D90000200B76602000146054597D0FF1FE78065
:105DA000A0A2930760F817E7FF1F2303F73697E7D2
:105DB000FF1FA38007369307002617E7FF1F232B3B
:105DC000F734E5779387072117E7FF1F2316F7348A
:105DD000B14597E7FF1F2382073497E7FF1FA38E84
:105DE000A7324A8597000000E780E01621B7914767
:105DF00063E3870297B501009385852B17A5010002
:105E00001305C57897900100E780C0CA17B5010057
:105E100013054524B1B797E4FF1F83C4A42F97E768
:105E2000FF1F83C7172FA204DD8C83A7C9046D143D
:105E3000228697E5FF1F9385F52D280082978E0413
:105E400093160401B7750200C1823000A69509457A
:105E500097D0FF1FE7804097930770F817E7FF1F61
:105E60002308F72A994597E7FF1FA385A72A95BF1F
:105E7000914763E3870297B501009385652317A5D2
:105E800001001305A57097900100E780A0C217B527
:105E900001001305A51DE9B597E4FF1F83C48427FE
:105EA00097E7FF1F83C7F726A204DD8C83A7C904E9
:105EB0006D14228697E5FF1F9385D52528008297CC
:105EC0008E0493160401B7750200C1823000A695B6
:105ED0000D4597D0FF1FE780208F930780F8BDBF47
:105EE00017B501001305451B97900100E78060D4AA
:105EF000930790F82304F100834719008D4528008B
:105F0000A304F100834729002305F1009700000056
:105F1000E78060041305C01297C0FF1FE78060424E
:105F2000014597D0FFFFE780A0150D4597000000C1
:105F3000E78020D2294597C0FF1FE780804097C0A7
:105F4000FF1FE780E0307DB397E7FF1F23ACA72A50
:105F5000828097E7FF1F9387E72A03A30700630365
:105F60000300028317430000670003B541114AC0D4
:105F700097F6FF1F83D6E679328917D6FF1F03569F
:105F8000064422C426C206C62A84AE8497000000B6
:105F9000E780606435C12DC0994763FF970483474C
:105FA000140003470400A207D98F13978700A18329
:105FB000D98FC2073167C1831307C755639EE702B4
:105FC00097D7FF1F83D7A73FA301F400A183230224
:105FD000F40097F7FF1F83D7C77391C7A302F4009C
:105FE000A1832303F400A68517B50100130545100E
:105FF00097900100E78000AC97F7FF1F83C7076108
:10600000B9CF97D5FF1F83D5853B17B50100130581
:10601000E50F97900100E780E0A92686A28517D5B5
:10602000FF1F0355C53997000000E780E0BC6301FE
:10603000090497E7FF1F83C7271D9DCB95C897E7E6
:10604000FF1F83C767048DE722852244B2400249BF
:10605000A68592444101174300006700E3A517B5E8
:1060600001001305A50B97900100E78080BCC1B724
:10607000B240224492440249410182808347550044
:106080008345450017B5010013054505A207DD8DC1
:1060900017930100670003A217B50100130505035C
:1060A000179301006700E3B88D4763FBB70A01113E
:1060B00026CA06CE22CC0344350097E4FF1F83C4D2
:1060C000B41497B5010093852506B337800017E710
:1060D000FF1FA30BF71209C497B50100938585052F
:1060E00017B501001305850597900100E780809C96
:1060F00097E7FF1F83C7571163869700970000003B
:10610000E780202B97E7FF1F83C717108DC78547B0
:106110002306F100B7E7040083A747177000854501
:1061200013055030829717B501001305250297908B
:106130000100E78000B09967938757EE2316F100BE
:10614000680085479145A30781002307F100970068
:106150000000E78040E0F2406244D2440561828062
:106160008280894763F7B708011122CC06CE26CA80
:106170008344250085472A84639DF404914763F591
:10618000B704034545008347340022055D8D97D74A
:10619000FF1F2396A72297000000E780A04C996775
:1061A000938767EE2314F1008347340023059100A1
:1061B000A305F10083474400954528002306F1001C
:1061C00097000000E78020D9F2406244D244056184
:1061D0008280FDF89967938767EE2314F10097D7C3
:1061E000FF1F83D7C71DA305F10023050100A1836D
:1061F000E1B782800111996722CCD51717F4FF1FF0
:106200001304C4402314F1008347040026CA97F402
:10621000FF1F938404502305F10083D70400280056
:106220009545A305F100A18306CE2306F100970052
:106230000000E78040D203D604008345040017B570
:106240000100130525F297900100E780A086F24037
:106250006244D244056182809D677971D917231603
:10626000F10097F7FF1F83C7673A06D62307F100AF
:10627000A9C3B7E70400FC47414697E5FF1F938594
:1062800025E71305F10082976800CD4597000000CF
:10629000E78060CC97F5FF1F83C5453717B5010030
:1062A000130545EF97900100E780C080B25045612B
:1062B0008280B7E70400BC47414681451305F100E1
:1062C0008297D9B75DC1411106C622C4930750FA1F
:1062D0002300F5009307A005A300F50089472301DB
:1062E000F5009147A301F500F947A302F50097F7E0
:1062F000FF1F9387A73183C70700230205002A8465
:106300002303F50097E7FF1F938717F083C7070064
:10631000414697E5FF1F9385A5DDA303F50097F799
:10632000FF1F83D7073F2304F500A183A304F500D3
:1063300097D7FF1F83D7A7082305F500A183A305DF
:10634000F500B7E70400FC47310582972285F14547
:1063500097000000E7802024230EA4002181A30ED3
:10636000A400B24022444101828082805D710A858E
:1063700086C6A2C497000000E78000F537E4040059
:106380007C448A850810794682973C441305E103D2
:10639000094681458297101093050002014597D068
:1063A000FFFFE7804034B640264461618280B7C772
:1063B000A55A01119387C7333EC497E7FF1F83C7D0
:1063C000B7E43EC6B7F7070003C7070106CE22CCE5
:1063D000A5476313F70001A01164930504F0930629
:1063E00000100146254597C0FF1FE780E03D3000C3
:1063F000930504F0A146294597C0FF1FE780C03CE4
:1064000097E5FF1F83C555E017B50100130545E962
:1064100097800100E780006AF24062440561828053
:1064200001119165A1463000938505F02D4506CEFA
:1064300097C0FF1FE78040392247B7C7A55A938707
:10644000C7336314F702B24517B50100130585D8A9
:10645000B335B00097E7FF1FA388B7DA9780010034
:10646000E7804065F24005618280814517B50100F3
:10647000130585D897E7FF1FA38807D897800100E9
:10648000E780406397000000E780A0F2E1BFB7C754
:10649000A55A79719387F7353EC6B7E70400FC47E4
:1064A000AA8506D622D4414608088297B7F7070086
:1064B00003C70701A5476313F70001A01164930503
:1064C00004E8930600100146254597C0FF1FE780AA
:1064D000A02F7000930504E8D146294597C0FF1FFF
:1064E000E780802E17B50100130545DF9780010076
:1064F000E7802074B25022544561828079719165A1
:10650000D1467000938505E82D4506D697C0FF1F3C
:10651000E780802B3247B7C7A55A9387F73517B561
:106520000100130565D56310F702B7E70400FC47C7
:1065300017E5FF1F1305C5BB41460C08829717B529
:106540000100130565D197800100E780806EB2508D
:1065500045618280B7F7070003C70701A5476313AA
:10656000F70001A091654111930600100146938543
:1065700005E8254506C697C0FF1FE780E024B24026
:1065800017B50100130545C34101178301006700DA
:10659000436AC16769768146FD17050613970601B0
:1065A00041836364B7003E8582803307D50003478B
:1065B0000700B98F214713F817008583630508008A
:1065C000B18FC207C1837D171377F70F6DF785066B
:1065D000F1B741C5A547054763F2B70883471500E2
:1065E000034705003168A207D98F13978700A1835D
:1065F000D98FC207C1831308C855054763900707A1
:10660000411106C622C426C203442500914763F007
:1066100087049307540063ECF502A301C5002182AF
:106620002302C5009304340091C6A302D500A182C1
:106630002303D5002A84A68597000000E780A0F5F3
:1066400026942300A4002181A300A4000147B240A6
:10665000224492443A854101828005473A858280EE
:10666000B7C7A55A01119387E7343EC42AC6B7F7C6
:10667000070003C7070106CE22CC26CAA54763132D
:10668000F70001A091642A84938504EE930600101C
:106690000146254597C0FF1FE78000133000A14643
:1066A000938504EE294597C0FF1FE780E011A2857E
:1066B00017B501001305C5C097800100E780803F32
:1066C00097000000E780C0CAF2406244D2440561EE
:1066D000828001119165A1463000938505EE2D451C
:1066E00006CE97C0FF1FE780200E2247B7C7A55AE6
:1066F0009387E7346318F702B24517B50100130515
:10670000A5B197D7FF1F239CB7CAC205C181978047
:106710000100E780203A97000000E78060C5F24062
:1067200005618280D147D14517B501001305C5B079
:1067300017D7FF1F2315F7C897800100E780803720
:1067400017D5FF1F0355A5C797000000E78080F10C
:10675000F9B721C1411126C206C622C4AE848DC537
:106760002A8497000000E780205E97E7FF1F83C719
:10677000A7A999CB22852244B240A6859244410123
:106780001733000067004333B24022449244410172
:106790008280828001114AC806CE22CC26CA4EC60B
:1067A00093F715002E899DCFAD673717004093876B
:1067B000A7AA1CC397200000E780E0FEB7E704000B
:1067C000BC4F13060019854517D5FF1F034505BFAC
:1067D000829713451900F2406244D2444249B249BB
:1067E0000561828093F725006382071C17F7FF1F5E
:1067F000035707F2954763F9E70C014417F6FF1FAB
:10680000130606E19306300513055004130810041F
:106810009308B00413039005930764006374F704AE
:106820003A84FD5997F4FF1F83C484DE97F7FF1F56
:1068300083C717DEA204DD8CAD679387B7556383EA
:10684000F41463E3970AA9679387A7556386F41442
:10685000A28517F5FF1F1305A5DB97000000E78051
:1068600080EFF5A8B307860083C50700639AD504B7
:1068700083C517006396A50483C5270063920505A9
:1068800083C53700639ED50283C54700639A15030D
:1068900083C7570063966702A2890DE897F5FF1F2B
:1068A00083D505E7B3853541C20517F5FF1F1305ED
:1068B00025D6C1814E9597000000E780C0E965A804
:1068C00005044204418089BF3A84FD598547E3EBC2
:1068D00087F459CC854517F5FF1F130565D397003D
:1068E0000000E78040E769A0B1679387C7556380E0
:1068F000F404B5679387D755E39CF4F4A28517F5A4
:10690000FF1F1305E5D097300000E780E01A8947A4
:106910006307F4049305E4FFC205C18117F5FF1F67
:10692000130525CF97000000E78000420DA89700CF
:106930000000E780C04011C9A28517F5FF1F1305AD
:1069400025CD97000000E78020400546A28517F579
:10695000FF1F1305E5CB97F0FFFFE7806061A68579
:1069600017B501001305859997800100E780801411
:10697000FD57E395F9F297F7FF1F239B07D81345BF
:10698000290091BDA28517F5FF1F130565C897F073
:10699000FFFFE780E06EE1B7A28517F5FF1F130543
:1069A00025C797F0FFFFE780606F55BF93F745005D
:1069B0000145E38207E217B501001305659597804D
:1069C0000100E780002797300000E780E01D1345B5
:1069D000490011B5411122C437E404005C5C06C6CD
:1069E000354697A501009385A54317B5010013050A
:1069F000A509829711E917B5010013052592978023
:106A00000100E780002301A08327041C82972A84C9
:106A1000054597C00000E78040D697600100E780F9
:106A2000605B97600100E780603097B00000E7800E
:106A3000C0E72285B2402244410182801567B71722
:106A400000401307575598C3D8439D66558FD8C348
:106A5000D843FD76758FD8C3D8431367F70FD8C3D3
:106A600035671307C7CC98C382804111054506C618
:106A700022C426C297C0FFFFE780604A1305A00426
:106A800097B0FF1FE780A062757585457D1597C09B
:106A9000FFFFE78000347D7585451305F53697C007
:106AA000FFFFE780603D371400408327840A8D454F
:106AB0001305002093E707202324F40A97C0FFFF63
:106AC000E7802031B7E4040097C0FFFFE7804076FD
:106AD000C85897800100E780C01517B5010013055D
:106AE000A5FA97800100E780C0148327840C8545B0
:106AF000414593E707082324F40C97C0FFFFE78084
:106B0000A0378D451305000897C0FFFFE780C0360A
:106B100097C0FFFFE780A06337A5070013050512A4
:106B200097C0FFFFE780405F014597C0FFFFE78008
:106B3000606595450545894717F7FF1F230CF7BC8E
:106B400097C0FFFFE780A065B7E700E013070006E6
:106B5000238DE7403707000423A0E71097D0FFFFFD
:106B6000E780C0F697D0FFFFE780800A970000001B
:106B7000E78080E697000000E780C08A9700000069
:106B8000E78060B597E0FFFFE78000E7970000002F
:106B9000E780C01C97000000E780600B83A7040813
:106BA00017050000130545BF829797D7FF1F23875E
:106BB000A780BC4C130600648545829797000000AF
:106BC000E78000E897C0FF1FE78080820145828050
:106BD000B7F7070003C70701A547AE866316F7009E
:106BE0009397450191C301A0AA850146254517C386
:106BF000FF1F670063BD4111B2862E86AA852D4511
:106C000006C697C0FF1FE78020BCB2400145410186
:106C100082809307000463E8C7021D71A2CC2A8416
:106C2000080886CE32C697800100E78040DDB24674
:106C30001008A285294597C0FF1FE780E0B8F640FD
:106C40006644256182803955828041110D658D45EC
:106C500006C697C0FFFFE780C017B71700408D66D4
:106C600023A6D70A17F5FF1F130505AB1387C70A1D
:106C70009387870A1CC15CC5856689675CC958C152
:106C800014C518C9B7E70400B24003A3871E410129
:106C900002838145B307B5008387070089E717237F
:106CA00000006700C3C28505C205C181E5B7411177
:106CB00026C2E97797F4FF1F938484B622C4938792
:106CC000A7552E842381B4002E86AA8517F5FF1FB1
:106CD000130545B506C62390F400A38104009780F0
:106CE0000100E780C0D193052400C205C18117F5DA
:106CF000FF1F130505B397000000E780C089B38725
:106D000084002382A7002181A382A7009305640049
:106D10002244B24026859244C205C1814101172315
:106D200000006700C3BA09C99307800263E6B70091
:106D3000170300006700E3F7828017F5FF1F034584
:106D4000259F828097F7FF1F83C747AD89E71723E9
:106D500000006700C3B7828097F7FF1F83C727AF84
:106D600099EF411106C697200000E78040A2B2408B
:106D7000854717F7FF1F230CF7AC41018280828003
:106D8000630E0532638C05325D71CAC04EDE86C665
:106D9000A2C4A6C252DC56DA5AD85ED662D466D2F3
:106DA0006AD0B9472A89AE8963F9B706394697A5EB
:106DB00001009385655D97800100E780E0C131EDBA
:106DC0008347E900130710036394E702854717F729
:106DD000FF1F2305F7A417A501001305E55B97F72F
:106DE000FF1F239C07A297000000E780C0EA71A064
:106DF0001307000317A501001305055DE395E7FEE2
:106E000097F7FF1F238C07A097F7FF1F239707A073
:106E100017A501001305C559F9B797F7FF1F83C7D9
:106E2000E79F63870722BD6AB96B938CFA55014AC5
:106E300017FBFF1F130B0B90138CEB65938AFA66FD
:106E400005A8B307490183C6070097F7FF1F83D73B
:106E5000C79CB1E39307A005639BF600854717F72E
:106E6000FF1F231CF79A97F7FF1F2385D78C050A6E
:106E700093170A01C183E3E637FDB64026449644E2
:106E80000649F259625AD25A425BB25B225C925C6A
:106E9000025D61618280054D639BA7039307500AE1
:106EA000639EF600894717F7FF1F2318F79693078D
:106EB00050FA17F7FF1FA30FF78655BF9307A005DA
:106EC000E387F6FA97F7FF1F239907944DB71387C7
:106ED00017004207DA9741832380D70017F6FF1F78
:106EE000231DE6928D47E3F4E7F817F4FF1F0344F0
:106EF000948497F7FF1F83C7078422045D8C930750
:106F0000F4FFC207C1839306F00DE3EDF6FA930791
:106F10006400C207C183E31CF7F493052400C20593
:106F2000C18117F5FF1F1305058197F0FFFFE7806B
:106F3000806633078B008347570003474700A2074B
:106F4000D98F17F7FF1F231A078C6318F50E81449A
:106F5000630CA40197E4FF1F83C4047EA20497E797
:106F6000FF1F83C7777DDD8C170500001305E5DB68
:106F700097F0FFFFE78080FD63878407636D9C02C5
:106F80009387EB556382F40497E7FF1F83C7C77AA3
:106F900005476389E70681CB1387A7051377F70FAA
:106FA0008D4663F2E6081307F0072300E100A30013
:106FB000F10089459DA063829405E39754FD97F005
:106FC000FFFFE780A02911A8A28517E5FF1F130581
:106FD000A57697F0FFFFE780600D014597F0FFFF72
:106FE000E780C0F669B5A28517E5FF1F1305C574D4
:106FF00097F0FFFFE7802017CDB797F0FFFFE780FE
:10700000A01FE1BF930710F8130511002300F10042
:1070100097F0FFFFE780402BFD450A8597000000B1
:10702000E78020C95DBFA28517E5FF1F1305C57066
:1070300097F0FFFFE78020C84DB79307F007894519
:107040000A852310F10097000000E78080C605B58F
:10705000C14763FE3705414697A501009385053971
:107060004A8597800100E780209731E18347090135
:1070700013071003639CE700854717E7FF1F2309E9
:10708000F76A17A501001305A537B1BB1307000365
:1070900017A501001305C539E397E7D497E7FF1F4C
:1070A0002388076817A50100130505372DBBCE857A
:1070B0004A8597C0FFFFE7802011C1B3828041114C
:1070C00026C2AE848D4522C406C62A8497C0FFFF1F
:1070D000E78080DAB717004099C803A5C70C418D37
:1070E00023A6A70CB240224492444101828003A50A
:1070F000870C418D23A4A70CF5B7834705000347F0
:107100001500A207D98FC2076177C187130727200F
:10711000639AE70083452500370504001703000044
:10712000670023FA8280411193078008F3B7078034
:1071300093F787083EC601000100B7170040130708
:1071400070052380E704130780FA2380E704010019
:10715000010003C7D7001377F70EA386E70023804B
:107160000704B247F3A707800100010041018280B4
:10717000011106CE97000000E78020FB294597B05B
:10718000FF1FE780201BB7E700E03707400023A080
:10719000E71801000100B787004023810700238022
:1071A0000700A3800700B717004003D7A7014207D5
:1071B00041831377F7F342074183239DE7001307C9
:1071C000800873370780137787083AC601000100EB
:1071D000130770052380E704130780FA2380E70470
:1071E0000100010003C7D70013670701A386E7006A
:1071F00023800704B247F3A707800100010005655B
:107200008545130505C097C0FFFFE780E0C6F24043
:1072100097F7FF1FA384079C97F7FF1F2381079C05
:1072200097F7FF1F2386078A0561828017E6FF1FF5
:10723000130646628147B2861303F00FA94833084C
:10724000F6000348080013F7F70F6307A80C63065E
:1072500068008507E39517FF2947B387E600238079
:10726000A70097E7FF1F9387A75F5DA8411113D77A
:1072700065001347170006C693F63500058B954742
:1072800091CA054699476387C60009469D476383AF
:10729000C600A14713F645003336C00093F68503B8
:1072A000050685C2A145638BB604E145638AB60431
:1072B000930580026388B604930580036393B60048
:1072C000914697F5FF1F2382F58097E5FF1F238DD9
:1072D000C57E97E5FF1FA389D57EBE8517A5010052
:1072E0001305051A97700100E780C07CB2408547FE
:1072F00017E7FF1FA30BF77C410182808546D1B7BA
:107300008946C1B78D4675BF17A501001305C5197C
:10731000177301006700037A17E7FF1F130747542D
:10732000BA972380B700E147E302F5F493077002B0
:10733000E30CF5FC82802A8723800500814717E54E
:10734000FF1F130525511308F00F2946B306F5005A
:1073500083C606006396E60297E6FF1F93864650B3
:10736000B69783C7070005452380F5009947636EEC
:10737000F7029D4763FDE700E147630DF700828058
:10738000638506018507E393C7FC0145C5B72380E4
:1073900005008280B737004003C7370083C7050068
:1073A00093F70704D98F2380F5008280797126D264
:1073B0004AD097F4FF1F83C4648317F9FF1F130992
:1073C000298206D622D44ECE52CC56CA5AC8B3070A
:1073D000990083C7070093F7F70FA5C79387140099
:1073E00093F7F70F0D476361F70C17E7FF1F230FA4
:1073F000F77E97E7FF1F9387277FA69783C707002E
:107400001307100293F7F7036389E7226363F70A10
:10741000054463808720E382076809476389E7148E
:1074200013070002E387E752B7E700E037074000A1
:1074300023A0E71801000100CA942380040023A0C0
:10744000E710B787004003C76700058BE3080772A2
:1074500097E6FF1F83C6A6790547E393E6702947A1
:107460002381E70209472383E7022385E70297E7A1
:10747000FF1FA38D076497E7FF1FA38A0776B787CF
:107480000040A381070017E7FF1FA3030764054718
:107490002383E700B250225492540259F249624ABF
:1074A000D24A424B4561828097E7FF1F23800774D1
:1074B00089B7130730026386E70A63E6E714130708
:1074C0004002638AE70813070003E39FE7F497E7A6
:1074D000FF1F93872771A69703C70700A14713775C
:1074E000F70FE313F71617EAFF1F130A2A3883472B
:1074F0006A0097E6FF1F2381F65C97E7FF1F83C7AB
:10750000573791C7FD5797E6FF1F2387F65A97E530
:10751000FF1F83C5B53597E7FF1FA38FB75897E7C0
:10752000FF1F83C7A73493F907089306000493F756
:107530000706639DD74A9307A0096387F51463E4A0
:10754000B7109307F0056384F548930750096382E9
:10755000F52801440DABFD5717E7FF1F230DF75426
:10756000E1B5FD5717E7FF1F2306F75475BD17A5B3
:1075700001001305E50497700100E780806B97E731
:10758000FF1F93872766A69703C40700814917EA60
:10759000FF1F130A2A461374F40F97AA0100938A57
:1075A000AA0263C78904294597700100E7806055E6
:1075B000854717E7FF1FA30DF74217E7FF1F230AB1
:1075C000874217E7FF1F2303F75037E700E0B706AE
:1075D00040002320D7180100010037860040834770
:1075E000A60293F7370F2305F6022320D7102DBDEF
:1075F000B3073A0183C507005685850997700100D6
:10760000E780404B79BF854717E7FF1F2302F73E0E
:1076100021BD17E7FF1F1307E75C26970347070005
:1076200097E6FF1FA384F63097E6FF1F2381E6301D
:1076300017E7FF1F230CF748C5BB854717E7FF1F58
:107640002306F72ED5B39307400A638DF5349307CD
:10765000200B6388F5369307100AE39CF5EE830749
:107660002A00014463D1074297E7FF1F83C73720F1
:1076700093F63700638E061A0546638EC6220946C6
:107680006399C61A1D4775A217E5FF1F0345251EFE
:10769000C94717EAFF1F034A9A1D97E5FF1F83C5D5
:1076A000251D17E4FF1F0344B41C6319F510CD47D3
:1076B0006316FA1093077008639CF5021307300FE6
:1076C000B7170E006308E4001307900DB7B7040066
:1076D0006314E40817E7FF1F2326F73EBE8517A5AE
:1076E00001001305E5EE97700100E780A03C95B519
:1076F00093078008639DF50033048040B777460008
:107700001374F40F938787CDB3D78702E1B793073C
:107710009008639AF5003304804091671374F40F66
:107720009387C766D5B79307A008639BF50033041A
:107730008040B7173D001374F40F93870790E9B7A3
:107740009307B008639AF50033048040916713747F
:10775000F40F938797D04DBF93F5F5078D47639B43
:10776000F50033048040B7975B001374F40F9387E0
:1077700007D859BF8947639BF50033048040B7772A
:107780000B001374F40F9387071BBDBF8547639AE3
:10779000F50033048040DD671374F40F938767E3CB
:1077A000A5B789E9330480408D671374F40F93877C
:1077B00077DC99BFF1679387072029BF9700000006
:1077C000E78000A7A285528597000000E78040A6C9
:1077D00049B39305610017E5FF1F0345450917E409
:1077E000FF1F0344D40897000000E78000B593050D
:1077F0007100228597000000E78020B43C0017E765
:10780000FF1F232BF73C834761002304F1008347CC
:107810007100A304F100894717E7FF1F230EF72823
:107820008357810017E7FF1F2312F7040944A1AC17
:10783000154793F64700B336D00093F787038506C4
:1078400085C32146638BC7066146638AC706130654
:1078500080026388C706130680036393C7009147BD
:1078600017E6FF1F2302D62697E6FF1FA38EF624F6
:1078700097E7FF1F238BE72417E7FF1F034747FF07
:107880009376070497E7FF1F83C797FE8DEE137764
:10789000770C93067008630CD7021377F7078D46B1
:1078A000631ED70AB307F040B7955B0093F7F70F55
:1078B000938505D881A81947ADBF854755B7894736
:1078C00045B78D4771BF930670086311D702130740
:1078D000300FB7150E006389E7021307900DB7B597
:1078E00004006383E7021307700845BF9306800C0A
:1078F0006311D702B307F040B775460093F7F70F4F
:10790000938585CDB3D5F50297E7FF1F23ACB71A52
:10791000F9B39306900C631AD700B307F040916552
:1079200093F7F70F9385C566F1BF9306A00C631B11
:10793000D700B307F040B7153D0093F7F70F9385D5
:107940000590C9B79306B00CE319D7F4B307F0401C
:10795000916593F7F70F938595D06DB78946631BB3
:10796000D700B307F040B7750B0093F7F70F938577
:10797000051B49BF8546631AD700B307F040DD6594
:1079800093F7F70F938565E3B5BF09EBB307F040B5
:107990008D6593F7F70F938575DCADB7F16593852A
:1079A00005209DB783472A00C18B99C7854717E7F4
:1079B000FF1F2306F71071BE97E7FF1F23810710F3
:1079C00049BE854717E7FF1FA301F71059B63C00D2
:1079D00017E7FF1F2322F72009479307000323140B
:1079E000F10097E6FF1F2389E60C2DBD6399075828
:1079F000A94763EBB74417A701001307A7A58A059A
:107A0000BA959C41BA97828717E4FF1F034434E676
:107A1000094A630C440F636C8A0885476309F40ABA
:107A20009307F00F17E7FF1F0347070963F6E70007
:107A300017E7FF1F2302F70817EAFF1F034ACA07C9
:107A4000930700041374FA0F63F44701130400044E
:107A500097E7FF1F9387471883AA0700228617E539
:107A6000FF1F1305A5E0D685330A8A40A29A9770B6
:107A70000100E780C0F897E7FF1F238F470397E7D0
:107A8000FF1F23AB571597E7FF1F83C7F702154763
:107A90006399E762B7E700E03707400023A0E718E3
:107AA00001000100B78600402380860285A58D472E
:107AB000630CF40A9947E315F4F697A7010093873E
:107AC000E79F17E7FF1F2329F710A947A1BF17E773
:107AD000FF1F0347C71197E7FF1F9387E7FF49463B
:107AE00097A50100938585A66306870097A50100E9
:107AF0009385C5A13E8597700100E78040F017E7A8
:107B0000FF1F232BA70CC94731BF97E6FF1F83C672
:107B1000060E054797E7FF1F938707FC6394E6026D
:107B20003E851306700297A501009385A59F977067
:107B30000100E780C0EC17E7FF1F232FA70893077A
:107B40007002CDB53E851306300497A501009385DC
:107B5000A59797700100E78080EA17E7FF1F232DA4
:107B6000A706930730047DBD97E5FF1F83C525D089
:107B700017A50100130505A797700100E78080F3A2
:107B8000854A17EBFF1F034B8B0697E5FF1F83C545
:107B900005CE17A501001305E5A463185B0B9770CC
:107BA0000100E78020F197E7FF1F83C747CCB5CBE3
:107BB000E368F4E617A401001304849D638C670155
:107BC00017A401001304449D6386470117A4010014
:107BD0001304049E228597700100E780400E137500
:107BE000F50F93071500860717E7FF1F2306F7EE2B
:107BF0008D4717E7FF1FA301F7EE97E7FF1F938756
:107C0000A7ED0147BE861376F70F89076365A602C5
:107C100097E7FF1F23A2D7FC97E7FF1F83C7C7EB98
:107C200011B597A701009387A78F17E7FF1F23259B
:107C3000F7FA9147C5BB3306E40003460600A3806C
:107C4000070005072380C7007DBF97700100E7800C
:107C500060E697E7FF1F83C787C1E1D7E362F4DCE3
:107C600017A401001304C48F638C570117A40100EB
:107C70001304848F6386470117A401001304449002
:107C8000228597700100E78080031375F50F930735
:107C90001500860717E7FF1F2300F7E48D4717E756
:107CA000FF1FA30BF7E297E7FF1F9387E7E2014768
:107CB000BE861376F70F8907E37CA6F43306E4004B
:107CC00003460600A380070005072380C700D5B739
:107CD00097E5FF1F83C5A5B917A5010013054591B9
:107CE00097700100E78000DD97E7FF1F83C797DEED
:107CF00093E7470017E7FF1FA30EF7DC83472A002F
:107D000017E7FF1FA306F7DCA9B017A501001305AD
:107D1000658F97700100E780C0F197E7FF1F938799
:107D200027DB83C7070017E7FF1F2301F7B417E41A
:107D3000FF1F034464D833348000B1B317A501009A
:107D40001305858D97700100E780A0EE97E7FF1F70
:107D500083C757D893E7070117E7FF1FA30CF7D690
:107D600083472A0017E7FF1F2304F7D66FF06FFE43
:107D700017A501001305858B97700100E78060EB64
:107D800003470A007D8B51EFB787004003C76702A6
:107D90001377C70B136727002383E70203C7A702E4
:107DA0001377C70B136727002385E70203C7E70292
:107DB0001377C70B136727002387E70203C727033F
:107DC0001377C70B136727002389E702854717E757
:107DD000FF1F230DF7B417E7FF1F230BF7C017E7AB
:107DE000FF1F2309F7CC17E7FF1F2306F7CC97E700
:107DF000FF1FA38D07B297E7FF1FA38B07BE97E76F
:107E0000FF1FA38907CA97E7FF1FA38607CA97E743
:107E1000FF1FA38D07CA97E7FF1FA38A07DC6FF038
:107E20004FF389476312F70297E7FF1F83C747A401
:107E30009146638CD70863E0F604638EE70C6369B0
:107E4000F70A05476380E70EFD5717E7FF1FA305F5
:107E5000F7C637074000B7E700E023A0E7180100A6
:107E60000100B78600401306F0FC2381C60223A060
:107E7000E7106FF06FDB130720086382E708636287
:107E8000F70213071008E391E7FC378700408347A8
:107E9000670293F7C70B93E727002303F7026FF0FE
:107EA0004FEB130730086389E70213074008E39D8F
:107EB000E7F8378700408347270393F7C70B93E71B
:107EC00027002309F7026FF0CFE837870040834788
:107ED000270393F73707F5B7378700408347E70253
:107EE00093F7C70B93E727002307F7026FF06FE6BE
:107EF000378700408347E70293F73707F5B737879F
:107F000000408347A70293F7C70B93E72700230599
:107F1000F7026FF00FE4378700408347A70293F71B
:107F20003707F5B7378700408347670293F737076E
:107F3000ADB7179501001305657097700100E780D4
:107F400040CF97E7FF1F23830792D5B31795010012
:107F50001305C56F97700100E780A0CD97E7FF1F5D
:107F60002396079097E7FF1F938707B503C4070081
:107F7000894763F3870009441374F40F29B6130784
:107F80000002E393E7EC6399090A638FF500930716
:107F900020026381F508179501001305A56E9770FF
:107FA0000100E78020B14DB5179501001305C56AA2
:107FB00097700100E780E0C70144179B0100130B95
:107FC000EB6AA14AB3078A0083C507005A850504F6
:107FD00097700100E78000AEE31654FF179501008B
:107FE000130585C197700100E780A0C417E4FF1F47
:107FF0000344048811E497E7FF1F238B078461B4CF
:108000008947E313F4E4854717E7FF1F2302F7844A
:108010006FF02FD417E6FF1F0346768597E5FF1F05
:1080200083C5E584179501001305C56497700100A9
:10803000E78040A86FF0EFD1638FF504930710023B
:10804000E39BF5F497E5FF1F83C585821795010033
:108050001305456497700100E780C0A597E7FF1FEF
:1080600023AC47B797E7FF1F9387C7A5944383D7F0
:10807000470017E7FF1F034747A517D6FF1F232712
:10808000D67E1D4497D6FF1F2394F67E97D7FF1FF9
:108090002381E77ECDBA97D5FF1F83C5657D1795F0
:1080A00001001305A56097700100E780A0A097D795
:1080B000FF1F238F077897D7FF1F2399077A6FF049
:1080C000EFF62547E388E79C19476391E702B786F7
:1080D000004023808602B7E700E03707400023A076
:1080E000E71801000100130600FC41B31307100A52
:1080F0006391E702B786004023808602B7E700E07D
:108100003707400023A0E71801000100130680FC98
:10811000A9BB1307A009E38FE7FC1307400AE38B11
:10812000E7FC13072002E387E7960547E384E79619
:10813000B7E700E03707400023A0E718E39209966D
:1081400001000100B786004023808602130620FC50
:1081500029BB17E7FF1F034737966308F71E63E73E
:10816000E7029547630EF70E99476308F704B78651
:10817000004023800602B7E700E03707400023A055
:10818000E718010001001306A0FCC5B19307F00534
:10819000630AF700930750096306F700930710027C
:1081A000E317F7FCB7E700E03707400023A0E71824
:1081B00001000100B786004051BF97E9FF1F83C946
:1081C000A98F93070004CE8A63F43701930A000451
:1081D00097E7FF1F938747A003AA070013F4FA0F3E
:1081E0002286D28517D5FF1F1305456897700100B9
:1081F000E780E080B3878940529417E7FF1F230D83
:10820000F78A97E7FF1F23A9879C638E0902B78728
:10821000004023805703B7E600E03706400023A064
:10822000C6180100010003C7270213470704238172
:10823000E70203C727021377C70F2381E70223A0B2
:10824000C6106FF06F9EB786004023800602B7E726
:1082500000E03707400023A0E71801000100FDB54A
:10826000378700408347370097E6FF1F83C656864F
:1082700093F70708D58FA301F700B7064000B7E7CB
:1082800000E023A0D718010001001306A0FC230181
:10829000C70223A0D7106FF02F9997E7FF1F93878E
:1082A0006794A69783C7070093F7F70FD9CF97E78F
:1082B000FF1F83C7C793D1EB17D7FF1F0347D77F94
:1082C000930700026313F70897D7FF1F9387075A96
:1082D00003AB070097DAFF1F83CA8A5917DAFF1F1B
:1082E000034A1A5997D9FF1F83C9A958D2875687BD
:1082F000CE865A8697D5FF1F83C5855517950100F1
:108300001305453C97600100E780C07A97D7FF1FAF
:1083100023AA677B97D7FF1F2388577B97D7FF1F19
:10832000A384477B97D7FF1F2381377B97D7FF1FF6
:10833000A38F8750B7E700E03707400023A0E71876
:1083400001000100B7860040D1B3B7E700E037076E
:10835000400023A0E71801000100B786004025B5C2
:1083600029472381E70209472383E7022385E702A0
:108370002387E7022389E7026FF06F8F03C7670047
:10838000118B6309079083C75700918BB5CF17E70F
:10839000FF1F0347C78585476313F70697D7FF1F5E
:1083A000A385E77297D7FF1F2382075897D7FF1F30
:1083B0002380076497D7FF1F238E076E97D7FF1F71
:1083C000238B076E97D7FF1FA382075697D7FF1FF0
:1083D000A380076297D7FF1FA38E076C97D7FF1F55
:1083E000A38B076C97D7FF1FA382076E97D7FF1F3A
:1083F000A38F077EB787004011476FF06F8917D7AB
:10840000FF1FA306F74479BF854717D7FF1F230F28
:10841000F75017D7FF1F230DF75C17D7FF1F230B4C
:10842000F76817D7FF1F2308F76869BF854717D775
:10843000FF1F230DF74E17D7FF1F230BF75A17D730
:10844000FF1F2309F76617D7FF1F2306F76617D705
:10845000FF1FA30D074C17D7FF1FA30B075817D7F4
:10846000FF1FA309076497D7FF1FA38607648280B5
:10847000411106C697000000E78080FBB7870040E7
:1084800023800700130740FC2386E7001307C0047E
:10849000A386E70017D7FF1F1307473D2398E70080
:1084A00017D7FF1F13078740239AE70017D7FF1F2F
:1084B0001307074C239CE70017D7FF1F13078757A5
:1084C000239EE70029472381E70209472383E70228
:1084D0002385E7022387E7022389E702A3810700B8
:1084E000930600F8A380D700930690022380D7005C
:1084F000FD562383D7002381E700B706400037E706
:1085000000E02320D71003C7170013671700A380CC
:10851000E700B24097D7FF1F239C075A4101828092
:10852000411106C697000000E78080F0B787004041
:1085300023800700130700FC2386E7003147A3864A
:10854000E70017D7FF1F130767322398E70017D7F5
:10855000FF1F1307A735239AE70017D7FF1F13073D
:108560002741239CE70029472381E702094723830A
:10857000E7022385E702A3810700930600F8A380A2
:10858000D700930690022380D700FD562383D7009F
:108590002381E700B706400037E700E02320D7102B
:1085A00003C7170013671700A380E700B24097D7EF
:1085B000FF1F239F075041018280F16793870720A7
:1085C00017D7FF1F2320F750854717D7FF1F231DFD
:1085D000F74EA14717D7FF1F2309F74E97D7FF1F65
:1085E000A385074E97D7FF1F2382074E97D7FF1FFC
:1085F0002380072697D7FF1FA38B0724814717D512
:10860000FF1F13052525FD5517D6FF1F1306462509
:108610002947B306F5002380B600B306F600238091
:1086200006008507E397E7FE97D7FF1F238A075ABF
:1086300097D7FF1FA386075A97D7FF1F2383075A91
:1086400097D7FF1FA38B074697D7FF1FA38907461E
:1086500097D7FF1F2384074697D7FF1F238F074411
:1086600097D7FF1F238E074497D7FF1FA388074480
:1086700097D7FF1F2385074497D7FF1FA38307566C
:10868000828017D7FF1F0347875685476316F70079
:1086900017030000670003E917030000670083DD8C
:1086A000411106C697F0FFFFE78020A8514597A02B
:1086B000FF1FE78020C897000000E780C0FC371745
:1086C00000408357A701B24093E7070C231DF70032
:1086D000854717D7FF1FA303F75097D7FF1F2380A6
:1086E000075041018280411122C406C617D7FF1FDF
:1086F0000347E74F85472E8613F4F50FAA856317C6
:10870000F70417D5FF1F1305A52A97600100E7801E
:10871000002F97D7FF1F238D072CB7870040238496
:108720008702B7E600E03706400023A0C618010024
:10873000010003C7A7021377C70F2385E702B240E2
:10874000224423A0C61001454101828017D5FF1F96
:108750001305C51997600100E780602A97D7FF1FAE
:108760002386071CB787004023828702B7E600E014
:108770003706400023A0C6180100010003C76702A6
:108780001377C70F2383E7025DBF411106C6970029
:108790000000E780C0E2B240410117F3FFFF67002D
:1087A000639D97D7FF1F83C77743C1CBB78700402F
:1087B00083C75700918B91EB97D7FF1F2381074207
:1087C00097D7FF1F238C0740828097D7FF1F83C74F
:1087D000E74099C7FD1717D7FF1F2301F740828095
:1087E00097D7FF1F83C7A73F09476368F70085072F
:1087F00017D7FF1F2305F73E8280411106C697F069
:10880000FFFFE78020971305200397A0FF1FE78055
:1088100060B2B717004083A7470C13974701634B1B
:10882000070097000000E780E0E7F94717D7FF1F30
:108830002306F73AB24041018280828097D7FF1F1A
:1088400083C7D73989EFB717004083A7470C139721
:108850004701634B0706170300006700A3E44111BB
:1088600006C697F0FFFFE780A0B497D7FF1F83C726
:10887000F70BA1CB97D5FF1F83C5650B89C917D50A
:10888000FF1F1305E50A97E0FFFFE780A04F97D78A
:10889000FF1FA38D070897D7FF1F2389072237E7FC
:1088A00000E0B70640002320D718010001003786FA
:1088B00000408347660293F7370F2303F602232015
:1088C000D710B24041018280828041C9D9C597D773
:1088D000FF1F83C7E71FD1C3011122CC4AC84EC670
:1088E00056C25AC006CE26CA52C42E89AA8901444D
:1088F000930A0004371B030063772403B3078940FE
:10890000C207C183BE8463F4FA0093040004C20466
:10891000C180130A1BD497D7FF1F83C727019DE38C
:108920007D1A631C0A00F2406244D2444249B249B3
:10893000224A924A024B0561828097F0FFFFE7804E
:1089400020A7D1BF338589002694A68542049700CD
:108950000000E78080D9418045B7828097D7FF1F0C
:108960009387872C18429C4383D645000345070014
:1089700083C5C700035646006396A50083D5E7006C
:10898000638DD502011106CE2386A7002397D70059
:10899000B705CF00DC4B9385757D05077D162EC28C
:1089A000230001003AC42316C1002317D10099C344
:1089B0000A858297F240056182808280DC4DDC4B23
:1089C00081CFB7E70400904503A38705914517D5EC
:1089D000FF1F0345A525028382806D713C083EC6BA
:1089E000B707E500232291103EC8AA843C083285CF
:1089F000232611103ECA23248110232021112E8901
:108A000097300000E78020562A84979501009385CF
:108A1000E5CE17850100130565B797600100E78073
:108A20006009A285179501001305C5DD9760010057
:108A3000E7804008294597600100E780800CB70572
:108A4000CB009385757D680097100000E780405F3C
:108A5000A285680097300000E780404301478146C7
:108A60007000CA85268597200000E780C08205CD6A
:108A70002A8497950100938565C817850100130521
:108A8000E5B097600100E780E002A285179501003C
:108A9000130505D897600100E780C001294597605C
:108AA0000100E78000068320C11003248110832485
:108AB0004110032901105161828097D7FF1F9387CE
:108AC000A71618429C43797122D406D603480700A2
:108AD00083C807012A8483D6450003554600639660
:108AE000080183D82701638DD80223880701050771
:108AF0002399D7003708CC00DC4B1308787D3ACC9B
:108B00001307F5FF42CA23080100231EE100231FBB
:108B1000D10099C7080832C62EC482973246A245B2
:108B2000228597000000E78080EBB2502254456117
:108B300082806D713C083EC0B707E5003EC23C082C
:108B40003EC42326111023248110232291102317C1
:108B500001002318010023190100231A0100231B1F
:108B6000010097B7FF1F83D7E78799E3C167FD1718
:108B70002316F10097B7FF1F83D7E78691EB97D7AE
:108B8000FF1F9387670A9C439C43DC4783D70700FA
:108B900017B4FF1F13040485584C2317F1008357A3
:108BA0004400484B2318F10031E19795010093856B
:108BB000E5BB178501001305659D97600100E780FF
:108BC00060EF179501001305A5BB97600100E780D2
:108BD00060EE294597600100E780A0F28320C11074
:108BE00003248110832441105161828097A7FF1FC5
:108BF00083C7B77F89EBB7E70400BC5782975C4C0B
:108C000023AA0700E1BFFD1797A6FF1FA38FF67CDD
:108C100003560701834704014C470A85230BF100E3
:108C200097300000E780A02397D7FF1F9387C7FFE7
:108C30009C430147814688430A866C0097100000D8
:108C4000E7806065AA8429C197950100938505B2E4
:108C5000178501001305859397600100E78080E583
:108C6000A68517950100130565B297600100E7809E
:108C700060E4294597600100E780A0E8584CB7E719
:108C80000400BC57484B9DBF97A7FF1F83C7F775CC
:108C9000F5D7B7E70400BC4F1044854517D5FF1F33
:108CA0000345C5F882971DBF5C4EDC4BB9CFB1CDF3
:108CB000411122C4178501001305458D2E84979517
:108CC00001009385E5A806C697600100E78080DE75
:108CD000A28517950100130525AE97600100E78076
:108CE00060DD294597600100E780A0E1B7E7040057
:108CF0002244B24003A3870517D5FF1F034505F3A0
:108D0000130640069145410102838280411122C42D
:108D100017A4FF1F1304C46A1C4C06C689C7DC4392
:108D200099C34C488297584CB7E70400BC57484B4E
:108D300082975C4CB240224423AA07004101828002
:108D400017A7FF1F1307C769834707009306F00B98
:108D5000850793F7F70F63E9F60097A6FF1F2381B6
:108D6000F668034507008280930700F8FDB7835734
:108D700045006386071001114AC817A9FF1F130990
:108D8000696652C4032AC90106CE22CC03274A01D0
:108D900026CA4EC656C2F15735E31307D00DFD570C
:108DA000636EC704B7E9040083A709072A84130583
:108DB000860042054181B284AE8A8297232AAA00A6
:108DC0000325C9015C49A9E797950100938545965C
:108DD000177501001305857B97600100E78080CD42
:108DE00017950100130585A597600100E78080CCE9
:108DF000294597600100E780C0D0DD57F24062440A
:108E0000D2444249B249224A924A3E850561828053
:108E100093874400B705CF002319F5009385757D2E
:108E2000310597100000E780A0210325C901834583
:108E30006400310597300000E78040050325C90133
:108E40002686D685310597300000E78040017146BF
:108E5000A2854A8597600100E78060BA504419CA2C
:108E600083A78905854517D5FF1F034525DC829714
:108E7000814769B797000000E780E0CBD5BFFD5779
:108E80003E858280411126C297A4FF1F938484559A
:108E9000D84C22C437E404003C54484B06C68297A1
:108EA000DC4C0323C4052244B240924423AA0700A9
:108EB00017D5FF1F034585D7854541010283411121
:108EC00026C297D4FF1F938424D69C4006C622C492
:108ED0004AC0D5C3DC43C5C35CC12300B5002A84A6
:108EE0009795010093850580177501001305056AA4
:108EF00097600100E78000BC294597600100E7808A
:108F000040C09C4023A4070023A2070097A7FF1F8F
:108F10009387074BDC4FDC4B91C729559700000026
:108F2000E78000DF97A7FF1F9387C74BDC4FDC4B21
:108F300089C797000000E78020F537E90400832700
:108F4000C905894517D5FF1F034545CE829783275D
:108F5000C905914517D5FF1F034545CD82979C4014
:108F600003A347016309030022852244B2409244CF
:108F7000024941010283B240224492440249410124
:108F800082800111328506CE22CC26CA2E849730EB
:108F90000000E78040FDAA84978501009385C5778E
:108FA000177501001305855E97600100E78080B0AA
:108FB000030784000356640083554400A686179572
:108FC00001001305658197600100E780A0AE294587
:108FD00097600100E780E0B297A7FF1F83C7A73E15
:108FE000639D9700014597000000E78060D28145AE
:108FF0000A8597000000E780C0ECF2406244D2444A
:10900000056182806D712324811023261110232293
:10901000911093F745002E84638707143C083EC0E7
:10902000B707E5003EC23C083EC4231701002318E1
:10903000010023190100231A0100231B010097A737
:10904000FF1F83D7E73799E3C167FD172316F100A8
:1090500097A7FF1F83D7E73691EB97D7FF1F93871B
:10906000A7BC9C439C43DC4783D7070017A7FF1F7F
:10907000130707352317F100544F83574700231870
:10908000F100DC4AA1E7978501009385256D1775EE
:1090900001001305A54F97600100E780A0A1178587
:1090A00001001305E56D97600100E780A0A0294548
:1090B00097600100E780E0A4134544008320C110BD
:1090C00003248110832441105161828097A7FF1FE0
:1090D00083C7772F2555D9C3FD1717A6FF1FA304F4
:1090E000F62E03D6060183470701CC460A85230BDB
:1090F000F10097300000E78080D697D7FF1F938755
:10910000A7B29C4317A7FF1F1307872B9786010061
:109110009386066A88430A866C0097100000E780F1
:109120008017AA8451D99785010093852563177507
:1091300001001305A54597600100E780A097A6856B
:10914000178501001305856497600100E78080960C
:10915000294597600100E780C09A268597000000A6
:10916000E78000BB91BF93F725009DC7B7E70400D8
:10917000BC47414681452808829725559700000045
:10918000E78000B928089305F00F97000000E780FA
:1091900040D3134524001DB793F71500014599DF0F
:1091A00097000000E78020991345140001BF5C4D33
:1091B000411106C688C317D7FF1F2327F7A6B7E7B5
:1091C000040083A70708170500001305E5E382974D
:1091D000B24097D7FF1F238BA7A40145410182808E
:1091E00001113335A000A307A100B7E7040083A74E
:1091F000471706CE1306F1008545130550308297B8
:10920000F240056182808280411122C406C697D750
:10921000FF1F83C727A3014489EF97B7FF1F83C7A9
:10922000B7FE054499E717C4FF1F0344243E1344C7
:109230001400228597000000E780C0FA178501001E
:109240001305856B09E4178501001305E56B2244BE
:10925000B2404101176301006700C385797122D4D0
:10926000A30F010037E404008327841726D24AD0D5
:1092700006D6AA842E89130550309305F10132C613
:10928000829732468347F10193150601C18185CB50
:1092900001452EC697000000E780C0F483274417DD
:1092A000B2454A8626858297054597000000E780EB
:1092B00060F3B25022549254025945618280832750
:1092C00044174A8626858297EDB741119397050189
:1092D00022C406C626C2C1872E8463D40702B7E41F
:1092E0000400FC5417A5FF1F0345C512829719C13E
:1092F000BC5482972165218DB240224492444101A1
:10930000828093F715008DC7B7E7040083A7471A3B
:1093100017A6FF1F1306060F97D5FF1F9385C5914C
:1093200017A5FF1F0345050F829713451400E9B7E2
:1093300093F7250099CFB7E70400BC4F13060064EC
:10934000894517A5FF1F0345E50C829713452400A7
:1093500065B793F785009DC7B7E7040003A8871A90
:109360001307401F97A7FF1F83C7C70A814613062D
:109370004006994517D5FF1F0355058D02981345E3
:1093800084009DBF93F745000145BDD7B7E40400B5
:1093900083A7041817D5FF1F0355058B8297BC4C74
:1093A00013060064914517A5FF1F0345A506829784
:1093B0001345440091B797D7FF1F83D7E788639879
:1093C000A70217D7FF1F2312B78817D7FF1F231F26
:1093D000C78617D7FF1F231CD7862E861785010047
:1093E0001305C557BE85175301006700A36C178589
:1093F0000100130525581763010067008383035795
:10940000450097D7FF1F83D72784631AF704C167E6
:109410004111F91722C417D7FF1F2327F78237E41A
:10942000040097D7FF1F23A3078297D7FF1FA38BA3
:1094300007807C4C06C6894517A5FF1F034585FD9F
:1094400082977C4C914517A5FF1F0345A5FC829789
:109450002244B240410117030000670023DB178557
:10946000010013052551175301006700837C7D150A
:10947000954763E2A71C178701001307A7450A0554
:109480003A951C41011122CC06CEBA972E848287D0
:10949000178501001305854E97500100E78060791C
:1094A000A1A203C7250099476311F7022E859700F3
:1094B0000000E78000F5834564001785010013056F
:1094C000E54C97500100E780E05E97B7FF1F238DC2
:1094D00007D2178501001305254D7DBF03C7250061
:1094E00095476319F702C16717C7FF1F0357C77571
:1094F000F91703D5A5006309F702B7E7040083A7AE
:10950000C7178297178501001305054B9750010077
:10951000E7802072854717B7FF1F2307F7CE17850F
:1095200001001305E54B8DBF97C7FF1F239EA77052
:1095300083D7E50097C6FF1F2399F67083D70501EF
:1095400097C6FF1F2394F67083D7250197C6FF1F88
:10955000239FF66E97C7FF1FA386076E631BE50266
:10956000B7E70400BC4F096613060690A14517A58E
:10957000FF1F034525EA82970356E4008355A400A4
:10958000178501001305854497500100E78080523C
:1095900051B79307700F2316F100B7E7040083A7B4
:1095A000870D17A6FF1F0346E6E66C0082974DF96C
:1095B000854717C7FF1FA307F7685DB71785010029
:1095C0001305C542D1BD83C5250091476392F502BD
:1095D000178501001305054397500100E78060657A
:1095E00097000000E78080C2F240624405618280FB
:1095F00099476392F502228597000000E78060E0BA
:109600008345640017850100130545389750010014
:10961000E780404AD1BF9547639AF500834714001D
:10962000E1F31785010013052540BDB5178501003D
:1096300013050540E1BF82806D712324811023262C
:10964000111023229110328401CD8947630AF5025B
:109650008320C11003248110832441105161828032
:10966000178501001305853DAE8497500100E78002
:10967000405CA285268597C0FFFFE780A0F0C9BFA8
:10968000B7E70400FC4728008297178501001305FF
:10969000A53B97500100E780C0598347810039C43A
:1096A0001307000B6380E7021387A7051377F70FF3
:1096B0008D4663EDE602A285280097C0FFFFE78094
:1096C000805F79B78547E3F587F883459100177583
:1096D00001001305E520B335B00097B7FF1F2385C0
:1096E000B79A97500100E780E03C9DB7034791008F
:1096F000A207D98F35671307D7556385E7086368D5
:10970000F7022D671307B7556387E706316713071D
:10971000C755638AE70429671307A7556394E702CF
:10972000A285280097D0FFFFE780409715B73967DB
:109730009306E765638DD70663E9F6001307E755DF
:109740006380E706A28528003DB73D679306F7557D
:109750006386D7061307F766E396E7FE97D0FFFF09
:10976000E780C0AFF5B50146A285280097D0FFFF7E
:10977000E7800080F1BDA285280097D0FFFFE78039
:109780002090F9B58947E3F587EC9305E4FFC2051E
:10979000C1811305A10097A0FFFFE780E0A24DBDA6
:1097A000A285280097D0FFFFE780409055B5A2859D
:1097B000280097D0FFFFE780009B59BD97D0FFFF9F
:1097C000E78080A371B5411122C417A4FF1F1304C1
:1097D000A4C5AA8617860100130646112285C14535
:1097E00006C697500100E78000460357440097A73C
:1097F000FF1F938767C42393E700035764002394F4
:10980000E700B240224441018280411106C6970020
:109810000000E78080FBB7E7040083A7871417A642
:10982000FF1F130666C0D54501458297B2404D46DD
:1098300097A5FF1F938545C013057030410117039D
:1098400000006700E3A161712324811A37E404005A
:10985000832704082326111A2322911A2320211B6F
:10986000232E311917050000130565A6829717A945
:10987000FF1F130929BA994785442300A900231C17
:10988000F100978501009385650A930740061775D7
:1098900001001305A5CF231CF1082308910097C9E7
:1098A000FF1F938909E797500100E780A02083D527
:1098B0000900178501001305650697500100E78030
:1098C000601F294597500100E780A02303D50900B8
:1098D000896997000000E78040EF8327441710084C
:1098E00085451305503082978327441717A6FF1F1D
:1098F000130686B4CD45130570308297832744172D
:1099000017A6FF1F130646B1B545130560308297B1
:109910008327441730088945130510318297832720
:109920004417300989451305203182978327441550
:10993000938509900D458297832744159385099057
:1099400011458297A30591002306910023089100F9
:1099500002CD230C0100832784163009914513059D
:1099600070408297832784161306B100854513053E
:1099700000408297832784167000854513051040A8
:1099800082978327841630088545130520408297E7
:109990008327841610088545130550408297832736
:1099A00004157D558297832744137D5582977D55F5
:1099B00097A0FFFFE78000CC8327440C829797A0F5
:1099C000FFFFE78040A78327841417A6FF1F130615
:1099D000A6A5D5450145829789471306700F814595
:1099E00028092306F1009780FFFFE780C0708D47AC
:1099F0001306000881452808230CF1089780FFFF13
:109A0000E780606F9147230CF100977701009387FF
:109A100067A9984383C747003AC8230AF10097D043
:109A2000FFFFE780E09470008545054597A0FFFFA4
:109A3000E78060CB30099305700F094597A0FFFFC1
:109A4000E78060CA3008930500080D4597A0FFFF26
:109A5000E78060C910089545114597A0FFFFE78092
:109A600080C8C16717C7FF1F1307071EF9171CC35C
:109A70002322070017A5FF1F1305859997A0FFFF55
:109A8000E78040C58327C41D17C5FF1F1305451A6E
:109A900082973C4803450900854582978320C11A77
:109AA0000324811A8324411A0329011A8329C11925
:109AB0005D618280C16717C8FF1F0358E818F91756
:109AC0006301F8083DCDB5CD011126CAB7E4040005
:109AD00083A7841222CC2E862315B10006CE2A84B9
:109AE00001478146ED45428582972AC611ED1785CB
:109AF00001001305A5E497500100E7808013F240B0
:109B00006244D24405618280FC440356A100A285D0
:109B100082972C0017C5FF1F0355051397A0FFFF61
:109B2000E78000C869DD17850100130565E29750DD
:109B30000100E780001083A7C412ED45280082973A
:109B40007DBF8280411106C61DC9854717A7FF1F2B
:109B5000A309F78C354697A5FF1F9385E58B130561
:109B6000603097A7FF1F238F078A97F0FFFFE780DA
:109B7000206FB240410117F3FFFF6700236997A7E9
:109B8000FF1FA380078AF9B7C16717C5FF1F0355D9
:109B9000A50BF9176307F500B7E7040003A3C71780
:109BA00002838280854717C7FF1F230DF7080145F1
:109BB00017F3FFFF670003631783FFFFE702034FFD
:109BC0002A8408452E89B28919C900C19715000059
:109BD0009385A586610597300100E780C000814428
:109BE0007D5A97100000E780E03963C7A4048144E0
:109BF00097100000E780003A63C8A40497C7FF1FCE
:109C0000938707059C43DC47B307F94091872302FC
:109C1000F400638309048327C900B307F4409587E0
:109C2000A302F4001C4C89C79C4799C322858297E4
:109C30001783FFFF6700C34A5C4413971400850431
:109C4000BA972390470171BF1C48139714008504ED
:109C5000BA972390070069BF832789000547B30798
:109C6000F4409587A302F40083570400638EE70253
:109C70008DC309476384E7040D47E395E7FA9787A7
:109C800001009387272F1CCC978701009387872F8C
:109C900011A897870100938767F51CCC978701006F
:109CA0009387C7F55CC8BDBF97870100938707E11D
:109CB0001CCC97870100938767E1EDB79787010078
:109CC000938707301CCC9787010093876730D9BFF3
:109CD00095E51783FFFFE702033F004618448347DB
:109CE000940075839D8B6317F70097100000E78041
:109CF00060B448C41783FFFF6700233F8280178347
:109D0000FFFFE702A33A13893500C16442094111FC
:109D1000AA890144F11413590901054A2EC6971066
:109D20000000E7802026B2456348A40001454101B8
:109D30001783FFFF6700C33A83A7090013171400B6
:109D4000BA9783D707006388B7006394970063745A
:109D50002A010504E1B70545D9BF1783FFFFE702D4
:109D60000334AA892E89328BB6843A8ABE8A97A098
:109D70000000E78060FA71C9268597200000E7801F
:109D800020098D4763E7A7007D551783FFFF670014
:109D9000833483DB440097100000E780A0242A84EA
:109DA00097100000E7804025930774003144330585
:109DB000850263CDA70297100000E780A0229710CC
:109DC0000000E78020222A8497100000E780C0224C
:109DD0009307740031443305850263C3A7049710C9
:109DE0000000E78020209307450029A89710000075
:109DF000E7808020330585021307F0179307C0170B
:109E0000E35FA7FA2D55E3C277F963040B02D68608
:109E10005286A6854A8597200100E78060B9B5B7CC
:109E200097100000E780401D330585029307C5FFAA
:109E3000D1BF832749001385C90083D52700970028
:109E40000000E78000EC61F581B769553DBF97C719
:109E5000FF1F2391A7E097C7FF1F938767DF9043FA
:109E600081470C463307F500420741836393B700EF
:109E700082805446139847008507C2962390E600D7
:109E8000D5B797C7FF1F9387A7DC9C4303C58700FF
:109E9000828017C5FF1F0355E5DB82801783FFFF14
:109EA000E7026322C1671387D7FF630BE502636A8A
:109EB000A700F1176300F50201451783FFFF670054
:109EC000C3221387E7FF6302E502FD171D8D1335DB
:109ED0001500E5B797500000E78000267D15C5BF47
:109EE00097500000E78080FAD5BF97500000E780C8
:109EF000A0F8EDB71783FFFFE702E31C4111AA8426
:109F000001442EC697100000E780C008B2456348A0
:109F1000A400014541011783FFFF6700031D9C4812
:109F2000131514003E9583570500E385B7FE05041D
:109F3000C9BF03485500814693F7F60F63E5070153
:109F400081473E858280584593975600BA9703D73C
:109F500027006316B70003D70700E304C7FE850692
:109F6000E1BF8346450001479377F70F63E4D700CD
:109F7000814711A81C45131657000507B29703D651
:109F80000700E313B6FE3E8582801783FFFFE702DA
:109F9000E31193170501C18797CAFF1F938A4ACB24
:109FA000635BF00883A70A00C0479C47035704007F
:109FB000198D420541816368F500014422851783AC
:109FC000FFFF6700E31112052A94CDBFDC4713940D
:109FD0004900014A3E94834744006341FA02014A22
:109FE000834754006349FA028509C20993D90901DC
:109FF00083A70A009847E3EBE9FCC1B71C44131997
:10A000005A00A6853E994A8597000000E780C0EE79
:10A0100005E1050AC9B75C4413195A00A6853E99A3
:10A020004A8597000000E78020ED19E1050A4DBF41
:10A03000E30C09FA61B7AA8481495DBF1783FFFF6A
:10A04000E70263081C452A8481E79307C5001CC505
:10A050001C44231204001CC09307F00F63EDB700EB
:10A0600093F5F50F228597200000E78020E2178303
:10A07000FFFF6700830793940501C167C18063F9FF
:10A08000F500A685228597200000E78040E5C5B74A
:10A09000C18193F5F50F228597200000E78000DF4E
:10A0A000A685228597200000E78040E0C9B797C7C2
:10A0B000FF1F9387E7B9884382801C4599C797C7DC
:10A0C000FF1F23A7A7B8014582807D55828097C7CF
:10A0D000FF1F9387E7B79843834745004847920798
:10A0E0003E9582801783FFFFE702E3FD6171004523
:10A0F0001C183EC6B70780013EC81C183ECA8357CD
:10A10000440002CE02D002CC231EF100834784001B
:10A110002A8902D22301F1023C083ED402D69700DC
:10A120000000E78000FB835705002316F1029750DB
:10A130000000E780A0C32307A1025C400355640030
:10A14000F18313F717008347F10252055181F99B00
:10A15000D98FA307F10297100100E780C07439CDB1
:10A16000AA840355050097A00000E780C0BB83D7F1
:10A1700004002AD26800231CF10083D72400231D89
:10A18000F1001C4803D647008C4397200000E7806D
:10A1900000CD8347B400CA86178601001306868B5C
:10A1A0008117A305F4006C00481097200100E78098
:10A1B00020805D611783FFFF670023F32155D5BF22
:10A1C0001C45B1CF03C5A700894613576500630B33
:10A1D000D7028D46630ED70285466300D702130768
:10A1E00040063305E50203C7B700418B15CB83C793
:10A1F000B700BD8B3355F54082801375F503130707
:10A20000803EC5B709671375F50313070771D1BF02
:10A21000372709001375F5031307077CD9B70145E4
:10A2200082801783FFFFE70203EA03A98500630C1E
:10A2300009048347B900AE8493F7070E85C303452D
:10A240009900930520030D810505B305B5028844E7
:10A25000610597300100E78020A935A02E85970081
:10A260000000E78020F62A8419CD97000000E780DF
:10A27000605C8325C900B307B54063FA87002E945C
:10A28000B305A440E9F51783FFFF670003E68545A2
:10A290007DBF1783FFFFE70203E32A8403D5050090
:10A2A000011132C636C43AC22EC002CA02CC02CE56
:10A2B00097A00000E78020A782452ACA22852ECCDD
:10A2C00097000000E780E0E003570500231EE1004F
:10A2D00097500000E78080A9A24632469247230F9C
:10A2E000A10036874C08B2862285014697000000FF
:10A2F000E780E0A605611783FFFF670003DF178390
:10A30000FFFFE70243DC61711C183EC6B7078001FE
:10A310003EC81C183ECA3C0800453ED4AA8402CC64
:10A3200002CE02D002D202D697000000E78060DAA7
:10A330008357050035592316F10297500000E78036
:10A34000E0A22307A10209C48357440081EB2159ED
:10A350004A855D611783FFFF670023D903556400B9
:10A360005205518197100100E780E0532A8965D199
:10A370008347B40093F7070E99C7130584019730FC
:10A380000100E780A09883574400231EF100834713
:10A3900084002301F1025C4003550900D98313F7BF
:10A3A000070883471102231CA10093F7F707D98FF1
:10A3B000A300F10283572900231DF1005C40F183C3
:10A3C00013F717008347F102F99BD98FA307F10216
:10A3D00097A00000E78020952AD235D983479400C2
:10A3E0006800139757008347B400FD8BD98FA305EE
:10A3F000F4001C4803D647008C4397200000E780F8
:10A4000000A6A687177701001307C76474000546E6
:10A410004C10268597000000E78060942A890DD9AA
:10A420008347B400A685FD8BA305F40097000000C8
:10A43000E78060DF31BF1783FFFFE702C3C88324D3
:10A4400085FE2A844111268597000000E78080D789
:10A45000834734FF93F7070E8DCB2AC626859700D6
:10A460000000E78060C809CD834734FFB245FD8B0B
:10A47000A309F4FE91C5228597300100E780C086CC
:10A4800041011783FFFF670043C67DD98327C4FFBF
:10A490002685829775F5834734FF93F7070E91C79A
:10A4A000228597300100E7806086032584FE9700AF
:10A4B0000000E78000E5E9B71783FFFFE702A3BDCF
:10A4C0009C4141112A8903C7070089472E8493566E
:10A4D00067006380F6040D466388C6049307F0079F
:10A4E0006304F7022E8597200000E780C0A7AA84A6
:10A4F0008149C16B130C490097B7FF1F93874775BC
:10A500009C43984763E4E90441011783FFFF670018
:10A5100043BC03D745008547E3F8E7FE2E85972027
:10A520000000E780A0A9E1B703D74500E3FEE7FC00
:10A530002E8597200000E78000A3AA84228597201B
:10A540000000E78060A4C204C98C5DB7DC470355F6
:10A55000A900139A49003E9A93170501C187635DCC
:10A56000F00083570A006397A70263E77403832709
:10A57000CA00034D5A002DA0A1672167A98F1307B8
:10A58000F7EFE374F7FE6397090097000000E78098
:10A59000209161FD85098DB783278A00034D4A000C
:10A5A000835DA90003576900216A138BC7003AC66F
:10A5B000814A33CA4D01631E5D0197B7FF1F938720
:10A5C000A7699C43E1DBA286628681452685829746
:10A5D000D1B7A1679387F7EF930C4BFF63F2470363
:10A5E000B2455A8597F0FFFFE780A0710DC10327A0
:10A5F0008B00104709CE10436382C4023107D5BFD8
:10A60000EE85668597000000E780008F71F99386DC
:10A610001A0093FAF60F130B0B0271BF8356440016
:10A620005C43E3E9F6F622853AC697100000E7801E
:10A63000807DA1679387D7042A8A035D440032474F
:10A6400063E897008347D90093E707F8A306F9006A
:10A650001C4766852286E2858297C1670844FD17FC
:10A66000337AFA00529508C02312A40125B797B790
:10A67000FF1F9387E75D9843814715C314478147C0
:10A6800063FFD500939745004C47BE9519C903C792
:10A69000550081476375E600DC451606B2973E8596
:10A6A000828003C745008147E37BE6FE16069C4592
:10A6B000F5B71783FFFFE702639FAA892E8A8144BB
:10A6C00097BAFF1F938ACA5883A70A00984763E680
:10A6D000E4001783FFFF6700A3A0DC471394440046
:10A6E00001493E9413BB140083474400634BF900B7
:10A6F000014913BB140083475400634FF9008504DC
:10A70000E1B70844931759005287DA860146A285BB
:10A710003E9582990509C9BF48449317590052874D
:10A72000DA860546A2853E9582990509E9B7178321
:10A73000FFFFE7024399814517F5FFFF1305054821
:10A7400097B7FF1F2398075097000000E780A0F6F7
:10A750001783FFFF6700639997B7FF1F9387474FE2
:10A760009C4395C31783FFFFE702E395814517F5E7
:10A77000FFFF1305A54497000000E780C0F317838F
:10A78000FFFF6700839682801783FFFFE702039233
:10A7900037E404008327841241112315E100AE89B8
:10A7A0003289368A3A8681460147ED45AA848297E6
:10A7B0002AC621C90356A100D28597400100E7802F
:10A7C00000248327C413CE8526858297058905C971
:10A7D0008327440D2314210101462C0026858297EE
:10A7E0002A8401C9B7E7040083A7C712ED452800F2
:10A7F0008297228541011783FFFF6700638E4944DA
:10A80000D5B76554FDB75C41FD175CC182801783E5
:10A81000FFFFE702438BB7E70400FC5F8297954791
:10A820003305F50281450D811783FFFF6700E38B38
:10A830001783FFFFE7022389B7E70400FC5F8297D5
:10A8400095473305F5020D811783FFFF6700E38904
:10A850001783FFFFE7022387B7E7040083A7870B6F
:10A860000355050082971783FFFF6700038817834E
:10A87000FFFFE7024385035505003287AE86179632
:10A88000FF1F035686C197B5FF1F9385253D97008F
:10A890000000E780A0EF1783FFFF670003851783A1
:10A8A000FFFFE7024382B7E7040083A7C717829739
:10A8B0001783FFFF670063831783FFFFE702A3800F
:10A8C000B7E7040083A7871397B5FF1F9385053962
:10A8D000829701451783FFFF670023811773FFFFEE
:10A8E000E702637EB7E7040083A7C71F814517957A
:10A8F000FF1F035585B682971773FFFF6700E37E3E
:10A900001773FFFFE702237CB7E7040083A78713D1
:10A9100097B5FF1F93858535829701451773FFFF14
:10A920006700A37C1773FFFFE702E379B7E7040032
:10A9300083A7C71F81451795FF1F035505B8829749
:10A940001773FFFF6700637A1773FFFFE702A377B0
:10A950002E8597800000E78020AF97800000E78079
:10A9600020EC1773FFFF670043781773FFFFE702C0
:10A97000837597800000E78020F61773FFFF67005C
:10A98000C3765C49E1175CC95CC583572501A10703
:10A990002319F50083570501A1072318F5008280CC
:10A9A000F1473305F50297B7FF1F9387272E9C4386
:10A9B0003E9582808D476315F60803D7460085478C
:10A9C00063F0E7081773FFFFE702E36F368536840D
:10A9D0002E8997100000E780005929C98357440049
:10A9E00093140501C18063E397042285971000004A
:10A9F000E7806057FD14231294009307A0026300C0
:10AA0000F5029307B0026307F50293079002631FF4
:10AA1000F500228597000100E780008501A8014626
:10AA2000CA85228597A00000E780A0AF1773FFFFBB
:10AA30006700A36B228597100000E780C003FDB775
:10AA4000828097B6FF1F9386A6249C42014599CF2A
:10AA50009843D44217B6FF1F232CE6226396D700F3
:10AA600097B6FF1F23A8E6221385C7FE82801773BF
:10AA7000FFFFE702436597000000E780A04B7144A9
:10AA800033058502914597900000E78060E811E565
:10AA900065551773FFFF6700436597B7FF1F23A531
:10AAA000A71E97000000E780E04833058502914526
:10AAB00097900000E780C0E561DD97B7FF1F23A7EF
:10AAC000A71C97000000E780E04697B7FF1F239779
:10AAD000A71A97000000E780E04597B7FF1F239073
:10AAE000A71A97770100938727FC17B7FF1F232B1F
:10AAF000F71897070000938707E917B7FF1F23216F
:10AB0000F718014579B71773FFFFE702C35BAA8502
:10AB100017B5FF1F1305851697100000E780C05B6F
:10AB20001773FFFF6700635C1773FFFFE702A3590A
:10AB300097000000E78060FD97100000E780405B11
:10AB400097B7FF1F9387C7149C4391CF1387C7FE06
:10AB500019CB83D5C7FF17B5FF1F1305E513972042
:10AB60000100E78060181773FFFF67000358177331
:10AB7000FFFFE702435597000000E780C0EC09CDD6
:10AB8000834785002A8493F7070499EB0355E50072
:10AB900097000000E78080F91773FFFF6700E35418
:10ABA0008347C5009304450117B9FF1F1309490ED8
:10ABB00085E3832709005CC997B7FF1F23AA970C79
:10ABC00083274900F1FB97B7FF1F23A5970CE9B72F
:10ABD000FD172306F500610597800000E78000D689
:10ABE0008307840063CB07048347840093E707F857
:10ABF0002304F400B7E704009C5F82974205A9474D
:10AC000041813375F5028347840093F707FCC98FB0
:10AC10002304F4008347D4003E951C402318A4006D
:10AC200089CF984319CB8347C4005040814585079D
:10AC30003305F502420541810297832709005CC86C
:10AC400097B7FF1F23A697048327490089E797B783
:10AC5000FF1F23A197048347C4009DDF8355040190
:10AC600017B5FF1F1305450397200100E780C007B4
:10AC700025B71773FFFFE702034597B7FF1F9387B9
:10AC8000E7269C4701448583858B85E3AE84B285A6
:10AC90003A8697100000E780804B2A8419C59710E8
:10ACA0000000E780C041829408CC22851773FFFF23
:10ACB0006700A3431773FFFFE702433F41112E894B
:10ACC00032C6AA8997000000E780C03132471306D8
:10ACD0000502CA86970500009385C5CC17B5FF1FEE
:10ACE0001305C5F997000000E780E0F82A8425C91C
:10ACF0009304C50097000000E780E0411946AA854B
:10AD0000268597100000E7808015854526859710D9
:10AD10000000E7806011177501001305A5D64E9558
:10AD200083450500268597100000E78020165C48C3
:10AD300031468145A1075CC85CC483572401E117F3
:10AD40002319F40083570401E1172318F4001C4C65
:10AD50003E859770FFFFE780003AA3042501228516
:10AD600041011773FFFF6700A3371773FFFFE70267
:10AD700083354111AA842EC632C497100000E780A3
:10AD80006036004DB2452246834784000CC050C057
:10AD900093F7F70393E707042304F4002318040050
:10ADA000268597100000E780803183479400A946EC
:10ADB0002317A40013D7370005073307D7029D8B4D
:10ADC00085072306F400A306E40083C70401D848DE
:10ADD0008507230FF7FE17B7FF1F130767EB5843CD
:10ADE000232A04009307440129E317B7FF1F2323F5
:10ADF000F7EA17B7FF1F232DF7E817B4FF1F130457
:10AE0000A4E9228597200100E78040E01C44858B5F
:10AE10005D8D19E58145228597200100E780C0EC12
:10AE200041011773FFFF6700432C1CC317B7FF1FB7
:10AE30002322F7E6D9B71773FFFFE702C328970568
:10AE40000000938565B7014597000000E78000B0DA
:10AE500001451773FFFF670043291773FFFFE702E0
:10AE6000832697000000E78080B01773FFFF67001C
:10AE7000C3278347C500A5E31773FFFFE702A32499
:10AE80002A840355E50097000000E78000C821C12F
:10AE90008347840093F7F7FB2304F4001C4091C719
:10AEA000DC4381C74C400145829797000000E78052
:10AEB00080B917B5FF1F130525DE97200100E78035
:10AEC000E0E40355E40097000000E78020C6177314
:10AED000FFFF6700832182801773FFFFE702A31E35
:10AEE00097B7FF1F9387C7DA97050000938565C85A
:10AEF00017B5FF1F130545DA23A0070023A207009B
:10AF000097200100E78020CE1773FFFF6700E31D45
:10AF10001C4D91CFDC4381CF1773FFFFE702A31ACB
:10AF20008345070082971773FFFF6700031C828029
:10AF300097B7FF1F938787D89C4303C5070082807C
:10AF400097B7FF1F938787D79C4303C5170082805D
:10AF500097B7FF1F938787D69C4303C5270082803E
:10AF600097B7FF1F938787D59C4303C5470082800F
:10AF700097B7FF1F938787D49C4303C53700828010
:10AF800097B7FF1F938787D39C4303C557008280E1
:10AF900097B7FF1F938787D29C4303C567008280C2
:10AFA00097B7FF1F938787D19C4303C577008280A3
:10AFB00097B7FF1F938787D09C4303C58700828084
:10AFC00097B7FF1F938787CF9C4303C59700828065
:10AFD00097B7FF1F938787CE9C4303C5A700828046
:10AFE00097B7FF1F938787CD9C4303C5B70011E137
:10AFF0001D45828097B7FF1F938747CC9C4303C5AD
:10B00000C700828097B7FF1F938747CB9C4303C538
:10B01000D700828097B7FF1F938747CA9C4303C519
:10B02000E700828097B7FF1F938747C99C4303D5EA
:10B030000701828097B7FF1F938747C89C4303C5CA
:10B040002701828097B7FF1F938747C79C4303D58B
:10B050004701828097B7FF1F938747C69C4303D55C
:10B060006701828097B7FF1F938747C59C4303D52D
:10B070008701828097B7FF1F938747C49C4303C50E
:10B08000A701828097B7FF1F938747C39C4303C5DF
:10B09000B701828097B7FF1F938747C29C4303C5C0
:10B0A000C701828097B7FF1F938747C19C4303C5A1
:10B0B000D701828097B7FF1F938747C09C4388576B
:10B0C000828097B7FF1F938767BF9C4303D5C70252
:10B0D000828097B7FF1F938767BE9C4303D5E70223
:10B0E00019E11305800C828097B7FF1F938707BD76
:10B0F0009C4303C50703828097B7FF1F938707BC54
:10B100009C43C85B828097B7FF1F9387A7BA884389
:10B11000828097B7FF1F938727BA8843828019E1FF
:10B120007D558280F5DE984265DFFDD917B7FF1F98
:10B130001307C7DB1847AA877155058B631D0724C2
:10B1400003C507001547E37DA7FC03C737001305B8
:10B15000F0057D171377F70FE364E5FC03C3570091
:10B16000E30003FC83C86700E38C08FA03C7770099
:10B17000494579171377F70FE364E5FA03C7A7008A
:10B1800011481305F7FF1375F50FE36BA8F803CE0D
:10B1900097000D481305FEFF1375F50FE362A8F83D
:10B1A00003C8B7006309080065181378F80F130582
:10B1B000600DE36705F703C5C70079487915137576
:10B1C000F50FE36FA8F403C8D7000D457D18137879
:10B1D000F80FE36705F503D80701930E40175118E0
:10B1E000420813580801E3ED0EF303C8E7007D1889
:10B1F0001378F80FE36605F303C827017D18137869
:10B20000F80FE36F05F103C88700C54E7518137872
:10B21000F80FE3E70EF103D86701856E938EBEE069
:10B220006D18420813580801E3EC0EEF03D84701EC
:10B230006D18420813580801E3E40EEF03D88701A4
:10B240007918420813580801E36C05ED03C8A701FB
:10B250007D181378F80FE36505ED03C5B7011D48A8
:10B260007D151375F50FE36DA8EA03C5D701714885
:10B2700079151375F50FE365A8EA03D5E7011308FF
:10B28000E00F7D1542054181E36CA8E803C5070284
:10B29000494879151375F50FE364A8E8C85301C947
:10B2A00037C834005915130858BFE36BA8E603A844
:10B2B000870237C53400130555BF5918E36205E707
:10B2C00017B5FF1F232AC59E03C6050117B5FF1F2B
:10B2D0002326F59E0545E375C5E403D82501D0492D
:10B2E00033760603E31E06E203C61501E30A06E20F
:10B2F00017B6FF1F2320B69C83C52700014663872E
:10B30000A50003C61700F1453306B60283C707033D
:10B310009305C00272971A071307C70516031A97F9
:10B3200096084697B387B70241553E973297420732
:10B3300041836362E8061773FFFFE702C3D83685CF
:10B3400097800000E780E06797000100E780604792
:10B350002A8497A00000E780C0592A9497F0000043
:10B36000E780A0252A9497900000E780E0802A9447
:10B3700097F0FFFFE780E06F2A9497400000E78096
:10B3800060932A9497700000E780E09B22951773E2
:10B39000FFFF670083D582801773FFFFE702A3D208
:10B3A0004111A307A10097A00000E780E0C4930526
:10B3B000F100170500001305E5B597F0FFFFE780E2
:10B3C000802F014541011773FFFF670003D21773F8
:10B3D000FFFFE702C3CC17B4FF1F130424B10328F7
:10B3E000840079599368180097B4FF1F23A414B1FF
:10B3F0001378180063100802BA84BE89368B328A2B
:10B400002E89AA8A97F0FFFFE780E0A77D15269591
:10B4100019E531594A851773FFFF6700C3CB97F0D1
:10B42000FFFFE78040A67D152695A167E353F5FE53
:10B4300097B7FF1F938787E298433E8C814B01CBE0
:10B44000014597F00000E7806043933B15004A8573
:10B45000DA865686D28597900000E780004D2A89CB
:10B4600011CD1C44F99B17B7FF1F2325F7A883278D
:10B470000C00CDD3E3800BFA829769BF268597B77E
:10B48000FF1F23A707A697F0FFFFE780809C414698
:10B49000CE8517B5FF1F1305E5AE97300100E78095
:10B4A000005697D00000E78080980325040B97D0C2
:10B4B0000000E780409C054597D00000E78040A34E
:10B4C000054597000000E78060EDA9B797B7FF1F1B
:10B4D0009387C7A19C47858BEDC71773FFFFE702D2
:10B4E00083BE17B5FF1F130525A897B7FF1F23AF0E
:10B4F000079E97B7FF1F23AD079E97B7FF1F23AB8C
:10B50000079E97200100E780608097500000E78049
:10B5100020F597100100E780E04B97100100E780CD
:10B52000E05197B7FF1F9387E79A9C4391C7054562
:10B5300097800000E780801F97B7FF1F938747839E
:10B540009C4399C741657D1597700000E78080A1F5
:10B5500097F00000E780203D97D00000E780C08E84
:10B5600097B7FF1F938787AD9C43139717016356C7
:10B57000070097F00000E78040AC97B7FF1F23A3B8
:10B5800007A097B7FF1F23A107A097B7FF1F23AFFF
:10B59000079E97B7FF1F23AD079E97000000E78027
:10B5A000008C97000000E780007297F0FFFFE780B3
:10B5B000401897F00000E78080D51773FFFF670001
:10B5C000C3B2828097B7FF1F9387479288438280D8
:10B5D0001773FFFFE70223AF97800000E780A07496
:10B5E00097800000E78000771773FFFF6700E3AFE5
:10B5F0001773FFFFE70283AB2A849304140201113F
:10B600002E85B289A685214636C63A899730010033
:10B61000E780803C0DE9B24638082686CE851305C2
:10B62000940497500000E780A04021462C084A85EA
:10B6300097300100E780403A133515000561177314
:10B64000FFFF6700E3A90145D5BF1773FFFFE702BE
:10B6500083A79305450617A5FF1F13056566971079
:10B660000100E78060681773FFFF670003A8177386
:10B67000FFFFE70243A541112EC697F0FFFFE780C9
:10B68000601BB24588C141011773FFFF6700E3A546
:10B690001773FFFFE70283A1AA842E84978000001E
:10B6A000E780406BAA898545228597000000E780E6
:10B6B000E07D83C7E4011389940899E313890403A7
:10B6C000CE85228597000000E780407C21469305C7
:10B6D0001902228597000000E780607897B7FF1F66
:10B6E0009387C7808C43228597100000E780C08233
:10B6F000214693858402228597000000E78020760A
:10B700001773FFFF6700C39D1773FFFFE7022399BD
:10B71000397197F00000E78020B49305400661E995
:10B7200097800000E780405F6302051497A7FF1F22
:10B7300083C7C75A13B7170097A6FF1F2380E65A7F
:10B74000014499CFC16417A9FF1F1309297A9309EE
:10B75000400EFD1497000000E780C0866342A40AF3
:10B7600097F0FFFFE780000D4169B7290900096ADA
:10B77000FD7A2A8B81447D199389F97B130A0A711A
:10B78000938A8AC797000000E780C08363D7A40428
:10B790001304400EB387840217A7FF1F1307077512
:10B7A0000324070B3E948357C4016382270B184080
:10B7B0003307EB4063EAE900834744008507B3871A
:10B7C0004703D6976365F70801468145094597F019
:10B7D000FFFFE780604EAA8B29E597400000E780D5
:10B7E000C08285476317F50689659385057117A59E
:10B7F000FF1F1305E54C97100100E780E04E95A070
:10B80000B30734030327090BBA9703D7C7016308AB
:10B81000970003C75700A38207002382E7000504AF
:10B8200015BF9305C500228597000000E78080E6DC
:10B830005E852286976501009385052697F0FFFFB8
:10B84000E780E0525E8597100000E780608A8504FB
:10B8500015BF97A7FF1F938767699C478D83858BCB
:10B86000C1F721611773FFFF6700E3860146854535
:10B87000094502D002D202D402D697F0FFFFE7803A
:10B88000A043AA8479DD97F00000E780209C13890B
:10B89000C4002A8481454A8597000000E780005F44
:10B8A0000C4041464A8597000000E780405B8329B1
:10B8B00044006385090C4E8502D802DA02DC02DE00
:10B8C00097300100E780A03F2ACE141005462C08CF
:10B8D00008184ECC97500000E780200A1375F50F2A
:10B8E00051ED8355840093E525004A8597000000BB
:10B8F000E780E05E11460C104A8597000000E78063
:10B90000005601469765010093858519268597F0B5
:10B91000FFFFE780C045268597000000E780407D57
:10B920005C40A1D3014685450D4597F0FFFFE780B8
:10B93000A038AA841DD548401389C400973001005F
:10B94000E780E0372AC64A8597000000E780404C30
:10B950003246636FC5004C404A8597000000E7807F
:10B96000005001468145268597F0FFFFE780204083
:10B97000268597000000E780A077E5B58355840011
:10B98000ADB71763FFFFE702037497A7FF1F938705
:10B99000E7559C471DC193E7870017A5FF1F1305B7
:10B9A000253217A7FF1F2327F75497100100E780C0
:10B9B00080311763FFFF67004373DD9B17A7FF1FED
:10B9C000232AF75297300000E78020647DF117A505
:10B9D000FF1F1305E52E97100100E7802033D1BF2C
:10B9E0001763FFFFE702A36B4169AA892E8AB28A17
:10B9F000368BBA8B814417ACFF1F130C2C4F930C62
:10BA0000400E7D1997F0FFFFE780C05B63C4A40080
:10BA100001443DA03384940383270C0B3E94835749
:10BA2000C401638627055A87D6865286CE851305BC
:10BA3000040397000000E780E0BB01C923800B00EE
:10BA400022851763FFFF670003698347F40185C3FD
:10BA50005A87D6865286CE85130594089700000033
:10BA6000E78040B909C585472380FB00D1BF850425
:10BA700051BF835745006380071E1763FFFFE7022E
:10BA8000E36201112A8497000000E780C04D09C9D4
:10BA900085476309F50605611763FFFF6700436487
:10BAA00097E00000E780407B7DF5835744004947DD
:10BAB000ED9BE392E7FEC145228597000000E780F9
:10BAC0004033AA84228597000000E780204F035767
:10BAD000440002CE91472A89631AF7002285970015
:10BAE0000000E780A0513C082ACC3ECE97E0000041
:10BAF000E780C0755C55C5D374084A86A6850545A0
:10BB0000829751BF03574400D147E3F6E7F8032A71
:10BB10000400C169014997AAFF1F938A2A3D130BAC
:10BB2000400EFD1997F0FFFFE780C049634FA90E53
:10BB30002285032A040097000000E780C042A14547
:10BB40002A89228597000000E780A02AAA842285FE
:10BB500097000000E780804A14402A86AA89780866
:10BB60002685CA8597000000E780C0E7AA8405D52E
:10BB700003C7F40189476315F7008347C10181DFDB
:10BB80005546D2851385640097300100E78020E791
:10BB9000014597800000E780001901C583D7C401E3
:10BBA000A5E797A7FF1F938767349C479355190014
:10BBB000858913D73700058B01CF8983858B6399DE
:10BBC000B70001452EC697000000E780C0DBB245F4
:10BBD0004E8597800000E780A01E0346C1012A849D
:10BBE00093751900268597900000E780203935C1AC
:10BBF000268597800000E7802018268511C0014522
:10BC000097800000E780404B97300000E780E03FDE
:10BC10008547E312F5E883C754001307F00FE38C60
:10BC2000E7E68507A382F400BDB5B304690383A7E3
:10BC30000A0BBE9483D7C401638B37015546D28566
:10BC40001385640097300100E78000D955DD0509B0
:10BC5000D1BD5DD86DB782801763FFFFE702034552
:10BC600097800000E780400B05C1C164014417A91B
:10BC7000FF1F1309A9279309400EFD1497F0FFFF3A
:10BC8000E7804034634EA40017A5FF1F130545034A
:10BC900097100100E78020031763FFFF670043440C
:10BCA000330534038327090B3E958357C501638809
:10BCB00097002312050097800000E780E00B050441
:10BCC00075BF97A7FF1F938767229C478D83858B3E
:10BCD0008DE31763FFFFE702033F17A5FF1F13055F
:10BCE00025FE97100100E78060021763FFFF6700E1
:10BCF000C33F82801763FFFFE702E33C9705000024
:10BD00009385C5A017A5FF1F130585FB971001009C
:10BD1000E78060ED1763FFFF6700233D1763FFFFB8
:10BD2000E702633A8841B7E70400BC5B05054205BA
:10BD30004181829709C585472300F50005051763F2
:10BD4000FFFF6700833A83C7F5FF2E858507A38F22
:10BD5000F5FE828083C7F5FFFD1793F7F70FA38FDA
:10BD6000F5FE99EF1763FFFFE702E335B7E704003D
:10BD7000BC571385F5FF82971763FFFF6700E33613
:10BD800082801C41035745008D8FBA951CC1231238
:10BD9000B5003E85828093D78500A2051441DD8DD4
:10BDA000835745001387E6FF18C189072312F50062
:10BDB00013D685004111238FB6FEA38FC6FE410125
:10BDC000828018419307F7FF1CC183574500850700
:10BDD0002312F500A30FB7FE8280835745008D8F95
:10BDE0002312F5001C41BE950CC12E858280AA87C6
:10BDF00003D7470008410D8FAA952392E7008CC313
:10BE00008280184108453305A7408280835745004A
:10BE1000035765001D8F1C4108453385A740330536
:10BE2000A74082801763FFFFE702E32941112EC676
:10BE30002A8497000000E780A0FDB2456373B50037
:10BE400001A0835744000840BE952312B4003E95DC
:10BE500041011763FFFF670043291763FFFFE702F4
:10BE6000832641112E84B28532C697000000E780F8
:10BE7000A0FB3246A28597300100E78040B841011F
:10BE80001763FFFF670063261763FFFFE702A32323
:10BE90002E84854597000000E78000F92300850087
:10BEA0001763FFFF670063241763FFFFE702A32107
:10BEB00041112317B100894597000000E780C0F6C3
:10BEC0008347E1002300F5008347F100A300F5005C
:10BED00041011763FFFF670043211763FFFFE7027C
:10BEE000831E93D78500A2054111DD8D2317B10074
:10BEF000894597000000E78020F38347E100230095
:10BF0000F5008347F100A300F50041011763FFFF2F
:10BF10006700A31D1763FFFFE702E31A139785016C
:10BF200093D78501C166938606F0D98F13D7850014
:10BF3000758FD98FA2053707FF00F98D4111DD8D6F
:10BF40002EC6914597000000E78000EE6C00114678
:10BF500097300100E780A0AA41011763FFFF670047
:10BF6000C3181763FFFFE70203161C41854503C48E
:10BF7000070097000000E78080E622851763FFFF37
:10BF80006700A3161763FFFFE702E3131C4141118B
:10BF9000894503C7070083C717002307E100A307EC
:10BFA000F10097000000E78080E30355E1004101C4
:10BFB0001763FFFF670063131763FFFFE702A31018
:10BFC0001C414111894503C7070083C71700230798
:10BFD000E100A307F10097000000E78040E08357ED
:10BFE000E100410113D58700A2075D8D4205418123
:10BFF0001763FFFF6700630F1763FFFFE702A30CE0
:10C000000C4141112A841146680097300100E780F5
:10C01000009F9145228597000000E78040DCB247F1
:10C02000C166938606F01397870113D58701598D52
:10C0300013D78700758F598DA2073707FF00F98F37
:10C040005D8D41011763FFFF6700230A1C45BE9504
:10C050000CC18280AE87944391E6584101EF0CC138
:10C060005CC1828003C7570013671700A382E700F3
:10C07000B687D5B70CC3EDB7AA87084119CD1841CB
:10C08000D44398C36313D500D8C32A870346570007
:10C090009376160081E6232007008280944381CAAC
:10C0A0008C4203A847008CC363930601CCC3799AE2
:10C0B00014C3A302C7003687D1BF1C45DC471D8DC2
:10C0C000B777DBB6938777DB09853305F502420541
:10C0D00041818280F147B385F50248452E958280E3
:10C0E0008347450085072302F50082801763FFFF21
:10C0F000E70263FD2A8409E41763FFFF6700E3FE9C
:10C1000083474400F5DBFD1793F7F70F2302F40094
:10C11000E5F71C4403D7270005072391E700DC431C
:10C1200099C3228582974C4889CD83475400898BD7
:10C1300099E71C4422859C479C439C478297232A6D
:10C1400004000040232004007DB71763FFFFE702CF
:10C1500083F78357250041112EC681EB01442285C8
:10C1600041011763FFFF670043F80357050081474C
:10C17000F146E305F7FEB385D702404585072E94C7
:10C180008345440008C4F5F5B247AA8481E7232A11
:10C19000040009A81C456C0022859C439C4382979F
:10C1A00048C84DDD85472312F400B2472320040020
:10C1B000231804002319F4005C485CC483D72400CE
:10C1C000FD172391F40061BF1763FFFFE702A3EFA0
:10C1D00097A7FF1F9387C7B0884323260500232412
:10C1E0000500410597100100E78040B21763FFFF8B
:10C1F0006700A3EF1763FFFFE702E3EC17A4FF1F3D
:10C20000130404AE1C40411199CF9C472300B50094
:10C210002AC65CC197000000E78040FB1C40DC435D
:10C2200099C33245829741011763FFFF6700E3EB33
:10C230000347450029E3584DAA877D551DCF176355
:10C24000FFFFE70243E81CC3DC4797A6FF1F23A9B3
:10C25000E6A8F156130507012390D70097050000C3
:10C260009385050297100100E780E0970145176369
:10C27000FFFF670083E77D55828082801763FFFFA1
:10C28000E70263E401116146814528009760FFFFE2
:10C29000E78060E697A7FF1F938787A49C43280049
:10C2A0009305F00FDC473EC697000000E780C0F41E
:10C2B00005611763FFFF670043E397A7FF1F93879D
:10C2C00027A29C43D847A1679387C702631EF70A3A
:10C2D000397106DE22DC26DA80004AD84ED652D4E6
:10C2E00056D23285B28497000000E780C0C7AA8981
:10C2F000268597000000E78020C92318A4FC268526
:10C3000097000000E78040C82319A4FC2685970009
:10C310000000E78060C783D744000A8A231AA4FC80
:10C32000858393F7F70F230EF4FC8607BD0793F779
:10C33000073F3301F1408A8A01498347C4FD63679F
:10C34000F902CE85130584FC232C54FD97000000D0
:10C35000E78080EA5281130104FCF2506254D25407
:10C360004259B259225A925A2161828026859700F9
:10C370000000E78060C193171900D6970509239044
:10C38000A7001379F90F55BF828097A7FF1F9387E6
:10C3900027959C43D847A1679387A702631AF70A9A
:10C3A000397106DE22DC26DA80004AD84ED652D415
:10C3B00056D23285B28497000000E780C0BAAA89BD
:10C3C000268597000000E78020BCFD572318A4FCB9
:10C3D00026852319F4FC97000000E780E0BA83D794
:10C3E00044000A8A231AA4FC858393F7F70F230ECF
:10C3F000F4FC8607BD0793F7073F3301F1408A8AB3
:10C4000001498347C4FD6367F902CE85130584FCA7
:10C41000232C54FD97000000E78000DE52811301B9
:10C4200004FCF2506254D2544259B259225A925AE0
:10C4300021618280268597000000E780E0B4931791
:10C440001900D69705092390A7001379F90F55BF56
:10C45000828097A7FF1F9387A7889C43D847A1672F
:10C4600089076310F70A397106DE22DC26DA8000BC
:10C470004AD84ED652D456D232853289970000001F
:10C48000E78060AEAA894A8597000000E780C0AFC8
:10C49000835749000A8A2318A4FC858393F7F70F72
:10C4A000230CF4FC8607BD0793F7073F3301F140E7
:10C4B0008A8A8144834784FD63E7F402CE851305AD
:10C4C00084FC232A54FD97000000E780E0D25281CB
:10C4D000130104FCF2506254D2544259B259225A08
:10C4E000925A216182804A8597000000E780C0A9A6
:10C4F00093971400D69785042390A70093F4F40F24
:10C5000055BF82809797FF1F9387877D9C43D847AD
:10C51000A1679387E704631EF70A397106DE22DC00
:10C5200026DA80004AD84ED652D456D23285B2840A
:10C5300097000000E78020A3AA89268597000000C5
:10C54000E78080A42318A4FC268597000000E780DC
:10C55000A0A3231AA4FC268597000000E780C0A2B0
:10C5600083D744000A8A2319A4FC858393F7F70F25
:10C57000230EF4FC8607BD0793F7073F3301F14014
:10C580008A8A01498347C4FD6367F902CE85130592
:10C5900084FC232C54FD97000000E780E0C5528105
:10C5A000130104FCF2506254D2544259B259225A37
:10C5B000925A21618280268597000000E780C09C06
:10C5C00093171900D69705092390A7001379F90F3F
:10C5D00055BF82809797FF1F938787709C43D847EA
:10C5E000A1679387C704631AF70A397106DE22DC54
:10C5F00026DA80004AD84ED652D456D23285B2843A
:10C6000097000000E7802096AA8926859700000001
:10C61000E7808097FD572318A4FC2685231AF4FC95
:10C6200097000000E780409683D744000A8A2319C8
:10C63000A4FC858393F7F70F230EF4FC8607BD0750
:10C6400093F7073F3301F1408A8A01498347C4FDCC
:10C650006367F902CE85130584FC232C54FD9700F3
:10C660000000E78060B95281130104FCF25062546B
:10C67000D2544259B259225A925A21618280268557
:10C6800097000000E780409093171900D69705099E
:10C690002390A7001379F90F55BF82809797FF1F4A
:10C6A000938707649C43D847A167DD076317F704A6
:10C6B0001763FFFFE70223A1797132853284970067
:10C6C0000000E780408A2AC6228597000000E780A4
:10C6D000A08B2311A102228597000000E780A0888B
:10C6E000B2452300A102280897000000E780C0B0EF
:10C6F00045611763FFFF6700439F82809797FF1F85
:10C700009387075E9C43D847A16793878704631785
:10C71000F7041763FFFFE702039B797132853284C8
:10C7200097000000E78020842AC622859700000039
:10C73000E78080852311A102228597000000E78011
:10C740008082B2452300A102280897000000E780FC
:10C75000A0AA45611763FFFF67002399828097971E
:10C76000FF1F9387E7579C43D847A1679387A70488
:10C770006312F7021763FFFFE702E3940111280039
:10C78000814597000000E78020A705611763FFFF40
:10C790006700A39582809797FF1F938767549C43F8
:10C7A000D847A167938757026319F7021763FFFF02
:10C7B000E70263910111328597F0FFFFE780A07ACD
:10C7C0002308A1008145280097000000E780C0A24F
:10C7D00005611763FFFF6700439182809797FF1FF2
:10C7E000938707509C43D847A1679387E702631B51
:10C7F000F7041763FFFFE702038D011132853284CE
:10C8000097F0FFFFE7804078AA84228597F0FFFF2A
:10C81000E7808077854709E9228597F0FFFFE78069
:10C8200080744205B337A000280081452318910089
:10C830003ECA97000000E780209C05611763FFFF58
:10C840006700A38A82809797FF1F938767499C435D
:10C85000D84799476313F7081763FFFFE702A386DA
:10C8600079713285328497F0FFFFE780C06F2AC666
:10C87000228597F0FFFFE78020712310A102228517
:10C8800097F0FFFFE780206E2301A102228597F039
:10C89000FFFFE780406DA301A102228597F0FFFF13
:10C8A000E780606C2302A102228597F0FFFFE780FA
:10C8B000806B2313A102228597F0FFFFE780A06A17
:10C8C000B2452314A102280897000000E780C09217
:10C8D00045611763FFFF6700438182809797FF1FC1
:10C8E000938707409C43D847A1679387C703631387
:10C8F000F7081753FFFFE702037D79713285328411
:10C9000097F0FFFFE78020662AC6228597F0FFFF99
:10C91000E78080672310A102228597F0FFFFE78060
:10C92000A0662311A102228597F0FFFFE780A06394
:10C930002302A102228597F0FFFFE780C062A302D5
:10C94000A102228597F0FFFFE780E0612303A102A7
:10C95000228597F0FFFFE7800061B245A303A102A3
:10C96000280897000000E780208945611753FFFFE2
:10C970006700A37782801753FFFFE702C37401119A
:10C980002A8497F0FFFFE780005EAA84228597F053
:10C99000FFFFE780605F228597F0FFFFE780C05EC2
:10C9A000035744008D4763F7E700228597F0FFFFA8
:10C9B000E780805D228597F0FFFFE780E05C28003C
:10C9C000A68597000000E780208305611753FFFFCD
:10C9D0006700A3719797FF1F938787309C43D847C1
:10C9E000A167FD07631FF7001753FFFFE702A36D61
:10C9F000328597000000E78040F81753FFFF67007B
:10CA0000C36E82809797FF1F9387872D9C43D847DB
:10CA1000A167E5076315F7081753FFFFE702A36A4D
:10CA200079713285328497F0FFFFE780C0532AC6C0
:10CA3000228597F0FFFFE7802055228597F0FFFFC2
:10CA4000E78080542310A102228597F0FFFFE78042
:10CA5000A053520551812311A10222852302010214
:10CA600097F0FFFFE7802050A302A102228597F0F4
:10CA7000FFFFE780404F2303A102228597F0FFFFCD
:10CA8000E780604EB245A303A102280897F0FFFF9C
:10CA9000E780807645611753FFFF6700036582805A
:10CAA0009797FF1F9387C7239C43D847A167938716
:10CAB000E703631FF7001753FFFFE702C3603285E8
:10CAC00097000000E78060EB1753FFFF6700E3610A
:10CAD00082809797FF1F9387A7209C43D847A16721
:10CAE00093874704631EF7021753FFFFE702A35D16
:10CAF00079713285328497F0FFFFE780C0462AC6FD
:10CB0000228597F0FFFFE7802048B245280897F07C
:10CB1000FFFFE780606E45611753FFFF6700E35C2E
:10CB200082809797FF1F9387A71B9C43D847A167D5
:10CB3000938787026310F7041753FFFFE702A35898
:10CB400079713285328497F0FFFFE780C0412AC6B1
:10CB5000228597F0FFFFE7800041B2452300A10244
:10CB6000280897F0FFFFE780206945611753FFFF12
:10CB70006700A35782801753FFFFE702C3540111D8
:10CB800097F0FFFFE780203EAA85280097F0FFFF7F
:10CB9000E780806605611753FFFF6700035597978D
:10CBA000FF1F9387E7139C43D847A167D107631FF3
:10CBB000F7001753FFFFE70203513285970000008B
:10CBC000E780A0FB1753FFFF6700235282809797EF
:10CBD000FF1F9387E7109C43D847A167C507631FD2
:10CBE000F7001753FFFFE702034E3285970000005E
:10CBF000E780A0F81753FFFF6700234F82809797C5
:10CC0000FF1F9387E70D9C43D847A167B907631FB0
:10CC1000F7001753FFFFE702034B32859700000030
:10CC2000E780A0F51753FFFF6700234C828097979A
:10CC3000FF1F9387E70A9C43D847A167AD07631F8F
:10CC4000F7001753FFFFE702034832859700000003
:10CC5000E780A0F21753FFFF670023498280979770
:10CC6000FF1F9387E7079C43D84789476318F7025C
:10CC70001753FFFFE70223450111328532C897F0B1
:10CC8000FFFFE780402EAA85280097F0FFFFE7808E
:10CC9000A05605611753FFFF6700234582809797D1
:10CCA000FF1F9387E7039C43D847A1678D07631154
:10CCB000F7041753FFFFE702034101113285328465
:10CCC00097F0FFFFE780202A13066100AA844C003A
:10CCD000228597300000E78000232800A68597F082
:10CCE000FFFFE780605105611753FFFF6700E33FD7
:10CCF00082809797FF1F9387E7FE9C4381CFDC4399
:10CD000091CB1753FFFFE702033C82971753FFFFB6
:10CD10006700A33D82801753FFFFE702C33A797192
:10CD20003C08AE843ED2A165B7070A002A843ED4EF
:10CD300048103C08DD053ED636C432C63AC297D00C
:10CD4000FFFFE780E02F12474810BA8597F0FFFFFA
:10CD5000E780C01332464810B28597F0FFFFE780A6
:10CD6000E014A2464810B68597F0FFFFE780001256
:10CD7000501001478146A685228597D0FFFFE780A6
:10CD8000805145611753FFFF670023361753FFFF9C
:10CD9000E702633301117C000329C501AE843ECA5A
:10CDA000A165B70707002A843ECC48087C00C5056A
:10CDB0003ECE97D0FFFFE780A0288345D9004808E2
:10CDC00097F0FFFFE780800C500801478146A68559
:10CDD000228597D0FFFFE780004C05611753FFFFC6
:10CDE0006700A3301753FFFFE702E32D83C79500C9
:10CDF00093F7F707A384F50097000000E78040F958
:10CE00001753FFFF6700632E1753FFFFE702A32BA3
:10CE100079713C08AE843ED2A165B70709002A8427
:10CE20003ED448103C08938545043ED632C636C4ED
:10CE300097D0FFFFE780C020A2464810B68597F044
:10CE4000FFFFE780A00432464810B28597F0FFFF4D
:10CE5000E780C005501001478146A685228597D0FE
:10CE6000FFFFE780404345611753FFFF6700E3275B
:10CE70001753FFFFE702232583C7950041112A843A
:10CE800093F7F707A384F50032852EC697F0FFFFCE
:10CE9000E780800F85672AC46370F50297700000F1
:10CEA000E78060E82246B24509ED114781462285B8
:10CEB00097000000E78060E641011753FFFF67001D
:10CEC000C32201478346F501DDB71753FFFFE70291
:10CED000E31D01113C003ECAB7070A003ECC3C00EE
:10CEE0003ECE83C79500AA89328593F7F707A384BE
:10CEF000F5002E8497F0FFFFE78000098567637DCA
:10CF0000F504A165AA8493858504480897D0FFFF9E
:10CF1000E7800013268597700000E780C0E02A892B
:10CF200029E19145480897F0FFFFE78020F6A685A4
:10CF3000480897F0FFFFE78060F7CA85480897F038
:10CF4000FFFFE780A0F4014781465008A2854E8587
:10CF500097D0FFFFE780203405611753FFFF67007C
:10CF600023188145480897F0FFFFE78020F2034926
:10CF7000090275BF1753FFFFE702431379711C10B5
:10CF80003ECAB7070F003ECC404D1C10AA84AE89A4
:10CF90004808994532C636893ECE97D0FFFFE780D4
:10CFA000200A32464808B28597F0FFFFE78000EE7E
:10CFB000630C0902A545480897F0FFFFE780C0E62B
:10CFC0002546CA8597200100E78060A350080147E5
:10CFD0008146CE85268597D0FFFFE780C02B45612F
:10CFE0001753FFFF6700C30F8355C402480897F02B
:10CFF000FFFFE780A0EB0355E402814505C58547A7
:10D0000085456301F502C167FD179305F00F630BBA
:10D01000F5007D1597700000E780608D9305150081
:10D0200093F5F50F480897F0FFFFE78020E683456A
:10D030000403480897F0FFFFE78040E583451403A9
:10D04000480897F0FFFFE78060E483552403480811
:10D0500097F0FFFFE78080E583554403480897F089
:10D06000FFFFE780A0E49DB71753FFFFE702A3058A
:10D0700083C795008146014693F7F707A384F5001F
:10D0800097000000E78040EF1753FFFF6700E305BC
:10D090001753FFFFE702230379713E841C103ECA39
:10D0A0002E89B7070F00A1653ECCFD051C10AA8490
:10D0B000480842C03AC23ECE36C432C697D0FFFFBF
:10D0C000E78000F832464808B28597F0FFFFE78016
:10D0D000E0DBA2464808B68597F0FFFFE78000DD59
:10D0E00012474808BA8597F0FFFFE78020DC024826
:10D0F000630C08029145480897F0FFFFE780C0D213
:10D100001146A28597200100E780608F50080147F3
:10D110008146CA85268597D0FFFFE780C017456105
:10D120001753FFFF670063FC8945480897F0FFFF2E
:10D13000E78080CF834704002300F5008347140075
:10D14000A300F500E1B71753FFFFE70223F683C7FB
:10D15000950001112A8A93F7F707A384F500328519
:10D16000AE8432C697F0FFFFE78000E232462A899C
:10D17000328597F0FFFFE78000DF85676373F90270
:10D18000AA894A8597700000E780E0B92A8419EDE2
:10D19000114781464A86A685528597000000E780A0
:10D1A000C0B705611753FFFF670083F39387E9FF5B
:10D1B00093F7F70F0547E366F7FE8347F50195EB15
:10D1C0008947E380F9FE8346F401528501474A8688
:10D1D000A68597000000E78040B4A167D9074808FA
:10D1E0003ECC230A010002CE97000000E780A0B0E9
:10D1F0004DBF639EE7008947639EF90093071020A7
:10D20000231FF50097700000E78000B76DBF094746
:10D21000E39BE7FA8D47E398F9FA228597700000BF
:10D22000E780C0DE9797FF1F9387C7CA9C4399E7A3
:10D230009797FF1F9387C7B39C4399C703D50400F3
:10D2400097800000E780E0CD231F040022855DBFAA
:10D250001753FFFFE70223E701113C003ECAB7075F
:10D260000B003ECC3C003ECE83C795002A89328518
:10D2700093F7F707A384F500AE8497F0FFFFE780EC
:10D28000A0D093170501C187635AF006A1652A84CF
:10D290009385E502480897D0FFFFE78060DAA28512
:10D2A000480897F0FFFFE78060C09797FF1F9387BC
:10D2B00027AC9C43A9EB01449375F40F480897F001
:10D2C000FFFFE780A0BC9355844093F5F50F480815
:10D2D00097F0FFFFE78080BB9355044193F5F50F6E
:10D2E000480897F0FFFFE78060BA01478146500881
:10D2F000A6854A8597D0FFFFE780E0F905611753BF
:10D30000FFFF670083DE416585460546A2857D15E2
:10D3100097500000E780A0BC59DD5105970001003F
:10D32000E780C08E130440063344850271B717535B
:10D33000FFFFE70243D90111B70706003EC683C7C6
:10D34000950021642A8993F7F707A384F500AE843A
:10D3500028009305A4040AC40AC897D0FFFFE780F9
:10D3600020CE300001478146A6854A8597D0FFFF31
:10D37000E78060F297E0FFFFE780801513049404D4
:10D38000480822CC230A010002CE97000000E78063
:10D39000809605611753FFFF670023D51753FFFFE2
:10D3A000E702C3D0C1642A8901449799FF1F93897A
:10D3B000E9B3130A8002FD1497E0FFFFE78080C104
:10D3C0006347A40001451753FFFF670063D1B3070C
:10D3D000440303A7C90ABA9703D707006306970057
:10D3E00083D72700638427010504F9B70545E1BF0A
:10D3F0001753FFFFE70283CB2A8A2E8999C123A006
:10D40000050081498144979AFF1F938AEA8D614BF9
:10D4100097E0FFFFE78040C263C7A4004E85175323
:10D42000FFFF6700E3CB3384640383A70A003E94C5
:10D430008357040099E763040900232089008504C9
:10D44000C1BF4146D2851305440097100100E78013
:10D45000A05875F5A289E5B71753FFFFE70203C58A
:10D4600039717C083ED4B7070A003ED67C083ED806
:10D4700083C795002A8A328593F7F707A384F500BE
:10D480002E8932C697F0FFFFE78000B0856763738F
:10D49000F5083246AA84328597F0FFFFE780A0ACFA
:10D4A0008547AA8963E8A706A165938585042810A6
:10D4B00097D0FFFFE780C0B8268597700000E7800F
:10D4C00080862A8429ED9145281097F0FFFFE78098
:10D4D000E09BA685281097F0FFFFE780209DCE8572
:10D4E000281097F0FFFFE780609A014781463010CF
:10D4F000CA85528597D0FFFFE780E0D9A16793875F
:10D50000770448183EDC230A010202DE97F0FFFF91
:10D51000E780607E21611753FFFF670063BC814590
:10D52000281097F0FFFFE7806096A685281097F0F7
:10D53000FFFFE780A0979797FF1F9387E7D19C4352
:10D5400081CB22856389090097D00000E780802382
:10D550008345040271B797D00000E7800022CDBF59
:10D560001753FFFFE70283B483C795004111AA89CF
:10D5700093F7F707A384F5003285AE84328A97F0DB
:10D58000FFFFE78060A08567637FF5022A899760C7
:10D590000000E78040792A84914631C58347F50130
:10D5A00005476387E70291C70D476366F704AD46F9
:10D5B0001DA89305050303250A00414697100100A5
:10D5C000E78080410DE941011753FFFF670043B138
:10D5D0009305950803250A00414697100100E7804E
:10D5E000A03F814669F54A86A6854E8597000000D2
:10D5F000E780C081C9BF83250A001305940897708E
:10D600000000E780E02819C1C146F1BF9797FF1FCE
:10D610009387478C9C4399E79787FF1F93874775AC
:10D620009C4399C7228597800000E780608969FD47
:10D630008547A30FF400228597B00000E780A08300
:10D64000228597600000E78020734E8581464A86D8
:10D65000A68597F0FFFFE780607BA167938757045B
:10D6600048003EC42302010002C697F0FFFFE78096
:10D67000806891BF1753FFFFE70263A283C795003D
:10D680004111AA8993F7F707A384F50032852E8903
:10D69000B28A97F0FFFFE780208F85676374F50EED
:10D6A000AA8497600000E78000682A840DED416B32
:10D6B000014A979BFF1F938B6B83130C400E7D1BBE
:10D6C00019A833048A0383A70B0B3E948357C40124
:10D6D00063836705050A97E0FFFFE780A08EE342BA
:10D6E000AAFE95460DA08357C50163969702930540
:10D6F000050303A50A00414697100100E780C02DED
:10D70000994611E181462686CA854E8597F0FFFF2E
:10D71000E780C06F85A883A50A00130504039770EE
:10D720000000E780E016C14679FD2285231E9400A3
:10D7300097A00000E7802074228597600000E780B2
:10D74000A0639797FF1F938727B19C43A9C323002A
:10D750000402228597D00000E78080EF4E85814645
:10D760002686CA8597F0FFFFE780406AA167938706
:10D77000070448003EC42302010002C697F0FFFFE1
:10D78000E780605741011753FFFF6700C394894743
:10D790002300F402E1B7397106DE22DC4AD88000AA
:10D7A00052D456D25AD026DA4ED65ECE2E8A32893E
:10D7B0002A8B97D0FFFFE780E07D06057105419930
:10D7C0008A8A3301A140232224FC231404FC97D02D
:10D7D000FFFFE780207C83479A000605350593F715
:10D7E000F7072315A4FCA304FA004A85232624FC8A
:10D7F00097E0FFFFE780407993170501C1876340F9
:10D80000F0025681130104FCF2506254D254425982
:10D81000B259225A925A025BF24B21618280AA8449
:10D820004A8597E0FFFFE7802076AA894A8597E03E
:10D83000FFFFE7806075A1659385C5022A891305FE
:10D8400044FC97C0FFFFE780A07F268597C0FFFFBD
:10D85000E780E073854511C94A86CE8597C0FFFFF2
:10D86000E780606DAA8B21E98945130544FC97E0A8
:10D87000FFFFE780A061A685130544FC97E0FFFF4A
:10D88000E780C062CE85130544FC97E0FFFFE78088
:10D89000E061CA85130544FC97E0FFFFE780006163
:10D8A00001478146130644FCD2855A8597D0FFFF75
:10D8B000E780609EB9B78145130544FC97E0FFFF00
:10D8C000E780C05CA685130544FC97E0FFFFE78076
:10D8D000E05DCE85130544FC97E0FFFFE780005D27
:10D8E000CA85130544FC97E0FFFFE780205C814474
:10D8F00097D0FFFFE780006AE3D4A4FA83A70B0167
:10D9000013971400BA9783D5070099C5130544FCF3
:10D9100097E0FFFFE78080598504D9BF797106D66B
:10D9200022D44AD000184ECE52CC56CA26D25AC85B
:10D93000AE893289AA8A97D0FFFFE780A0650605E5
:10D94000690541990A8A3301A140232A24FC231C3A
:10D9500004FC97D0FFFFE780E06383C799000605CA
:10D960002D0593F7F707231DA4FCA384F9004A852E
:10D97000232E24FC97E0FFFFE78000619317050149
:10D98000C187634FF0005281130104FDB25022544D
:10D9900092540259F249624AD24A424B456182800E
:10D9A000AA844A8597E0FFFFE780005EA165938522
:10D9B000A5022A89130544FD97C0FFFFE780406850
:10D9C000268597C0FFFFE780805C854509C9CA8529
:10D9D00097C0FFFFE78020592A8B29E1894513056D
:10D9E00044FD97E0FFFFE780604AA685130544FDEC
:10D9F00097E0FFFFE780804BCA85130544FD97E061
:10DA0000FFFFE780A04A01478146130644FDCE850B
:10DA1000568597D0FFFFE7800088B5B7814513058D
:10DA200044FD97E0FFFFE7806046A685130544FDAF
:10DA300097E0FFFFE7808047CA85130544FD97E024
:10DA4000FFFFE780A046814497D0FFFFE780805426
:10DA5000E3DBA4FA83270B0113971400BA9783D54D
:10DA6000070099C5130544FD97E0FFFFE7800044D8
:10DA70008504D9BF1743FFFFE702E36483474500EE
:10DA8000404DD5EFFD575DC483469400094763635D
:10DA9000D70A0346B400854663EEC6088306E40051
:10DAA00063CA06085C45F9562390D7009787FF1F85
:10DAB00083C7C72399E3A304E4009787FF1F9387D5
:10DAC000272B9C4381E78947A306F4009787FF1F14
:10DAD000938787789C4381E789472306F40097055D
:10DAE000000093854506AA841305040197F0000001
:10DAF000E780600FFD57231AF40281471CDC0148C0
:10DB00009787FF1F23A0871E9787FF1F9387C71D37
:10DB1000232E040304C0804397D0FFFFE780C05149
:10DB200061463306C502814522859740FFFFE780A5
:10DB3000805C81473E851743FFFF6700035BFD570D
:10DB4000D5BF1743FFFFE70203582A840355450258
:10DB500097600000E780201D19E5231E040017438D
:10DB6000FFFF670083588357E401F5DB930504FF4B
:10DB7000174501001305852C97E00000E78020146D
:10DB8000F9BF1743FFFFE70203542E89A165411136
:10DB90009385E5032A8436C432C6BE843AC297C050
:10DBA000FFFFE780E04912472285BA8597E0FFFF33
:10DBB000E780C02D32462285B28597E0FFFFE780DF
:10DBC000E02EA2462285B68597E0FFFFE780002E73
:10DBD000630309029145228597E0FFFFE780C02497
:10DBE0001146A68597100100E78060E141011743C7
:10DBF000FFFF6700834F8945228597E0FFFFE7809D
:10DC0000A02283C704002300F50083C71400A300EB
:10DC1000F500E9BF1743FFFFE702E34A83C795001A
:10DC2000444D054793F7F707A384F5001C424111C3
:10DC300083C707006367F7062E842A89B1C003C72C
:10DC4000D400630FF7021787FF1F130767121843EB
:10DC500005C3A386F40097A00000E780804983C72E
:10DC6000D40099E741657D1597400000E780802F3B
:10DC700083D72403918B89C797E00000E7800013C6
:10DC80004A85A28597F0FFFFE7808010A167C10752
:10DC900048003EC42302010002C697F0FFFFE78060
:10DCA000800541011743FFFF670023441743FFFF2F
:10DCB000E702634103D745008D47AA8441112E84B2
:10DCC00032892E8563E3E70297E0FFFFE780C02BF0
:10DCD000AA8523000900268597C0FFFFE780A028BA
:10DCE00041011743FFFF6700434097E0FFFFE780D4
:10DCF000A0292AC6228597E0FFFFE780E028B245E9
:10DD000085472A862300F900268597C0FFFFE78014
:10DD10008022F9B7397106DE22DC26DA80004ED681
:10DD200052D456D24AD85AD05ECEAE89B284AA8A8C
:10DD300097D0FFFFE78000250605130525024199CE
:10DD40000A8A3301A140232224FC231404FC97D027
:10DD5000FFFFE780202383C7990006054D0593F751
:10DD6000F7072315A4FCA384F9002685232624FCA9
:10DD700097E0FFFFE780402193170501C1876340CB
:10DD8000F0025281130104FCF2506254D254425901
:10DD9000B259225A925A025BF24B21618280AA8BBD
:10DDA00003AB040097C0FFFFE780601E51E583D7F7
:10DDB000440001498544F11793B71700A301F4FC0F
:10DDC000834734FCA165C9C79385E504130544FC6A
:10DDD00097C0FFFFE780C026A685130544FC97E0A7
:10DDE000FFFFE780A00ADE85130544FC97E0FFFFF4
:10DDF000E780C00B834734FC114691E30946DA857E
:10DE0000130544FC97E0FFFFE78060058144630A47
:10DE10000900416B7D1B97D0FFFFE780A01663CC04
:10DE2000A40201478146130644FCCE85568597C05F
:10DE3000FFFFE7804046B1B7A685130634FC970084
:10DE40000000E780E0E6933415002A8986048DBF40
:10DE50009385C504A5BF8327C90013971400BA97FB
:10DE600083D5070063886501130544FC97E0FFFF35
:10DE7000E780C003850445B71743FFFFE70223226D
:10DE800079711C103EC4B7070F003EC61C103EC877
:10DE900083C79500AA8A328593F7F707A384F50014
:10DEA000AE89328497E0FFFFE780000E93170501EB
:10DEB000C187635AF0062A8A228597E0FFFFE78030
:10DEC000A00C2A895285032B040097C0FFFFE7802E
:10DED000000C39ED8357440081440544F11793B792
:10DEE0001700A303F10083457100DA872287CA86F1
:10DEF0005286280097000000E780E0C8014781466D
:10DF00003000CE85568597C0FFFFE780C038A167F7
:10DF10009387D70348083ECC230A810026CE97F08A
:10DF2000FFFFE78040DD45611743FFFF6700A31A4D
:10DF3000A2851306710097000000E78060D7AA84CD
:10DF4000094455D13544E30055FB4A8597F0FFFF5E
:10DF5000E78000450D4441D9014497D0FFFFE78099
:10DF60006002634DA400C16B0144FD1B97D0FFFF0D
:10DF7000E7804001634EA4001544B5B7DC44131795
:10DF80001400BA9783D70700638327030504F1B70A
:10DF9000D84493171400BA9703D70700631B77017F
:10DFA00023902701268597A00000E780C0DA01446E
:10DFB0001DBF050465BF1743FFFFE702230F83C79B
:10DFC000950041112A8A93F7F707A384F50032855B
:10DFD0002E89328497E0FFFFE78000FB931705014D
:10DFE000C1876353F006AA89228597E0FFFFE78087
:10DFF000A0F92311A1004E85832A040097C0FFFFDA
:10E00000E780E0F839E58357440085440144F1177F
:10E0100093B71700A300F100034811000357210034
:10E02000D6875285CE862686CA8597F0FFFFE78081
:10E030006006A167F10748003EC42302910022C692
:10E0400097F0FFFFE78020CB41011743FFFF6700F8
:10E050002309A2851306110097000000E78040C540
:10E060002A84894455D98357210011678544BA977A
:10E07000C2071167C1831307F7EFE36FF7F89787BC
:10E08000FF1F938727E59C4381CB8545130521001E
:10E0900097500000E78060748355210022858144F9
:10E0A00097C0FFFFE78040E525D9231005002285B2
:10E0B00097A00000E78080CC85B71743FFFFE702F9
:10E0C00003FE83C7950041112A8B93F7F707A384BA
:10E0D000F50032852E8A328497E0FFFFE780C0EAA0
:10E0E00093170501C1876351F006AA8A228597E03C
:10E0F000FFFFE78060E92A895685832B040097C0DB
:10E10000FFFFE780C0E831E58357440081440544C0
:10E11000F11793B71700A301F10003483100DE8720
:10E120005A854A87D6862286D28597F0FFFFE780F8
:10E1300060F6A167ED0748003EC42302810026C6B1
:10E1400097F0FFFFE78020BB41011743FFFF670007
:10E1500083F8A2851306310097000000E78040B5E0
:10E16000AA8409445DD99167CA97C2071167C18320
:10E170001307F7EF0544E362F7FACA8597C0FFFF7C
:10E18000E78080D7014451F9814997D0FFFFE780AC
:10E1900060E063DBA900984893971900BA9703D70A
:10E1A000070005EF2390270197D0FFFFE78080DE6F
:10E1B0001544E384A9F6268597A00000E78000BCFB
:10E1C0009787FF1F938707D19C430144B9D74A859E
:10E1D00097500000E780005889B785097DB717433D
:10E1E000FFFFE702A3EC79713E847C083EC82E8ACB
:10E1F000B7071400A1653ECAE5057C08AA8908088E
:10E2000036C4428932C6BA8AC6843ECC97C0FFFF64
:10E21000E78000E3CA85080897E0FFFFE78000C7B2
:10E2200032460808B28597E0FFFFE78020C8A24683
:10E23000630A09049D45080897E0FFFFE780C0BE18
:10E240001D4681459740FFFFE780E0EA63890A08A1
:10E250009145080897E0FFFFE78000BD1146A685BD
:10E2600097000100E780A079100801478146D28518
:10E270004E8597C0FFFFE780000245611743FFFF0F
:10E28000670003E6B685080897E0FFFFE78000C255
:10E290001C400808D8439355C7018589120751834C
:10E2A000B205D98D97E0FFFFE78040C01C40080809
:10E2B00083C5870097E0FFFFE78040BD1C4008084A
:10E2C00083C5A70097E0FFFFE78040BC1C4008081B
:10E2D00083C5970097E0FFFFE78040BB85BF894576
:10E2E000080897E0FFFFE78020B483C704002300FD
:10E2F000F50083C71400A300F500BDB71743FFFF67
:10E30000E702C3DA83C795004111AA8993F7F7079B
:10E31000A384F5003285AE84328497E0FFFFE78066
:10E32000A0C693170501C187635DF0042A89032AFB
:10E33000040097C0FFFFE78080C519E983574400B8
:10E340000548F11793B71700A307F100814631A8DC
:10E350001306F100A28597000000E78060951DC5B7
:10E360001C459DC783D6470001480347F10093072A
:10E370008500D2884A86A6854E8597000000E780F2
:10E3800040E641011743FFFF670083D509487DBF81
:10E390001D486DBF1743FFFFE70243D165715C085D
:10E3A0003EC4B7077B013EC65C083EC883C79500E4
:10E3B0002A8A328593F7F707A384F500AE8997E0A0
:10E3C000FFFFE78040BA8357E100E1C78945280095
:10E3D00097C0FFFFE780C0C68145280097E0FFFF98
:10E3E000E780C0AA97C0FFFFE780A0CC9787FF1FF8
:10E3F000938787E69C431784FF1F0344248FAA84D6
:10E400003334800099C3136424009787FF1F9387D8
:10E4100027969C4399C3136444009787FF1F9387F3
:10E4200067AB9C4399C31364840083D50400280020
:10E43000014997E0FFFFE78060A783D5240028000B
:10E4400097E0FFFFE78080A683D54400280097E08F
:10E45000FFFFE780A0A597D0FFFFE780A0AE931550
:10E460000501C181280097E0FFFFE78020A4A28575
:10E47000280097E0FFFFE78060A39C446360F902F7
:10E48000014781463000CE85528597C0FFFFE78067
:10E4900080E059611743FFFF670083C4DC44131415
:10E4A000490028003E9497E0FFFFE780609683478D
:10E4B00044000347540089070607BA978607E36AB2
:10E4C000F5FC835524002800814A97E0FFFFE78090
:10E4D000E09D83454400280097E0FFFFE780009B14
:10E4E00083455400280097E0FFFFE780209A834788
:10E4F000440063C9FA00814A8347540063C1FA02A9
:10E500000509A5BF1C4413975A002800BA9783D564
:10E510000700850A97E0FFFFE7804099C9BF032BFA
:10E52000C40093975A0028003E9B83552B00850A10
:10E5300097E0FFFFE780809783550B00280097E066
:10E54000FFFFE780A0964DBF1743FFFFE702A3B789
:10E550005C4993E717005CC997A00000E78060B5AD
:10E560001743FFFF670063B81743FFFFE702A3B538
:10E570002E84814597F0FFFFE780C0E705C58357EC
:10E580000500FD172310F50009C48357250023104B
:10E59000F40097000000E78060FB01451743FFFF90
:10E5A0006700A3B431457DD823100400C5BF1743CD
:10E5B000FFFFE702A3AF83C7950041112A8A93F7B3
:10E5C000F707A384F50032852E89328497E0FFFF98
:10E5D000E780809B93170501C1876356F006AA89DF
:10E5E000C145228597E0FFFFE780A0802A8B4E85FA
:10E5F000832A040097C0FFFFE780609931E98357C1
:10E600004400231101000544F11793B71700A3003C
:10E61000F10081440348110003572100D687528539
:10E62000CE862286CA8597F0FFFFE780A0A6A16765
:10E630009387170248003EC42302810026C697E054
:10E64000FFFFE780406B41011743FFFF670043A9CD
:10E6500013061100A28597F0FFFFE7806065AA848A
:10E6600009E523110100094475B7930521005A8576
:10E6700097000000E78080EF835721002A84D9DBD0
:10E680009787FF1F938707859C4381CB854513059B
:10E69000210097500000E780401483552100268513
:10E6A000314497C0FFFFE78020852DD5231005005A
:10E6B000268597900000E780606C0144A1BF174356
:10E6C000FFFFE70243A041112E896C00AA8402C615
:10E6D00097F0FFFFE78000D20DC103570500050743
:10E6E0002310E50097000000E78040E681473E8563
:10E6F00041011743FFFF6700439F3247954765DBA2
:10E70000CA85268597300000E780800CC147E3402A
:10E7100005FE3244854741462310F4008357090023
:10E72000A685130544002311F40097000100E7803B
:10E73000002D228545BF1743FFFFE702239783C7BC
:10E7400095004111AA8A93F7F707A384F500328553
:10E75000AE89328497E0FFFFE780008393170501BD
:10E76000C1876356F0062A8AC145228597D0FFFFEC
:10E77000E7802068AA845285032B040097C0FFFF1E
:10E78000E780E08031E9835744002311010085448C
:10E79000F11793B71700A300F100014403481100DB
:10E7A00003572100DA875685D2862686CE8597F0D4
:10E7B000FFFFE780208EA1679387070248003EC4D1
:10E7C0002302910022C697E0FFFFE780C05241017B
:10E7D0001743FFFF6700C390A2851306110097F04F
:10E7E000FFFFE780E04C2A8409E5231101008944FA
:10E7F00075B726859305210097000000E78060EC3F
:10E80000AA8449FD83552100228597B0FFFFE78048
:10E81000A06E49F5014997C0FFFFE780A077635DCF
:10E82000A900184893171900BA9703D707000DEFEE
:10E83000035721002390E70097C0FFFFE780807512
:10E84000630625039777FF1F9387C7689C4399C783
:10E850000355210097500000E780C0EF2285979074
:10E860000000E780A0511DBF050975B795443DB76D
:10E8700005C19307F00F630FF500C547630CF50062
:10E880009307F5FF05453315F50042054181828068
:10E890000145828041657D158280B9E91743FFFFFC
:10E8A000E702638203450603328497000000E78095
:10E8B00060FC9305803EB305B502C205C18181CDE0
:10E8C0000357E402854763F8E7001305040197E066
:10E8D0000000E78060418357E40241677D1763854C
:10E8E000E700FD172317F4021733FFFF6700E37FEC
:10E8F00082801733FFFFE702837A004283C79500C7
:10E90000444D0349140093F7F707A384F5008347A8
:10E910000400220911673369F900A167B347F900C0
:10E9200041112A8BAE8A63ECE70E8347240013075C
:10E93000C00EB91793F7F70F6373F710034734004E
:10E94000C14763EEE70E834744001307E00793C710
:10E9500007086371F70C8349840083477400A20998
:10E96000B3E9F900856763F7F90A034A640083474E
:10E9700054004E85220A336AFA0097500000E7805F
:10E98000803A61C123962403834B3400137AFA0042
:10E99000239A34032388740323994403938904013D
:10E9A000631C090023A60402239804024E8597E005
:10E9B0000000E780A0353DA0034924004A85970068
:10E9C0000000E78020EB2397A402834744004E8594
:10E9D000A388F402E38D0BFCE30B09FC97E0000035
:10E9E000E780602E97900000E780407281460146E4
:10E9F000D6855A8597E0FFFFE7800058A167938787
:10EA000097033EC423020100480002C697E0FFFFBF
:10EA1000E780602E41011733FFFF6700C36B854419
:10EA2000A2862686D6855A8597E0FFFFE780C054E8
:10EA3000A167938797033EC423029100F1B7BD44B9
:10EA4000C5B79144F1BF1733FFFFE70223660111F9
:10EA50001C08404D3EC2B7070F003EC41C083EC60E
:10EA60002A89AE8997C0FFFFE780A0DA585C1C5C5A
:10EA70006346B70E6394E50063E2A70E3385A740B3
:10EA8000B3B7A700B305B7401306803E81469D8DFE
:10EA900097000100E780C0B693140501C180A1650D
:10EAA0009385C503480097B0FFFFE7806059814513
:10EAB000480097D0FFFFE780603D8355040448007D
:10EAC00097D0FFFFE780803E83552404480097D00D
:10EAD000FFFFE780A03D814589CCC167FD17930505
:10EAE000F00F6388F400268597500000E78020E04F
:10EAF000AA85480097D0FFFFE780403903554404BA
:10EB0000814501CDC167FD179305F00F6307F5003F
:10EB100097500000E780A0DDAA85480097D0FFFF4E
:10EB2000E780C03683456404480097D0FFFFE78044
:10EB3000E03583457404480097D0FFFFE780003537
:10EB4000500001478146CE854A8597B0FFFFE78098
:10EB5000807405611733FFFF67008358814481B7D4
:10EB60001733FFFFE702235683C7950093F7F70794
:10EB7000A384F50097000000E78020ED1733FFFF26
:10EB80006700A3561733FFFFE702435283C7950080
:10EB90004111404D93F7F707A384F5002A8A328587
:10EBA000B284AE8997D0FFFFE780003E2A8B26858E
:10EBB00097D0FFFFE780403D2A89268597D0FFFF49
:10EBC000E780603A93170B0163CA0702E177CA979F
:10EBD000C207C183116763E3E70293070910C20705
:10EBE000C1831307B00F637BF70093170901C18737
:10EBF000AA8A634AF000C54763FE570141011733F3
:10EC0000FFFF6700E34D97B0FFFFE780C028E317E1
:10EC100025FFD5B763080B026306090281446389A7
:10EC20000A02B7077F0023106405231124057CC066
:10EC3000568597000000E780E0C39304803EB3044C
:10EC4000950239A0B7077F00232004047CC08144CB
:10EC50000355240497E00000E780E0A2A1C497C018
:10EC6000FFFFE78000BB269593D7F441333795002B
:10EC7000AE97BA9708DC5CDCCE8552859700000021
:10EC8000E780A0DC99E023220404A1679387B703FF
:10EC900048003EC42302010002C697E0FFFFE78060
:10ECA0008005A9BF814701481CDC232E0403E9B776
:10ECB0001733FFFFE702234197C0FFFFE780C0370C
:10ECC000E1473305F502914597500000E78040C4C5
:10ECD000E55711C59777FF1F23A8A70081473E85F9
:10ECE0001733FFFF670063401733FFFFE702A33DC1
:10ECF0009777FF1F938707FF80433DC08357040426
:10ED00006390A70683572404639CB7043689B284B2
:10ED100097C0FFFFE780E0AF5C5C63C3B704639517
:10ED2000B7001C5C63EEA7028347640463F3F4003E
:10ED3000A6872303F4048347740463F39700A6872C
:10ED4000A303F4048357440441677D176385E700F8
:10ED500085072312F4043C4481C7CA85268582971F
:10ED60001733FFFF670063389777FF1F938787F795
:10ED70009C43014599C303C5870082801733FFFF79
:10ED8000E70263340111B70707003EC683C7950049
:10ED9000584D0AC493F7F7070AC8A384F5002A89D7
:10EDA000AE8411CB1C4283C707002304F700979061
:10EDB0000000E7800034216493055402280097B0D6
:10EDC000FFFFE780E02797000000E78020FAAA8590
:10EDD000280097D0FFFFE780600B30000147814695
:10EDE000A6854A8597B0FFFFE780E04A13044402F6
:10EDF000480822CC230A010002CE97E0FFFFE780FB
:10EE000080EF05611733FFFF6700232E1733FFFFE5
:10EE1000E702632B01117C003ECAB70707003ECC16
:10EE20007C003ECE83C795002E84AA8493F7F70713
:10EE3000A384F500A16593855502480897B0FFFFAC
:10EE4000E780002097000000E78040F2AA8548088C
:10EE500097D0FFFFE7808003500801478146A285D5
:10EE6000268597B0FFFFE780004305611733FFFF5A
:10EE70006700A3279777FF1F9387C7E69C43094541
:10EE800099C303C5970082809777FF1F938787E513
:10EE90009C43094599C303C5D70082809777FF1F1C
:10EEA000938747E49C43014599C303C5A70082802B
:10EEB0001733FFFFE702831F0111B70708003EC6A3
:10EEC00083C79500404D0AC493F7F7070AC8A38487
:10EED000F5002A89AE8429C41442854703C7060079
:10EEE00063E0E70A83479400094681496380C702CB
:10EEF000B307F740A304E400B339F00083C716005A
:10EF00002305F40097900000E780A01E0357240318
:10EF1000058B19C76386090097D00000E78000E9D8
:10EF2000216493058402280097B0FFFFE780401119
:10EF300097000000E78040F4AA85280097D0FFFFE3
:10EF4000E780C0F497000000E78080F5AA852800DC
:10EF500097D0FFFFE78080F3014781463000A68508
:10EF60004A8597B0FFFFE780003313047402480816
:10EF700022CC230A010002CE97E0FFFFE780A0D752
:10EF800005611733FFFF6700A3151733FFFFE70283
:10EF9000831301117C003ECAB70708003ECC7C00F9
:10EFA0003ECE83C795002E84AA8493F7F707A384E7
:10EFB000F500A16593858502480897B0FFFFE780BB
:10EFC000200897000000E78020EBAA85480897D02A
:10EFD000FFFFE780A0EB97000000E78060ECAA85C8
:10EFE000480897D0FFFFE78060EA50080147814654
:10EFF000A285268597B0FFFFE780E02905611733DA
:10F00000FFFF6700830E9777FF1F9387A7CD9C4371
:10F01000014599C303C5B70082801733FFFFE7029C
:10F02000830A0111B70707003EC683C79500404D0C
:10F030000AC493F7F7070AC8A384F5002A89AE84A7
:10F0400005C81C42054783C707006368F7060347E6
:10F05000B400630FF700A305F40097900000E78069
:10F0600040098347B400B9CF97D0FFFFE78000BFC6
:10F0700021649305B400280097B0FFFFE78040FCAF
:10F0800097000000E78060F8AA85280097D0FFFF6E
:10F09000E780C0DF014781463000A6854A8597B0EA
:10F0A000FFFFE780401F2904480822CC230A010003
:10F0B00002CE97E0FFFFE78000C405611733FFFF32
:10F0C0006700A30297D0FFFFE780E0BF55B7173373
:10F0D000FFFFE70243FF01117C003ECAB7070700AC
:10F0E0003ECC7C003ECE83C795002E84AA8493F745
:10F0F000F707A384F500A165AD05480897B0FFFFA9
:10F10000E78000F497000000E78020F0AA85480817
:10F1100097D0FFFFE78080D7500801478146A2853E
:10F12000268597B0FFFFE780001705611733FFFFC3
:10F130006700A3FB9777FF1F9387C7BA9C430945D6
:10F1400099C303C5C70082801733FFFFE702A3F707
:10F1500001117C00AE843ECAA165B70707002A846E
:10F160003ECCD1057C0048083ECE97B0FFFFE7803B
:10F1700020ED97000000E78020FCAA85480897D082
:10F18000FFFFE780A0D0500801478146A685228571
:10F1900097B0FFFFE780201005611733FFFF67007E
:10F1A000C3F41733FFFFE70203F283C7950093F719
:10F1B000F707A384F50097000000E78020F91733D4
:10F1C000FFFF670083F21733FFFFE70223EE83C7D9
:10F1D00095000329C501411193F7F707A384F500B2
:10F1E0001C4283C90700854763E637079777FF1FEF
:10F1F000938787069C432E84AA8485CF97000000BE
:10F20000E78080F389476306F502630409028347B8
:10F21000C900638037032306390197900000E78017
:10F2200040ED83572903898B89C797D00000E78079
:10F23000E0B72685A28597000000E78020F1A1674E
:10F24000CD0748003EC42302010002C697E0FFFF3D
:10F25000E78060AA41011733FFFF670063E89777F3
:10F26000FF1F938727A89C431D4599C303C5E7004B
:10F2700082801733FFFFE70203E50111B70707009C
:10F280003EC683C79500584D0AC493F7F7070AC8CE
:10F29000A384F5002A89AE8415C71C4283C70700E2
:10F2A00093968701E18663C4060685466381D70687
:10F2B0008346E7006388F6002307F7009790000075
:10F2C000E78020E321649305E400280097B0FFFF66
:10F2D000E78000D797000000E780A0F8AA85280003
:10F2E00097D0FFFFE78080BA014781463000A685AE
:10F2F0004A8597B0FFFFE78000FA3504480822CC22
:10F30000230A010002CE97E0FFFFE780C09E05615F
:10F310001733FFFF670063DD1733FFFFE702A3DA50
:10F3200001117C003ECAB70707003ECC7C003ECEF0
:10F3300083C795002E84AA8493F7F707A384F5006A
:10F34000A165B905480897B0FFFFE78060CF970037
:10F350000000E78000F1AA85480897D0FFFFE7800A
:10F36000E0B2500801478146A285268597B0FFFF8D
:10F37000E78060F205611733FFFF670003D717339B
:10F38000FFFFE702A3D2AA8401441779FF1F1309E4
:10F39000A995E14997C0FFFFE78000CA6344A40034
:10F3A000014519A833053403832709003E95835787
:10F3B00025006397970011051733FFFF670043D2BD
:10F3C0000504C9BF032E8500630A0E121773FF1FC1
:10F3D000130343B003230300631503002943639021
:10F3E000061203234E01631503001D4363990710A2
:10F3F0001733FFFFE702A3CAC689428A3E89BA8A49
:10F40000B684328BAE8B2A84B5E103554E0019E5E4
:10F4100001431A851733FFFF6700E3CBA167A98F6C
:10F42000116763FBE70097000000E78080F58145E6
:10F4300097F0FFFFE78080130844B70700E05841CA
:10F44000F98F18455CC1B707001FF98F1CC55C49CF
:10F4500091C7610597E00000E780408BE38A09FAD5
:10F46000228597900000E78060C65DB7328597C01F
:10F470000000E78040430D4349DD1C44116703D57C
:10F480004700A167A98F63FBE70097000000E780B2
:10F4900040EF814597F0FFFFE780400D0323840094
:10F4A00093164B01D1828347B300035663008588CE
:10F4B000FD8BA305F300FD777D8E558EFD76FD1641
:10F4C000B204F18E83274301C58E231273012313E7
:10F4D000D3002304530123052301A3044301BDDF0B
:10F4E000228597B0FFFFE780E0CDAA850844B5D11B
:10F4F000610597D00000E780207F8DB71D431A85F6
:10F5000082801733FFFFE70263BA0569AA84AE89D8
:10F51000328A0144FD5A7D1997C0FFFFE78080A61B
:10F520006347A40001451733FFFF670063BBD8445E
:10F5300093171400BA9703D70700631F370323906C
:10F54000570163070A00268597900000E780A08096
:10F550009C449DC383D76700B3F72701639E37019F
:10F56000D288014881470147814601468145268569
:10F5700097000000E78040E5050479BF1733FFFFDF
:10F58000E702C3B279711C103EC4B7070F003EC634
:10F590001C103EC883C79500AA8A328593F7F707E7
:10F5A000A384F5002E89328497D0FFFFE780C09DA9
:10F5B00093170501C187635AF006AA89228597D05F
:10F5C000FFFFE780609C2A8A4E85032B040097B0DA
:10F5D000FFFFE780C09B39ED835744008144054419
:10F5E000F11793B71700A303F10083457100DA8781
:10F5F0002287D2864E86280097E0FFFFE780A0583A
:10F60000014781463000CA85568597B0FFFFE780E5
:10F6100080C8A1679387F70348083ECC230A81007E
:10F6200026CE97D0FFFFE780006D45611733FFFFBF
:10F63000670003ABA2851306710097E0FFFFE78028
:10F640002067AA84094455D1528597E0FFFFE780DF
:10F6500020D50D4459D90546D2852685970000004E
:10F66000E78060EA2A8451B71733FFFFE702A3A5BA
:10F67000835507000346270041112A842E8532C690
:10F680002EC497E0FFFFE780A0D101C93246A24512
:10F69000228597000000E78000E741011733FFFF54
:10F6A0006700A3A41733FFFFE702639F83C795009A
:10F6B0004111AA8A93F7F707A384F5003285AE8932
:10F6C000328497D0FFFFE780208C93170501C18714
:10F6D0006357F00AC1452A8A228597C0FFFFE78059
:10F6E00040712A8D228597D0FFFFE780E0892A8923
:10F6F000228597D0FFFFE7800087930705F893F7EF
:10F70000F70F1307E007AA8B637BF706228597D0D4
:10F71000FFFFE78040852A8C228597D0FFFFE78096
:10F720008084AA8C5285032B040097B0FFFFE780EA
:10F73000008639E983574400231101008144F11701
:10F7400093B71700A300F100054403471100835647
:10F750002100938784005685DA8822885286CE85D8
:10F7600097F0FFFFE780E0A7A167E90748003EC4E4
:10F770002302810026C697D0FFFFE780C0574101D2
:10F780001733FFFF6700239513061100A28597E04A
:10F79000FFFFE780E051AA8409E523110100094435
:10F7A0006DB7930521006A8597F0FFFFE78060F150
:10F7B0002A8441FD835521009356C900131649013F
:10F7C00085486688E2875E87858A5182268597000C
:10F7D0000000E78060BF2A848DBF1733FFFFE70278
:10F7E000038C83C7950041112A8B93F7F707A384F5
:10F7F000F5003285AE89328497C0FFFFE780C0787C
:10F8000093170501C1876352F00A2A8A228597C09F
:10F81000FFFFE7806077AA8A228597C0FFFFE78015
:10F82000A0762A89228597C0FFFFE780C0739307DF
:10F8300005F893F7F70F1307E0072A8C6377F706AD
:10F84000228597C0FFFFE7800072AA8C228597C0AF
:10F85000FFFFE78040712A8D5285832B040097A01B
:10F86000FFFFE780C07239E58357440085440144B7
:10F87000F11793B71700A301F10003473100930775
:10F8800084005A85DE882688D6865286CE8597F0F3
:10F89000FFFFE78000958D4748003EC4230291009A
:10F8A00022C697D0FFFFE780004541011733FFFFD5
:10F8B00067006382A2851306310097E0FFFFE780AF
:10F8C000203F2A84894455D99356C900131649010B
:10F8D00085486A88E6876287858A5182D68597003F
:10F8E0000000E78060AEAA8449BF1723FFFFE7024C
:10F8F000E37B2A8981440144617A916A176BFF1F77
:10F90000130B4B5D97B0FFFFE780C06863C7A4008F
:10F9100022851723FFFF6700A37C832709009399A3
:10F920001400CE9703D507003307450142074183F2
:10F930006364570305C103270B0019C785453E853E
:10F9400097400000E78060E9832709000504CE970F
:10F950002390070085047DB797000000E78060A230
:10F96000832709000504CE972390070065D58145BC
:10F9700097F0FFFFE78080BFF1BF1723FFFFE7028B
:10F98000E37283C7950041112A8A93F7F707A3848E
:10F99000F50032852E89328497C0FFFFE780C05E74
:10F9A00093170501C187635AF004AA89832A0400CA
:10F9B00097A0FFFFE780A05D31E5835744008544B1
:10F9C0000144F11793B71700A301F1000348310078
:10F9D000D68752850147CE862686CA8597D0FFFFF7
:10F9E000E780406BA167F50748003EC42302910001
:10F9F00022C697D0FFFFE780003041011723FFFFA9
:10FA00006700036EA2851306310097E0FFFFE780D1
:10FA1000202A2A8489445DD99767FF1F9387874BE3
:10FA20009C4381CF044997B0FFFFE780A056AA8589
:10FA3000268597400000E78040DA1305040197000F
:10FA40000000E780C0EA228597800000E78000334D
:10FA50008144ADBF1723FFFFE702636483C79500AE
:10FA60004111AA8A93F7F707A384F5003285AE897E
:10FA700032842311010097C0FFFFE780E050931705
:10FA80000501C1876354F0062A8AC145228597C0C3
:10FA9000FFFFE7800036AA8B5285032B040097A056
:10FAA000FFFFE780C04E21E98357440085440144AD
:10FAB000F11793B71700A300F10003481100035793
:10FAC0002100DA875685D2862686CE8597D0FFFF1D
:10FAD000E780405CA1679387270248003EC4230269
:10FAE000910022C697D0FFFFE780E0204101172355
:10FAF000FFFF6700435EA2851306110097E0FFFF3A
:10FB0000E780001B2A8489444DD99767FF1F93879C
:10FB1000673C98433E8901CF044997B0FFFFE780D7
:10FB20006047AA85268597400000E78000CB130533
:10FB3000040197000000E78080DB97B0FFFFE780BB
:10FB4000604595443DD9930521005E8597F0FFFF00
:10FB5000E78020B7AA8435F11C480357210022858D
:10FB60002390E70097800000E78040218327090069
:10FB7000A9D70355210097400000E780A0BD35BFFD
:10FB80001723FFFFE702A35183C795004111AA8AFB
:10FB900093F7F707A384F5003285AE89328497C0C6
:10FBA000FFFFE780603E93170501C1876351F006B0
:10FBB0002A8A228597C0FFFFE780003D2A89528567
:10FBC000032B040097A0FFFFE780603C31E58357DB
:10FBD000440085440144F11793B71700A301F100D5
:10FBE00003483100DA8756854A87D2862686CE8535
:10FBF00097D0FFFFE780004AA167F90748003EC49D
:10FC00002302910022C697D0FFFFE780C00E41017A
:10FC10001723FFFF6700234CA2851306310097E0EE
:10FC2000FFFFE780E0082A8489445DD99167CA977D
:10FC3000C2071167C1831307F7EF8544E362F7FA40
:10FC40009767FF1F938707299843BE8B01CF04490D
:10FC500097B0FFFFE7800034AA8526859740000013
:10FC6000E780A0B71305040197000000E78020C8D3
:10FC700097B0FFFFE780003295443DD11C482285B4
:10FC800081442390270197800000E780200F83A7FD
:10FC90000B00B9D74A8597400000E780A0AB89B731
:10FCA0001723FFFFE70223422A844105B28497000D
:10FCB0000000E780C0C311C5228597800000E7805F
:10FCC000E00B81460146A685228597800000E780EB
:10FCD000C04E1C4C89C7DC4799C3228582971723E5
:10FCE000FFFF670083409767FF1F9387A7FF9C4331
:10FCF000014599C31385070182809767FF1F93878A
:10FD000067FE884382801723FFFFE702C33B9317F8
:10FD1000C600DD8DC2054111C1812A8432C697C05B
:10FD2000FFFFE780A0183246228511829375F60FF7
:10FD300097C0FFFFE780801541011723FFFF670091
:10FD4000C33A1723FFFFE702633679713C083ED2BE
:10FD5000B7070C003ED43C083ED683C79500AE845E
:10FD60002A8993F7F707A384F500A16593853504E5
:10FD7000481097A0FFFFE780A02CC165FD15014446
:10FD8000176AFF1F130A8A16930A400EAE892E8B3C
:10FD90002EC697B0FFFFE780E022420593170401CB
:10FDA0004181C183B24563E9A702C167FD1763873B
:10FDB000F500481097C0FFFFE780400F5010014743
:10FDC0008146A6854A8597A0FFFFE780C04C456124
:10FDD0001723FFFF6700C3303307540383270A0B41
:10FDE000BA9703D6C701630A3601638A3501481002
:10FDF00097000000E78060F1DA85050451BFB28505
:10FE0000EDBF1723FFFFE702832979717C083EC805
:10FE1000B70711003ECA7C083ECC83C79500AA896B
:10FE2000328593F7F707A384F5002E8997C0FFFF6B
:10FE3000E780801585676378F504A165AA84890544
:10FE4000080897A0FFFFE780A01F268597400000C5
:10FE5000E78060ED133415000A04A285080897C0F6
:10FE6000FFFFE780A002A685080897C0FFFFE78094
:10FE7000E00325CC014781461008CA854E8597A02E
:10FE8000FFFFE780404145611723FFFF6700A32480
:10FE9000B30754030327CA0ABA9703D70700631CA2
:10FEA000970003D6270063806505080897000000C7
:10FEB000E780A0E5DE8505042EC697B0FFFFE7804A
:10FEC00060114205931704014181C183B245E3E10A
:10FED000A7FCC167FD17E38FF5F8080897C0FFFF7F
:10FEE000E780C0FC41BFB285F9B7C165FD1501448B
:10FEF000176AFF1F130A8AFF930A80022E8BAE8BAC
:10FF000065BF1723FFFFE702031C18418347170053
:10FF100083460700A207D58FD207D1832390F5002F
:10FF200083472700034717008D45A207D98F918388
:10FF30002310F60097C0FFFFE78060EA1723FFFF5A
:10FF40006700A31A1723FFFFE7024316C1640144A9
:10FF50001769FF1F130989F993098002FD1497B0EF
:10FF6000FFFFE78020076347A40001451723FFFF39
:10FF700067000317330534038327C90A3E95835767
:10FF80000500E38597FE0504D9BF1723FFFFE702AD
:10FF9000E3112A8AAE89B284B68A97400000E780CE
:10FFA00080D819E591473E851723FFFF670043136B
:10FFB0002A894E8597C00000E780E08E2A84638EF0
:10FFC0000A048D476DD103570500C547E31D47FD62
:10FFD0000347F9018546AD47E317D7FC8347450042
:10FFE00081CF4146A6855D0597F00000E780C09E61
:10FFF000814755D9AD4745BF130965012302E50087
:020000040001F9
:10000000CA85268597100000E780606231C1A54748
:10001000E38B0AF82302040079B705C18357050072
:10002000E39247F94146A685190597F00000E7805D
:10003000A09A81472DD99947BDB74E8597000000FA
:10004000E78080F02A84954739DD130955004DBFBC
:100050004146A685231044012311340113051900DC
:1000600097F00000E780A099228597800000E78044
:10007000A0EA81470DBF1723FFFFE702C304797190
:100080007C003ECCB7070A003ECE7C003ED083C742
:100090009500B2842E8493F7F707A384F500130626
:1000A000A1002A892C00268597000000E780A0E5A2
:1000B000A16528088D0597A0FFFFE78060F89040B4
:1000C0008355A10003558100854697000000E78015
:1000D00000ECAA84AA85280897C0FFFFE78000DB10
:1000E0000356A10083558100280897000000E7808F
:1000F000C0C1300801478146A2854A8597A0FFFF0D
:10010000E7806019854748103ED42302910202D649
:1001100097D0FFFFE78020BE45611723FFFF6700F0
:10012000C3FC1723FFFFE70203FA79717C003ECC82
:10013000B7070A003ECE7C003ED083C79500B2844C
:100140002E8493F7F707A384F5001306A1002A89EC
:100150002C00268597000000E780E0DAA1652808DA
:100160008D0597A0FFFFE780A0ED90408355A1008B
:1001700003558100814697000000E78040E1AA8492
:10018000AA85280897C0FFFFE78040D00356A1004A
:1001900083558100280897000000E78000B73008E9
:1001A00001478146A2854A8597A0FFFFE780A00E00
:1001B00048102302910202D402D697D0FFFFE780B5
:1001C00080B345611723FFFF670023F21723FFFF6A
:1001D000E70263EF97000000E78060DB1723FFFF73
:1001E0006700A3F09767FF1F938707B0884382805B
:1001F0001723FFFFE70223ED835725004111AE844B
:100200002A842307B10017F5FFFF130525466C006C
:100210002316F10097A0FFFFE780E04991C42285F3
:1002200097800000E780E0D6FD572310F400130606
:1002300020028145130554009720FFFFE780A0EBC3
:1002400041011723FFFF670043EA1723FFFFE7027F
:10025000E3E579717C003ECCB7070A003ECE7C0016
:100260003ED083C79500AA89AE8493F7F7073285FD
:10027000A384F5001306A1002C0097000000E7807E
:1002800080C803558100114497400000E780A0A971
:1002900015C50355A100014497B00000E780A06098
:1002A00011CD035705008357810045446318F700BB
:1002B000854597000000E780E0F30144216993053C
:1002C0003900280897A0FFFFE78080D7A28528087B
:1002D00097C0FFFFE78080BB0356A10083558100D4
:1002E000280897000000E78040A2300801478146B7
:1002F000A6854E8597A0FFFFE780E0F948104AD415
:100300002302810202D697D0FFFFE780C09E45619D
:100310001723FFFF6700C3DC1723FFFFE70203D9A2
:100320009767FF1F9387079C2A8488432E8915C5EA
:10033000035745038357C4016311F70223260502BF
:1003400023180502410597D00000E780209C630632
:10035000090097800000E78060DB81449769FF1FF8
:100360009389C9B8130A800297B0FFFFE78080C65F
:1003700063C4A4049767FF1F9387879F9C4399C713
:100380000355C40197200000E780C0BD6307090042
:10039000228597800000E780C0A01306400E8145AB
:1003A00022859720FFFFE78000D5FD57231EF4002C
:1003B0001723FFFF6700C3D23385440383A7C90A0D
:1003C0003E95035705008357C4016317F700CA859C
:1003D00097000000E78000E2850479B71723FFFF4C
:1003E000E702C3CC83C795004111AA8993F7F707A9
:1003F000A384F5003285AE8497C0FFFFE780C0B8C4
:1004000085676378F5042A8997400000E780A0910A
:10041000014401CD83D70400314463882701854519
:1004200097000000E78080EF01444E85A2864A864F
:10043000A68597D0FFFFE780609DA167938717048B
:1004400048003EC42302810002C697D0FFFFE78028
:10045000808A41011723FFFF670083C81723FFFF2E
:10046000E702C3C49767FF1F9387C787804329C4E8
:10047000014597C00000E780002181470148C16421
:100480001CDC232E0403232004041769FF1F130917
:10049000E9A501449309400EFD1497B0FFFFE780E2
:1004A00060B2634FA400814517F5FFFF1305857FF8
:1004B00097A0FFFFE78020201723FFFF670043C2BC
:1004C000330534038327090B3E958357C5016387A2
:1004D0009700854597000000E78040E4050475BF5C
:1004E0009357050113D78700A380F50093170501E3
:1004F000C183A1832380E5002381F500A381A500AA
:1005000082801723FFFFE70203BC2300050083C797
:100510001500A300F50083C725002301F50083C75C
:100520003500A301F50083C745002302F50083C70A
:100530005500A302F50083C7650093059500A3034A
:1005400005002303F5002304050032859700000011
:10055000E78040F91723FFFF670023B91723FFFF48
:10056000E702C3B44111E9540DCD85CD93F9C5FF20
:100570002E842A89AA84338AA900B7EA0400631862
:100580009A020D88854411CCB7E704009C5F8297DE
:100590002AC622866C003305390197E00000E78007
:1005A0000046268541011723FFFF670063B383A739
:1005B0008A039104829793170501C183A183A38EB7
:1005C000F4FE93570501238FF4FEA183238EA4FE2E
:1005D000A38FF4FE6DB763E6D5021723FFFFE70292
:1005E00083AEB28741113686BE8536C697E00000DD
:1005F000E780E040B246410136851723FFFF6700E0
:10060000C3AE814636858280838705001387F50057
:100610003D05FD8793F77708834607007D1586061D
:10062000B58FA300F5006307B7007D178347170058
:100630009D83DDB782801723FFFFE702C3A8B7E7DA
:10064000040083A7070932872A863A8582971335E3
:1006500015001723FFFF670043A915C181478DC10E
:100660001723FFFFE70223A6414697E00000E7803B
:10067000003985473E851723FFFF670003A78147A1
:100680003E8582801DCD1723FFFFE702C3A34146AD
:1006900081452A849720FFFFE780E0A541468145F8
:1006A000130504039720FFFFE780E0A40147C1671B
:1006B0002322040438C87CC805451723FFFF6700C0
:1006C000C3A20145828081473DCDB5CD1723FFFFF1
:1006D000E702639FB2842E891306800581452A8430
:1006E0009720FFFFE78020A1CA8524C426859700B4
:1006F0000000E780C0F64146814522859720FFFF34
:10070000E780609F3044A285228597000000E78043
:10071000C0F293040401A285268597000000E780BB
:10072000E0EEA6851305040297000000E78000EEC6
:10073000228597000000E78020F585473E85172336
:10074000FFFF6700839A3E8582801723FFFFE70241
:10075000E3954111E9540DCD85CD93F9C5FF2E8464
:100760002A89AA84338AA900B7EA0400639844035B
:100770000D88814411CCB7E704009C5F82972AC69C
:1007800022866C003305390197E00000E7802027BE
:10079000268541011723FFFF6700839483A78A03FF
:1007A0009104829793170501C183A183A38EF4FE60
:1007B00093570501238FF4FEA183238EA4FEA38FFC
:1007C000F4FE6DB765CD1723FFFFE702238EB284D9
:1007D00011E605451723FFFF670083902A842E89C1
:1007E0000145EDD93C487848B3E6E700E5D6938665
:1007F000F7FFB3B7F6007D17032A4404BA9734C84D
:100800007CC863050A06C14913050A03B389494137
:100810002295637D3601B2862E86A685970000005C
:10082000E780A0DB7C40BE9464C065B7CE862E8690
:10083000CE8597000000E78040DAC114D2944E992B
:1008400023220404A2879306040103C7070003C6FA
:1008500007038507318FA38FE7FEE398F6FE304448
:10086000A285228597000000E78020DD2699C149F6
:100870003306994063EC9900A9DCA686A68513058A
:10088000040397000000E78040D579BF8147B30695
:10089000F4003307F6000347070083C50600850709
:1008A0002D8F2380E600E39437FF3044A285228514
:1008B00097000000E78060D8C1145DBF01458280C9
:1008C0000DC11723FFFFE702038013068005814552
:1008D0009720FFFFE780208205451723FFFF670071
:1008E000C38001458280814749C5C1C51713FFFFF9
:1008F000E702637DFC4141462E84AA846399C704C4
:1009000013860501A2878146C14503C7070003C5B9
:1009100007038507298F3305D600034505008506A3
:10092000298FA38FE7FEE392B6FE3044A285268589
:1009300097000000E78060D0228597000000E780E4
:1009400060F885473E851713FFFF6700037A13851C
:1009500007031D8E814522959710FFFFE780A07940
:100960007C40130700F813060402A2972388E702CD
:1009700051BF3E8582801713FFFFE702C3746D717C
:100980002E84B284AA859010280036899700000032
:10099000E780A0D309EDD55725A050400C40280092
:1009A00097000000E78040E27DD5FD142104F5F4B6
:1009B0002C004A8597000000E78020F3814761DD25
:1009C0003E8551611713FFFF670023721713FFFF66
:1009D000E702636F41112EC432C62C000546970012
:1009E0000000E78080F941011713FFFF6700E36F04
:1009F0001713FFFFE702236D01112A842EC602C8D8
:100A000002CA02CC02CE97E00000E780402BB2463B
:100A10002A86A285080897000000E78060FB13750E
:100A2000F50F05611713FFFF6700236C1713FFFF16
:100A3000E70263697971B2872A8421462308B100ED
:100A400013051101BE853AC436C697E00000E78061
:100A500000FBB24693059101368597000000E780C0
:100A600060A82285141035460C0897000000E78026
:100A700020F62A84224701E921460C103A8597E0A6
:100A80000000E780C0F7228545611713FFFF67006C
:100A9000C3651713FFFFE70203637171AE84AA8574
:100AA0000A85328497000000E78060BB11C90A867E
:100AB000A685228597000000E78020B8814711E1D4
:100AC000C5473E854D611713FFFF6700036217138B
:100AD000FFFFE702435C1D712A8AB289BE84354656
:100AE0008547130511012E8CB68A3A8BC28C468D30
:100AF0002308F10097E00000E78060F010100C0878
:100B00005285231F010097000000E780C0F82A8467
:100B10003DEDA1476313FD089307900591E0E5477C
:100B20003546E2851305110113990A012308F100E6
:100B30001359090197E00000E78060EC1357890022
:100B400093978A00D98F90080C085285231FF100D3
:100B500097000000E78020F42A8415E9A1E4938738
:100B6000FA0091831379F9003EC6631309004149E5
:100B7000668B8144C14B854DB247639F970C6A8653
:100B80008C0033855C0197E00000E78040E7228518
:100B900025611713FFFF6700C35393079004C9F043
:100BA000A547BDBF834701050947C14B2308F10095
:100BB00083471105A58FA308F10093872400814482
:100BC00063E1FB04014714083386E6008C08B38612
:100BD000E400BA95DA9683C6060083C505000507CA
:100BE000AD8E2300D600E390E7FE4147639CE70407
:100BF00090080C08528597000000E780C0E925D1D5
:100C000081A0B3069B00BA871008B305F6009008D0
:100C10003E9603C506000346060085078506298E15
:100C20002380C500E39277FF998F90080C085285C6
:100C3000BE9497000000E78000E68947014749D14C
:100C40002A84B1B790083E96034606001408BE9663
:100C50002380C600850759BFB24785046387971470
:100C600081471808B306F70098083E973386F900C5
:100C700003470700034606008507318F2380E600FF
:100C8000E39177FF90080C08528597000000E780F9
:100C900080E05DF53546E285130511012308B101B9
:100CA00097E00000E780A0D5139704014183939754
:100CB00084002183D98F10180C085285231FF1005E
:100CC00097000000E78020DD25FD8147101833875D
:100CD000F9003E960347070003460600B306FB00F3
:100CE0008507318F2380E600E39277FF65A8180817
:100CF000B306F70098083E973386F90003470700CC
:100D0000034606008507318F2380E600E3E127FFD5
:100D1000CA87639E770990080C08528597000000E7
:100D2000E78060D711FD81479800B306F70090086F
:100D300018103E973E9603470700034606008507B6
:100D4000318F2380E600E39177FF3546E285130576
:100D500011012308B10197E00000E78040CA139712
:100D600004014183939784002183D98F10180C08C4
:100D70005285231FF10097000000E780C0D1E311E6
:100D800005EC814710183387F9003E9603470700AA
:100D900003460600B306FB008507318F2380E6007B
:100DA000E3E227FFC109410BC1BB814785B7940826
:100DB000BE9683C6060018083E972300D700850715
:100DC00089BF638006321713FFFFE702C32C5971F6
:100DD0002A84BE89B28B85473546130511022E8BB6
:100DE000468C4289BA8A368A2300F10297E00000D5
:100DF000E780E0C010180C1022852317010297002D
:100E00000000E78040C963180512A147631FFC0674
:100E10009307900563930900E5473546DA85130586
:100E2000110293140A012300F102C18097E000002F
:100E3000E780E0BC93178A0013D78400D98F90080D
:100E40000C1022852317F10297000000E780A0C450
:100E50007DE1639209049307FA00BD88918391E0D4
:100E6000C144C207C183DE8C814A3EC6414DB247B0
:100E700063E2FA0E6286B3854B01881097E00000AA
:100E8000E78080B54DC93D557DA093079004E3965A
:100E900009F8A54759B7834701050947C14C230005
:100EA000F10283471105B3C7F900A300F10293874C
:100EB0002900814963E1FC04814618103306D700FC
:100EC0008C083387D900B69556970347070083C52A
:100ED000050085062D8F2300E600E390D7FE4147ED
:100EE0006390E70690080C10228597000000E780C9
:100EF00080BA35D189A0B3863A01BA871010B305FC
:100F0000F60090083E9603C50600034606008507D6
:100F10008506298E2380C500E39297FF3387EC4036
:100F200090080C102285BA9997000000E780A0B6BF
:100F30008947014741D165611713FFFF67006319B6
:100F400090083E96034606001410BE962380C60005
:100F5000850779B7B247850A93990A01939D8A005C
:100F600093D909016391570F85473546DA851305F3
:100F700011022300F10293D9890097E00000E78075
:100F800000A8B3ED3D0190000C1022852317B1039A
:100F900097000000E78020B059FD8147A68963EAE9
:100FA000970626860C084A8597E00000E78020A572
:100FB00081471810B306F700100898083E973E9630
:100FC00003470700034606008507318F2380E600AC
:100FD000E3E197FE639FA90590080C102285970016
:100FE0000000E78040AB21F981479810B306F70075
:100FF000900818183E973E960347070003460600E0
:101000008507318F2380E600E391A7FF4109C10CDA
:10101000B9BD18089000B306F7003E963387FC0070
:1010200003470700034606008507318F2380E6004B
:10103000B5B798084E97034707001C10CE9723803A
:10104000E700850941BF85473546DA85130511025A
:101050002300F10293D9890097E00000E780209AED
:10106000B3ED3D0190000C1022852317B1039700CA
:101070000000E78040A2E31005EC814718089000CB
:10108000B306F7003E963387FC000347070003468C
:1010900006008507318F2380E600E391A7FF4146D4
:1010A0000C084A8597E00000E7806095814718109A
:1010B000B306F700100898083E973E9603470700CE
:1010C000034606008507318F2380E600E391A7FFE2
:1010D00090080C10228597000000E780C09B1DD56A
:1010E00099BD7D5582801713FFFFE702C3FD0111F3
:1010F0002A842E8593055100328902C002C202C49F
:1011000002C69304740097F0FFFFE780A03D1D46E0
:10111000A6851305910097E00000E780408E100837
:101120008A854A8597000000E780E09619ED9307CD
:101130001400180883C60700034607008507050743
:10114000B18EA38FD7FEE397F4FE05611713FFFF5F
:101150006700A3F91713FFFFE70243F52E848C41C4
:101160004111AA89838715003289914463D307000E
:10117000A1449757FF1F9387270E9C43A1C7C1CA5D
:101180008D472310F10083C725004A852301F10014
:1011900083C73500A301F10083C745002302F10096
:1011A00083C75500A302F10083C765009305910032
:1011B000A30301002303F1002304010097F0FFFFC4
:1011C000E78040320C404A860A8597F0FFFFE780AF
:1011D00080330328040083564400A6881D088147F5
:1011E0000147E51642868A854E8597000000E78014
:1011F000408E2A8919E5A685228597B0FFFFE780F2
:10120000A0C24A8541011713FFFF670063ED4A86BC
:101210000A8597F0FFFFE780002F6DB71713FFFFD8
:10122000E702C3E82E848C414111AA898387150007
:101230003289914463D30700A1449757FF1F9387D6
:10124000A7019C43A1C7C1C68D472310F10083C7E6
:1012500025004A852301F10083C73500A301F10071
:1012600083C745002302F10083C75500A302F100A4
:1012700083C7650093059100A30301002303F100D8
:101280002304010097F0FFFFE780C0250C404A8649
:101290000A8597F0FFFFE780002783564400032864
:1012A00004008A85858EC2061D08C1822312D400DF
:1012B000A68881470147E51642864E8597000000C3
:1012C000E78060B041011713FFFF670063E14A86C2
:1012D0000A8597F0FFFFE78000234DBF1713FFFF3C
:1012E000E70263DEB335B000011185052A891315C5
:1012F000F601336515012308B10093051101368409
:101300003AC632C03EC442C297F0FFFFE780801D5C
:10131000A2471248425593D68700230BF10093054C
:10132000910193578800A30AD100A30BF100230C6D
:10133000010197F0FFFFE780E01A324702460328D9
:101340000400B337E000835644009207914411C271
:10135000A1444A85A68842860C0897F0FFFFE780E3
:1013600040772A8919E5A685228597B0FFFFE78097
:10137000A0AB4A8505611713FFFF670003D717135A
:10138000FFFFE702A3D201113EC68647B335B00086
:101390008505AA891315F6015D8D2308B100930513
:1013A000110136843A89B28442C446C297F0FFFFE5
:1013B000E780401322489248164593578800A30AB5
:1013C000F1009305910193D78800230B0101A30B32
:1013D000F100230C110197F0FFFFE780A0103247C6
:1013E000104083564400B337E000920703280900F9
:1013F000914891C0A1480C084E8597000000E780F5
:10140000809CAA8401E9835544004A8597B0FFFF78
:10141000E78080A1268505611713FFFF670043CC95
:10142000AA959307F00F171701001307A7A46317D6
:10143000B50013C5F7FF1375F50F828005058346C8
:10144000F5FFB58FBA9783C70700D5B70357450097
:1014500014419307F00F171601001306A6A1369743
:1014600042074183139506014181631BE500AD8F5F
:10147000B29703C50700130515F3133515008280D5
:10148000850603C5F6FFA98FB29783C70700D9BFAA
:101490001713FFFFE70223C3B28736842E86BA866E
:1014A000AA853E85BA8497F0FFFFE7806052634FBC
:1014B0000500228597E00000E78060802A86A686E6
:1014C000A285268597F0FFFFE78080501713FFFF66
:1014D0006700A3C11713FFFFE70243BD5D712A8BAD
:1014E000AE8A17150100130565962C00B284368A62
:1014F000BA893E8997F0FFFFE780C04F2A845DE1FB
:1015000034104146DA85280097F0FFFFE780404C11
:101510002A8449E98547A303F100A6C29307710015
:101520002408BEC4A68685470D462C18281002DC68
:1015300002DED6C0BEC697F0FFFFE78000442A84D3
:1015400035E183477102A6860D4693F7F70723001E
:10155000FA00C1473EDE2C188947281026DCA30379
:10156000F10097F0FFFFE78040412A8405ED4146F6
:10157000A6854E8597D00000E78060488D47A686F7
:101580000D462C182810A303F10097F0FFFFE78009
:10159000C03E2A8401E94146A6854A8597D00000CD
:1015A000E780E045228561611713FFFF670043B3C1
:1015B0001713FFFFE70223B197F70000938707EFA8
:1015C000984383C7470079712A89AE8417150100B3
:1015D000130545880C083AC42306F10097F0FFFF75
:1015E000E78040412A8405ED14104146CA85080869
:1015F00097F0FFFFE780C03D2A8415E114081546E7
:101600002C00081097F0FFFFE780803C2A8401E956
:1016100021462C08268597D00000E780403E228591
:1016200045611713FFFF670043AC1713FFFFE70285
:1016300083A997F70000938767E79C477971AA848D
:101640002E8417150100130565810C083EC697F01E
:10165000FFFFE780203A0DE914104146A6850808EF
:1016600097F0FFFFE780C03605E1140811466C00D3
:10167000081097F0FFFFE780A03519E58347F101D7
:1016800093F7F7032300F40045611713FFFF67008A
:10169000C3A51713FFFFE70203A33688A1488147BC
:1016A0000147E54697F0FFFFE780A0421713FFFFD1
:1016B0006700A3A31713FFFFE702E3A03688A14842
:1016C00081470147E54697F0FFFFE780C06F17139A
:1016D000FFFF670083A11713FFFFE702C39E0111FD
:1016E0002A842E850C0832C697F0FFFFE7808030F1
:1016F00009ED3247970601009386C6741008C1456C
:10170000228597000000E780E0D805611713FFFFEE
:101710006700A39D1713FFFFE702E39A4111C1473A
:101720002EC032C48A8509463EC23EC697F0FFFFEE
:10173000E780A02441011713FFFF6700039B1713E5
:10174000FFFFE70243984111AE8613061009AA85F0
:101750000A8502C002C202C402C697F0FFFFE780FA
:10176000202741011713FFFF670023981713FFFF7E
:10177000E70263953287970601009386A66E2E8650
:101780009305000297000000E780C0D01713FFFF09
:101790006700A3951713FFFFE702E3927971C14732
:1017A0002ACC2ED032D42C080D4628003ECE3ED274
:1017B0003ED602C402C602C802CA97F0FFFFE78005
:1017C000C01B45611713FFFF670023921713FFFF2C
:1017D000E702638F0111AA842E8417050100130507
:1017E000E5688A8597F0FFFFE780C02015E51408BB
:1017F0004146A6850A8597F0FFFFE780601D09ED49
:101800008347E1010347F101A207D98FCA07C983C2
:101810006177D98F2310F40005611713FFFF67006C
:10182000C38C15CD1713FFFFE702E3899747FF1F0E
:101830009387075090439745FF1F9385A54F174502
:10184000FF1F1305E54A97D00000E78000C5174544
:10185000FF1F1305E5491713FFFF670003891745AD
:10186000FF1F1305E54882808DCD1713FFFFE702A8
:1018700083859747FF1F9387A74B944301112E84BD
:101880000A869745FF1F9385E54A97D00000E780B9
:1018900040C60A850294014505611713FFFF6700E2
:1018A000C3847D5582801713FFFFE702C38197D061
:1018B0000000E78080D19747FF1F23ABA74617F5AD
:1018C000FFFF1305E5C997B00000E780C074171348
:1018D000FFFF670083811747FF1F1307A747931771
:1018E000150008433E95FD572310F500828017032D
:1018F000FFFFE702437D2A84084009E51703FFFF45
:101900006700A37E1C4158401CC06313E5005CC007
:101910008347550023200500F99BA302F50097A0FB
:10192000FFFFE780E07CC9BF1703FFFFE7020378F2
:101930009747FF1F9387074498432A8411CB834717
:10194000350093F7070289C70355050089450297BB
:101950001305440197B00000E780403B8355040025
:101960000355E40097300000E780A00C485819C5E3
:1019700097A0FFFFE780C077232A040213058403A2
:1019800097000000E780E0F68144B1499790FFFF9F
:10199000E780806E63CBA4028347340023200404D5
:1019A00093F727FCA301F40000489790FFFFE7801E
:1019B000A06D13161500814522859700FFFFE78073
:1019C00080731703FFFF6700A371B38734030329F4
:1019D000040385043E994A8597000000E78060F182
:1019E0002304090065B78347350093F7070299E39D
:1019F000014582808357E500E39CB7FEC167FD1770
:101A00006316F60005458280054599A81703FFFF78
:101A1000E702636B93170601C187B2842A840149E8
:101A20006359F002835705009DCB01456367F600BB
:101A3000034584003E953325A6001375F50F0DA0D0
:101A40001C4813171900BA9783D70700E38E97FA3B
:101A500005099790FFFFE7802063E343A9FE014556
:101A60001703FFFF670063681703FFFFE7020364C4
:101A7000AE89AA849790FFFFE780C0562A8497D04A
:101A8000FFFFE780A02EAA86014713068401970571
:101A90000000938585E41745FF1F1305E52B9790FC
:101AA000FFFFE780401D2A8925C98C441304C50027
:101AB00022859E0593F5050897A0FFFFE780003D6E
:101AC000CC4083877400E18163DD070493E505085A
:101AD000228597A0FFFFE780603B0D469385440079
:101AE000228597A0FFFFE780803783D504002285F9
:101AF00097A0FFFFE780A03E83D52400228597A012
:101B0000FFFFE780C03D03D6490083A50900228579
:101B100097A0FFFFE780A0344A851703FFFF670007
:101B2000235C93F5F5076DB71703FFFFE702A35991
:101B300001112A84328532C697A0FFFFE780A028D2
:101B40009780FFFFE7802035835704001747FF1F6A
:101B50001307C7393246231BF100930700F8A30D82
:101B6000F1001C471843231AA1008983858BB30712
:101B7000F740B28548083ECE231C0100230D01002A
:101B800097000000E78080EE05611703FFFF670004
:101B9000C3551703FFFFE7026351004101453DC4F0
:101BA0009304C40026853289AE8997A0FFFFE780A1
:101BB000802595452A8A2685035B040197A0FFFFAF
:101BC000E780E021268597A0FFFFE780203F8D4535
:101BD000AA8A268597A0FFFFE7806020268597A028
:101BE000FFFFE780A03D5C48420A135A0A01D297E2
:101BF0005CC423186401814763983A0146054D810E
:101C0000330625419337160013F5F70F1703FFFF2F
:101C10006700034D1703FFFFE702634889692A8BBA
:101C2000AE8B328AB68A81440144314CFD199790BB
:101C3000FFFFE780604463CDA4009790FFFFE7803B
:101C4000A046018D33B5AA001703FFFF6700A34824
:101C50003389840383270B003E9963170A00834767
:101C6000890085043E94E1B703560A00DE854A8563
:101C700033F6C90097000000E780E0F16DD105451B
:101C8000E1B71703FFFFE702034401112A847C0038
:101C90000355E5003ECAB70707003ECC7C003ECEA8
:101CA00097200000E78020082A898545480897A0EA
:101CB000FFFFE780E0399945480897A0FFFFE780DC
:101CC000A016AA844A8597200000E780A0082380F8
:101CD000A4009747FF1F938767219C434166130623
:101CE00006F09396870113D78701558F93D6870007
:101CF000F18E558FA207B706FF00F58FD98F1146D9
:101D00002C00138514003EC497D00000E78020CF3C
:101D10005008A38204008945228597000000E780CF
:101D2000E0E019C9AA851305840397A0FFFFE780A7
:101D3000A0323C4085073CC005611703FFFF6700E8
:101D4000C33A1703FFFFE70203389790FFFFE780CE
:101D5000A0352A8405049790FFFFE780E033330520
:101D6000A402F14791453305F50297200000E78072
:101D700020BA11E565551703FFFF67000337974742
:101D8000FF1F23A1A7FE9790FFFFE780E0312A8481
:101D900005049790FFFFE78020303305A4028945B2
:101DA000060597200000E780A0B669D59747FF1F7A
:101DB00023A2A7FA9790FFFFE780002F2A8405044B
:101DC0009790FFFFE780402D3304A4029747FF1F41
:101DD000239487F89790FFFFE780002D2A8497903F
:101DE000FFFFE780602B930714003385A702974716
:101DF000FF1F2394A7F6970701009387E7CA1747A9
:101E0000FF1F232FF7F40145BDB71703FFFFE702BC
:101E1000E329AA842E8901449749FF1F9389090D5C
:101E2000130A80069790FFFFE78000276347A4000E
:101E300001451703FFFF6700A32A3305440383A767
:101E400009024A86A6853E9597000000E780E0B922
:101E500019E10504C1BF0545E9BF1703FFFFE7020C
:101E60000324AA8A2E8BB28B368C3A8A8144014491
:101E70008149974CFF1F938C6C07130D8006979038
:101E8000FFFFE780602163C9A40011E085494E850A
:101E90001703FFFF670023243389A40383A70C02E1
:101EA0005E86D6853E994A8597000000E780E0B3BC
:101EB0001DC19790FFFFE780201F0544636D45011A
:101EC000D2866286DA851305090397000000E78051
:101ED000A0D411C1854985045DB71703FFFFE70250
:101EE000E31CC16441112A8901449749FF1F93896A
:101EF000E9FF130A8006FD1436C632C42EC297903D
:101F0000FFFFE780601992452246B2466348A4006D
:101F1000014541011703FFFF6700831C330544039C
:101F200083A709023E9509C683473500C18B9DC72B
:101F300091C68347350093F707028DC36306990066
:101F40008357E500639C27010357050001CB63E736
:101F5000E50083478500BA97E3CDF5FA050469BF2C
:101F60001703FFFFE7028314C1642A8901449749DC
:101F7000FF1F9389A9F7130A8006FD149790FFFFAE
:101F8000E78080116346A4001703FFFF6700431535
:101F90003305440383A709023E958357E500638A0E
:101FA0009700630499006396270197000000E7807B
:101FB000E0970504E1B71703FFFFE702C30D896946
:101FC0002A8AAE8A328BB68B8144174CFF1F130CC2
:101FD000ECF1930C8006314DFD199790FFFFE780DF
:101FE000A00B63C6A4001703FFFF6700830E3389AD
:101FF000940383270C028355CA015A863E994A8569
:1020000097000000E780609E31C1814D15A03384A8
:10201000AD038327090303D60B00D68533F6C90029
:102020003E94228597000000E780E0B609E9850D1F
:102030009790FFFFE7804004E3CBADFC01A8228529
:1020400097000000E780E08A23040400850471B74C
:102050001703FFFFE702A3044169AA8A014A174B4D
:10206000FF1F130BABE87D19C14B054C9790FFFF89
:10207000E78080026346AA001703FFFF6700A305FD
:1020800093098006B3073A0383290B02BE9983D7CD
:10209000E900638E270163842A01639A570103A430
:1020A000890301E84E8597000000E780C0BD050A5E
:1020B00075BF83570401639977099304C40026858B
:1020C00097A0FFFFE78020D485452A8D2685835C75
:1020D000040197A0FFFFE78080D0268597A0FFFF2F
:1020E000E78060E862056185635905048D452685B2
:1020F00097A0FFFFE780A0CE8945268597A0FFFF28
:10210000E780E0CD8945268597A0FFFFE78020CDB9
:102110008545268597A0FFFFE780A0CD8347050072
:10212000094793F7F707639AE7009945268597A033
:10213000FFFFE78000CCA30285014848337D2D01D5
:10214000231894016A9548C40040A1BF1703FFFFFC
:10215000E70263F737E404008327041D829797475B
:10216000FF1F83C7A7C51715FF1F1305653AA300F7
:10217000F5008327441C82978327841C814613061D
:10218000F00F8145014582971703FFFF6700E3F5D4
:102190001747FF1F130787B218439745FF1F83C5D3
:1021A000E5C19747FF1F9387E7BF83468703034631
:1021B00097036397D5009747FF1F2381C7C082808D
:1021C00083C587010347A7036317B6009747FF1F1F
:1021D0002386E7BE828003C687016317C70097473F
:1021E000FF1F238DD7BC828083C68701130750024F
:1021F0006319D700930760021747FF1F2300F7BC3E
:10220000828083C68701130660026315D600930798
:102210007002DDB783C7870155BF9747FF1F9387BC
:1022200067B8D44B0947638DE6081703FFFFE70241
:1022300083E91749FF1F130929B43E848347090026
:10224000918B9DCFB7E4040083A7041D829783A7D9
:10225000441C1745FF1F1305A5B2829783A7841C52
:1022600081461746FF1F0346A6B381450145829765
:1022700021C583470900ED9B1747FF1F230EF7AECB
:102280008347040093F7F70F85CB91471747FF1F4C
:102290002324F7B297000000E78080EB970000004E
:1022A000E78040EFB7E70400BC4F41469145174532
:1022B000FF1F0345A5AF82971703FFFF6700E3E207
:1022C00082801703FFFFE70203E08D474111630699
:1022D000F504C5476308F50285476310F502974783
:1022E000FF1F238FA7ACB7E70400BC4B930500107A
:1022F0001745FF1F034585AB829741011703FFFF79
:102300006700A3DE85471747FF1F230BF7AAB7E730
:102310000400BC4B93050020E1BF9747FF1F938744
:1023200067A8D44B1147638DE600B7E7040083A785
:10233000071D8297B7E70400BC4B930500044DBF0F
:1023400005491747FF1F232927A783C7070032C660
:102350002E8493F7F70FD5D3B7E4040083A7041DA9
:102360007D141374F40F8297E37689FCB245994784
:1023700003C61500E3F0C7FCFC4409061745FF1F20
:10238000130545A48297BC48930500081745FF1F15
:102390000345C5A1829779BF1703FFFFE702A3D2C8
:1023A0001747FF1F130707A04047184B1C409746CD
:1023B000FF1F23AFF69E6316E4001747FF1F232B72
:1023C000F79E130584FE9790FFFFE780C0AA035590
:1023D00064FF9780FFFFE780407397A0FFFFE780CF
:1023E00020D11703FFFF670043D01703FFFFE70269
:1023F00083CD9747FF1F9387E79AD84BDC4789C760
:1024000097000000E78080F985471747FF1F2325C5
:10241000F79A9747FF1F9387678A9C4393050002AB
:102420001745FF1F0345859883C787031747FF1F7D
:102430002306F798B7E70400BC4B82971703FFFF0A
:102440006700A3CA9747FF1F23A0A79682801703A0
:10245000FFFFE702A3C537E404007C4CA145174504
:10246000FF1F0345A59482977C48A1451745FF1F90
:102470000345C5939744FF1F9384C4928297DC441D
:1024800089EB97000000E78080D91703FFFF670002
:1024900023C503D567FF9780FFFFE7800067AA8900
:1024A0006DD1D84891476310F7027C4C9145174590
:1024B000FF1F0345A58F82977C4891451745FF1F55
:1024C0000345C58E829703A9490103D409018947B1
:1024D000B7E904001747FF1F2320F78E83A7091DC4
:1024E00021044204829783C784011715FF1F130537
:1024F000250261191717FF1FA30CF70083A7491CBA
:10250000418082979747FF1F238C078A83A7C91CA6
:10251000814609469375F40F4A85829711E99747DA
:10252000FF1F83C7279A89C79700FF1FE780E06ACC
:10253000B7E70400BC4F2146A1451745FF1F0345DF
:10254000E586829799B71703FFFFE702C3B793F7B2
:10255000052001112E8481CF97000000E78020E93B
:102560001345042005611703FFFF670003B893F7C5
:102570000510A9CF9744FF1F9384C482DC489700BD
:102580000000E78020C11737FF1F13072773184388
:1025900083C78401034787036318F700DC4489C7B6
:1025A00097000000E78080DF85471747FF1F23253E
:1025B000F780B7E70400BC4B930500021735FF1FF7
:1025C0000345C57E82971345041069BF93F705083C
:1025D000BDC79737FF1F83C7F77EE91719469735A1
:1025E000FF1F9385457E1305D10093F4F70F17392C
:1025F000FF1F0349297D97C00000E7804040939763
:102600000401C1831737FF1F1307477C231DF10007
:10261000231CF1009737FF1F9387C7783ACE3ACA39
:10262000D8432306010009CBDC43931589015408E4
:102630000D46E185680082971345040825B793F796
:102640002500A5C39737FF1F9387C775D84B8947C8
:102650006306F7029737FF1F83C7077213F7270038
:1026600011EF918B99CFB7E70400BC4F1306000A16
:1026700089451735FF1F034565738297134524006D
:10268000D5B59737FF1F938767639C4383C787033D
:102690001737FF1F2304F77297000000E78060DB05
:1026A000F1BF93F7050281CB97000000E78060DA65
:1026B0001345040245BD93F7850081CB97000000C8
:1026C000E780E0D21345840071BD93F7150081CBFC
:1026D00097000000E780A0B41345140061B593F79C
:1026E000450081CB97000000E78060B313454400AC
:1026F00095BD93F7050495C39737FF1F83C7876A76
:1027000091CB97000000E780A0A491471737FF1FE7
:102710002324F76A13450404B1B593F70501014575
:10272000E38207E49737FF1F9387C767D84B91472A
:102730006310F7049737FF1F938707649C4313D7F1
:1027400027008583D98F858B91E7B7E7040083A79E
:10275000071D8297B7E70400FC4F91451735FF1F0F
:102760000345C564829785471737FF1F2326F76403
:1027700013450401C5BB9737FF1F2385A7748280CB
:102780001703FFFFE70223949737FF1F23A2076277
:102790009737FF1F23A0076285471734FF1F1304D5
:1027A000E4511737FF1F2329F7601C4083C78703B5
:1027B0001737FF1F2304F7609790FFFFE78000940F
:1027C00029C59717FF1F23A9A7D41C401705000090
:1027D0001305A5D783C787031737FF1F2300F75EAD
:1027E0001717FF1FA306F7D29737FF1FA38C075AAF
:1027F000B7E7040083A7070882979737FF1F23874F
:10280000A75A1703FFFF6700438EB7C7898E9387C8
:1028100067ED1717FF1F2321F7D045BF1737FF1F9D
:1028200003474758795555E79737FF1F93878757D1
:1028300003C7170005079736FF1FA385E65603C792
:1028400017008D463377D7029736FF1FA38CE654C7
:1028500083C617001737FF1F13074746184393F621
:10286000F60FA9EE834787031737FF1F2308F75496
:1028700085471737FF1F2307F7529737FF1F9387A7
:10288000A74F9C430145998BA9E71703FFFFE70278
:10289000838337E404007C48C1451735FF1F034597
:1028A000E55082973C4885451735FF1F0345055085
:1028B000829701451703FFFF6700238383C7170033
:1028C00085466395F6008347970379BF8347A7033F
:1028D00061BF82809737FF1F83C7C74CA1CF17F313
:1028E000FEFFE702437E37E404009737FF1F238B88
:1028F000074A7C4885451735FF1F0345254B8297BE
:102900007C4C91451735FF1F0345454A82977C480B
:1029100091451735FF1F0345654982973C48C145DE
:102920001735FF1F034585488297014517F3FEFFC2
:102930006700A37B7955828017F3FEFFE702A37837
:102940002A84035565FF9780FFFFE780001C9737B7
:10295000FF1F93872745D847BE841DEF9790FFFF41
:10296000E78040789C48232004009DEB9737FF1FA9
:1029700023A287449737FF1F23AC8742B7E70400A1
:10298000BC4B89451735FF1F0345454282970145DA
:1029900017F3FEFF67006375630A8700184375BF6E
:1029A00080C39737FF1F23A78740C9BF7955CDB78D
:1029B00017F3FEFFE70223719737FF1F9387C75076
:1029C00088432326050023240500510597A0000015
:1029D000E780C03317F3FEFF6700237117F3FEFF94
:1029E000E702636E1734FF1F1304044E1C404111AD
:1029F00099CF9C472302B5002AC61CC1970000004E
:102A0000E78040FB1C409C4B99C3324582974101B3
:102A100017F3FEFF6700636D17F3FEFFE702A36A7B
:102A20004111444D328532842EC69790FFFFE780D6
:102A300080532AC422859790FFFFE780E05403A8C3
:102A40004400630C0800B2458357440018402246F6
:102A500083D54500AA8626850298410117F3FEFF1B
:102A60006700A36817F3FEFFE702E365404D1DC84A
:102A700008C097050000938565031305440197A0DE
:102A80000000E78040169737FF1F9387E7439C437A
:102A9000014589E79737FF1F23A8874217F3FEFFF9
:102AA0006700A3647D55DDBF17F3FEFFE702A36156
:102AB000011168009305F00F02C602C802CA02CCD9
:102AC00002CE97000000E780A0F1056117F3FEFF3A
:102AD0006700A3619737FF1F9387073F9C43D84741
:102AE000A1679D076319F70217F3FEFFE702A35DD5
:102AF000011132859790FFFFE780E046230AA1008D
:102B00008145680097000000E78080ED056117F3BC
:102B1000FEFF6700835D82809737FF1F9387C73A68
:102B20009C43D847A167938777036319F70217F38C
:102B3000FEFFE7024359011132859790FFFFE780BE
:102B40008042230AA1008145680097000000E780C9
:102B500020E9056117F3FEFF67002359828097374C
:102B6000FF1F938767369C43D84795476316F70442
:102B700017F3FEFFE7022355011132853284979047
:102B8000FFFFE780403E230AA10022859790FFFFC8
:102B9000E780803F83574400231BA10081453ECC42
:102BA0001C4068003ECE97000000E78060E30561AE
:102BB00017F3FEFF670063538280930785FF8DC381
:102BC0008327C5FF91CFDC4B81CF17F3FEFFE702D0
:102BD000834F032585FF829717F3FEFF6700E350BD
:102BE000828017F3FEFFE702034E2A843285979016
:102BF000FFFFE7804037BD4763EBA700184493779A
